:020000040800F2
:1000000000A00020610601080DC4000895F6000854
:100010000BC4000809C4000807C400080000000061
:1000200000000000000000000000000005C40008FF
:1000300003C400080000000001C400081BB1000850
:10004000C9060108C9060108C9060108C906010850
:10005000C9060108C9060108C9060108C906010840
:10006000C9060108C9060108C9060108C906010830
:10007000C9060108FD2E0008372A0008C906010834
:10008000C9060108C9060108C9060108C906010810
:100090006DC40008C9060108C9060108C90601089F
:1000A000B9A60008F9A60008A9A6000821A700081B
:1000B000E9A60008D9A60008C9A60008C9060108D3
:1000C000C9060108C9060108C9060108C9060108D0
:1000D000C9060108E5A80008D9A80008C906010852
:1000E00029B10008C906010879F50008C906010808
:1000F000C9060108C9060108C9060108C9060108A0
:10010000000000000000000000000000C906010817
:10011000C9060108C9060108C9060108C90601087F
:10012000C9060108C9060108C9060108C90601086F
:10013000C9060108C906010800000000000000000F
:10014000C9060108C9060108C90601080000000027
:10015000000000000000000000000000000000009F
:100160000000000000000000C9060108C9060108DF
:10017000C9060108000000000000000000000000A7
:0801800000000000C90601089F
:100188002DE9F04F2DED068B6B4D6C4B2B60A1B01C
:1001980000236B600DF006FE18B90DF025FE09F07E
:1001A80037FB09F0F3FB664B664C1A7842F0010204
:1001B8001A70654A4FF47001C2F88810002208923C
:1001C8000992226842F4803222600493236803F47F
:1001D80000330993089B01330893099B1BB9089BBB
:1001E800B3F5A04FF2D1236813F4003318BF0123ED
:1001F8000993099B012B69D0DFF84C81534BC8F850
:100208000C30636AAB60636A514EDFF870A1DFF8A7
:10021800709143F080736362636943F4FC0320AF19
:10022800636103238DF8323041F6FF7327F8503DA0
:100238004FF09040394602F075FE4FF6FF73304696
:100248003946ADF8303002F06DFE4248394602F0CA
:1002580069FE4148394602F065FE4048394602F0D9
:1002680061FE39463E4802F05DFE384607F058F810
:100278000C9B3C4AB3FBF2F33B4A3C4913603C4BB2
:1002880000221A603B4B5960F02188F823109A60CD
:1002980007221A60DFF8EC80DAF80830C8F8003076
:1002A80099E80300636987E8030043F480236361E6
:1002B8004FF48053B3610C980DA902F033FED8F8BF
:1002C800003013F0080F564629D163E02A4B12225A
:1002D8001A606368636063686360636843F480639B
:1002E8006360636823F47C136360636843F4881372
:1002F8006360236843F0807323602268114B920186
:10030800FBD55A6822F003025A605A6842F002028A
:100318005A60636803F00C03082BFAD16CE79AF86B
:100328009031012B36D8044A9AF89131926812F02C
:10033800805A00F0D7872DE09008002039910008F6
:10034800A82600200010024000ED00E00005FA0594
:100358000004004800080048000C0048001000484D
:100368000014004840420F00182000203F190100E7
:100378001C20002010E000E000200240D8110020DE
:10038800C438010830260020C34B002283F891218D
:1003980009F098FC64200AF0B2FE4FF48C72BF4852
:1003A800002112F08AF9E369BD4A43F00703E361CB
:1003B800A36943F4E123A361636943F4C023636140
:1003C80002F1E00E937BD07B4FEAD30C03F00701D8
:1003D800536803EB8C038900D3F820C04FF00F0A51
:1003E80088400AFA01F12CEA01011962196A1032EF
:1003F800084372451862E5D10022AA4900235354E4
:1004080001320E2AF9D1DFF8CCA20AF11A02FF2133
:1004180099540133072BF6D1A34AA44B1360DFF894
:10042800B8B2A34A0393032111705846002124222D
:1004380012F043F914228BF800209E49039BD8F848
:10044800008001228BF8182096F805B081F800B0DA
:10045800A3F5F171CAF824109749A3F591730B60BD
:10046800964B03EBCB0318F0200F5B78CAF82830C3
:1004780018BFCAF828200023914A40F2DC5122F81C
:1004880013100133082BF7D1384600211C2212F033
:1004980014F9BBF10E0F04D00BF0EF0BBBF1080FF2
:1004A80002D101238DF84030022006F0C7F818B1B8
:1004B8004088003018BF0120C8F340038DF836305B
:1004C800C8F380138DF83830C8F340338DF83030D6
:1004D800C8F3C03300F001008DF8333018F400631E
:1004E8008DF8350004D096F884315F1E7B427B413D
:1004F8008DF83430C8F300438DF83930AB6AB6F85C
:100508004401ADF84400003318BF01238DF83A3098
:10051800C8F300538DF83B30B6F84631ADF83E309D
:1005280018F4805FB6F8523118BF5B48ADF83C301C
:10053800C8F380438DF83730B6F850311CBFB0F897
:100548004C01ADF84400B3F5FA7FADF8423084BFF2
:100558000023ADF844305B4896F8D43185F82C3048
:10056800002385F82D3043709DF8403008F00101D4
:10057800002BC8F3C0028DF831108DF832200CBF63
:100588000023022301B902B1013309EB83094FF0BB
:10059800000AD9F808309A1E1A3303920593039B70
:1005A80033F8022F03934FF6FF739A4200F0358118
:1005B800110A0229CBB202D19DF8301003E00129BB
:1005C80004D19DF83110002900F022819DF83A10DD
:1005D800D2B261B19DF8401049B99DF8381009B1FF
:1005E800111F01E0A2F10801012998BF04232C4F33
:1005F8009DF83B104FEA02194F4431B19DF8401065
:1006080019B9043A032A40F2EC80012B66D1FF2382
:1006180085F8743085F87530214BC5F8847003EB84
:1006280009024FF00008517B50688DF82A1002F13A
:10063800080B1289ADF828200AA9022285F87880CB
:1006480006938DF82B2085F83080C5F83480C5F8DE
:100658003880C5F83C80C5F8708085F8768085F8C4
:10066800778002F05FFC069B9BF8021053F80900A4
:10067800424602F089FB38460EF0F0FB124B134954
:10068800C5F88830124BC5F88C30C5F890803846CC
:100698000A1D0AF0C3F8BBE0D81100205020002042
:1006A8008C5601089C08002064240020CA130020EE
:1006B800B91100201C040020E421002088590108F9
:1006C8002A110020BD0800207927000818090020F9
:1006D800592800089008002068240020022B46D1E1
:1006E8005FFA8AF21C2101FB02FC05EB0C089D4A0B
:1006F80088F879A0012188F8781002EB09014FF0F9
:10070800000B91F80DE0486888F87AB001F108020A
:100718000989ADF8281088F882B00AA9C8F8847049
:10072800CDF81CC08DF82AE006928DF82B3002F027
:10073800F9FB8C4B069A53F8090091785A4602F057
:1007480023FB38460EF08AFBDDF81CC08649874A31
:10075800C8F888206144864AC8F88C20C8F890B048
:1007680038460A1D0AF05AF80AF1010A50E0032B2C
:1007780035D19DF83730DFF82C82DFF82C923BB169
:1007880098F82EB0384608214FF6FF7200231AE079
:10079800BDF8422098F82EB0BDF84430B2F5FA7F83
:1007A8000BD97449B1FBF2F23846082192B202F033
:1007B800E2FB714B49F82B000AE07049B1FBF2F2F9
:1007C8003846012192B202F0D6FB6D4B49F82B0056
:1007D800C36098F82E30013388F82E3018E0042BC7
:1007E80016D195F82D80BDF83C20644B93FBF2F2AE
:1007F8003846BDF83E30012192B202F0BCFB95F8B4
:100808002D3005EB88080133C8F8580185F82D30DC
:10081800039B059A93427FF4C2AE95F82D2085F884
:100828007821584A584B92F800E0AEF11702002799
:10083800022A1F709C461AD86B6A3B44D3ED007A93
:10084800F5EE407AF1EE10FA02D1AB6A63BB26E00E
:100858004E4A07EB02080FCB88E80F009CF80030DF
:1008680010370133C02F8CF80030E5D1EDE7484B45
:1008780013F83E908CF8009003EBCE03D3F804A055
:10088800BAF1000FE1D04F45DFDA404A3B0103EBF4
:10089800020853440FCB013788E80F00F3E73D4FB8
:1008A8003B68DD0425D41DE03B4B3C4A13F83E0071
:1008B800107003EBCE035D68002DF0D00023834257
:1008C800EDDAC3EBC3016A18DFF8E080D2F80090D4
:1008D80041F8089001EB08079188B9809279BA71BC
:1008E8000133ECE70EF0EF03082BDFF8C48020D1CA
:1008F80022E09CF80020012AF4D9294B03EB0212CC
:10090800103210339342EDD053ED047AB6EE007AEC
:1009180067EE877A43ED047A53ED057A67EE877AB6
:1009280043ED057A53ED037A67EE877A43ED037A50
:10093800E7E7BEF10E0F0BD198F8003043F0100333
:1009480088F80030BEF1180F34D10AF0AFFD31E05D
:1009580098F8003023F0100388F80030BEF1190F22
:10096800F2E700BF8C560108180900208D2E0008F8
:100978005127000800127A007928000840420F0029
:10098800692800081C0400201720002058030020B4
:100998008859010830260020643D01087021002094
:1009A80060030020900800202020002071210020F2
:1009B800001900200AF05EFD3B68DFF84093C34D44
:1009C80058035EBFC24B01221A70049B049A1B781D
:1009D80043F0040313704FF48063ADF828301123FB
:1009E8008DF82A3063694FF0020A43F480230AA97C
:1009F8008DF82BA04846636102F094FAB54BB64ACD
:100A08001A6000200AF094FBB44B1D60636943F43C
:100A180080236361E36943F40013E361236B23F0EC
:100A280010032363236B43F010032363D9F82030AA
:100A380023F07063C9F82030D9F8203043F0806380
:100A4800C9F82030D9F8203023F07043C9F8203095
:100A5800D9F8203043F08043C9F82030032300241C
:100A68008DF82D30484640230AA98DF82E408DF880
:100A78002F400A938DF82CA006F0C0FD802348462D
:100A88000AA90A9306F0BAFD2B6823F001032B602C
:100A98002A68934B13402B60924B2B612B6843F0D1
:100AA80001032B60AC60EC60AC60AB688E4C43F427
:100AB8000043AB602B682B606B6823F0784323F40A
:100AC80000436B602B6843F001032B60B4F8583186
:100AD800002B40F08984B4F95A21002A40F084841C
:100AE800B4F95C21002A40F07F8400210C227F4861
:100AF8007F4E11F0E2FD002114227E4811F0DDFD49
:100B08007D4B002201201A7005F0BAFF337843F0BC
:100B180002033370794B4FF480529A610A25DFF84B
:100B2800DC91B9F814309BB283F48053A9F81430DF
:100B380019200AF0E4FA01200AF0FAFA19200AF05A
:100B4800DEFA013D00200AF0F3FA15F0FF05E6D1C0
:100B58004FF48053C9F81830694B9FED6A8AD3F86F
:100B68000090DFED698A99F80C3000EE103AB8EE83
:100B7800C00A20EE080A08F0F1FD644B83ED000A74
:100B8800634B4FF06E521A605A4BD3ED047A614BA7
:100B980067EE887AB7EE007AC3ED007A99F80030EC
:100BA80007EE903AF8EEE77A5B4BC7EE277AB0EE9D
:100BB800680AC3ED007A77EE677A584BC3ED007A7E
:100BC800574B83ED027AC3ED008AC3ED018A554B7A
:100BD80083ED027AC3ED008AC3ED018A08F0BEFDF9
:100BE800B0EE408AB0EE680A08F058FD20EE006AC0
:100BF80068EE086A66EE007A4B4BE6EE887AFF21CB
:100C08001B2220EE087AC3ED007A67EE007AF0EE38
:100C1800675AD7EE085AE7EE087A28EE468AC3EDF7
:100C2800015AA6EE808AC3ED027A83ED038A3F4B10
:100C38001D703F4B184611F040FD3E4ADFF8F8E0C2
:100C480012680570012112F0020F8EF800101FBF04
:100C5800417003218EF80010022118BF81705107DE
:100C680041BF9EF800104D1C8EF80050032548BF68
:100C7800455412F00A0F73460ED09EF80020042146
:100C88008154511CC9B205254554D11C0232D2B237
:100C98008EF800100621815439688D0641BF1A78F4
:100CA800551C1D70072548BF85540A0608D51A78B3
:100CB80009258554951C0132D2B21D700A25855428
:100CC8006579082D3AD00E2D41D137E00054004007
:100CD80088080020B026002005A90008FC10002084
:100CE800FFE0CF007A25E000D81100203023002053
:100CF800A826002004220020A001002000040048AB
:100D08008002002035FA8E3C000000007C020020A2
:100D180034020020380200209402002084020020BF
:100D280098020020880200206C020020F6010020B2
:100D380009110020FC180020081100201A7802F17F
:100D4800010E83F800E04FF00B0E00F802E01A786D
:100D580011F0040F4FF00C0C00F802C002F1010E64
:100D68001CBFDFF8C8C202325FFA8EFE83F800E0CB
:100D78001FBF8CF80020944A4FF0100C02F80EC0E8
:100D88001A7802F1010E5FFA8EFE4FF0120C11F480
:100D9800806F83F800E000F802C00ED094F80CC20F
:100DA800BCF1000F09D0DFF884C202328CF80020B1
:100DB800854A4FF0130C02F80EC01A7811F4007F20
:100DC8004FF0140C00F802C002F1010E1CBFDFF84E
:100DD8005CC202325FFA8EFE83F800E01FBF8CF817
:100DE8000020794A4FF0150C02F80EC0182D13D1C7
:100DF8001A784FF0160E00F802E002F1010E5FFAC1
:100E08008EFE4FF0170C00F80EC002F1030E0232EE
:100E1800D2B283F800E085540A0341BF1A78551C02
:100E28001D70192548BF8554CD0541BF1A78511C3E
:100E380019701A2348BF835400219822634811F07F
:100E48003CFC0DF0DEFC624B624A1A60624BB4F85F
:100E58004E111980614900230B808B7060490A602C
:100E6800B4F8962190B25F4921F813000133122B90
:100E7800F9D13B68D8045CBFB4F89C0108801B0713
:100E880040F1058194F89031062B00F2FA80DFE8F2
:100E980003F004070E3D5979790045F2F05201E05C
:100EA80042F6F822504B1A800DF061FDE8E007EE9B
:100EB800902ADFED4E6A4C4BB8EEE77ADFED4C7ABC
:100EC800E7EE267A42F6F82119800023FCEEE77A4D
:100ED800484A17EE901A42F823100133122BF7D123
:100EE800454A46491160464A4020137005F08EFC79
:100EF800002800F0C68001234FF0070C90F900008D
:100F0800404A8DE8081040213F4BB4E0364B42F68A
:100F1800F8221A80384B3D4A1A60394B102240207B
:100F28001A7005F073FC002800F0AB8001234FF025
:100F3800000E90F90000364A8DE8084040214FF431
:100F4800E13398E0284B42F6F8221A802A4B314ABE
:100F58001A602B4B082240201A7005F057FC002815
:100F680000F08F800123002590F900002A4A8DE8BF
:100F7800280040214FF4E13305F020FA274BC3F84D
:100F88007C017AE0184ADFF8A890DFF8A8C0DFF8FB
:100F9800A8E0234D234842F6F821118018490C2275
:100FA800062B0A704AD0002389F800308CF80030EC
:100FB8008EF800301B232B701B4B027005221A7011
:100FC8004FF4E13547E000BF09110020C02300209D
:100FD800E40A002060130020E80A00207C26002094
:100FE80070260020481B0020D6020020CDCCCC3F24
:100FF8000000B0C4001B00209C000020056D000804
:101008005C240020716F0008A0860100F16C0008C4
:10101800C56E0008D96C0008796E00089008002099
:101028008E1B00208B1A00208F1B00200811002027
:101038008C1A00208D1B00208C1B0020002189F8B1
:1010480000108CF800108EF8001002702121BF4AA1
:101058002970BF4D1370BF4BBF4A1A60402005F07E
:10106800D5FB70B101210023BC4A90F900008DE83E
:101078000A0040212B4605F0A1F9003018BF0120D5
:1010880028B9082008F092FBB24BB54A1A603B68B1
:10109800B44A13F4804F1FBF08211170AD49B248FC
:1010A80018BF086042F20101194003F0010003F47F
:1010B800005581B1AD4944F6206EA1F800E025B194
:1010C80008211170A349AA4D0D6020B10C2111709F
:1010D800A049A84808601178043951701A065ED5ED
:1010E800A548A64DDFF8ECA2C0F880A14FF0000992
:1010F8004946152200F5C270DFF8DCB285F8019088
:10110800C5F80490C5F8089011F0D7FAAAF10503BC
:101118004846CBF8003009F035F9994B02201B6896
:10112800EB6005F073FB18B9802008F03FFB2EE058
:101138006B7890F805E093490C2202FB0312527871
:10114800724504D00133DBB2042BF4D900236B7051
:10115800DBF800306A781B7890F90000002B4FF01C
:101168000C0303FB021314BF4FF0030E4FF0010EE4
:1011780000225B78CDF800E00192022105F01EF90B
:10118800814B18600028CFD0012009F0FBF87F4B75
:1011980018687F4B00F5C5721A6009F0A1F93B6821
:1011A8005B055DD5744D7B4BD5F89CA1C3F800A0B9
:1011B800042005F02BFB0421C5F8A00105F000FB75
:1011C800754B85F8A4010820C3F800A005F01EFBA4
:1011D800724BDFF808921860082105F0F1FA002137
:1011E80085F8A5012C22484611F067FA8E227C2347
:1011F80089F801204FF07D0BE02289F8003089F84A
:10120800032089F82BB0DFF8D89103932C22002112
:10121800484611F052FA039B89F800308A2389F86E
:1012280001301020A02389F8033089F82BB0C5F8C5
:10123800A8A105F0EBFA1021C5F8AC0105F0C0FA39
:1012480085F8B0012020C5F8B4A105F0DFFA202107
:10125800C5F8B80105F0B4FA85F8BC010BF018FD23
:101268003B684F4A13F4002318BF0123137009F099
:101278001FFF4C4B18606379052B02BF4A4B4FF494
:10128800C8721A80494B4FF47A721A8098F8003065
:10129800474A43F0080388F80030137823F0020324
:1012A80013703A6840F6020313406BB1414B424A4F
:1012B8001A60424B03221A70414B01221A70414AAC
:1012C80000231380404A1380A3683B603F4B0122F0
:1012D8001A70337863F07F03337021B0BDEC068B4E
:1012E800BDE8F08F013B092B3FF654A8D9F8180048
:1012F800386039464FF0904001F014FE4FF09043AB
:1013080008229A613C2009F0FAFE96F891319A4534
:10131800BFF63AA82E4A4FF0904B4FF4805108235D
:101328009161782006910592ABF82830039309F073
:10133800DBFE059A0699039B11857820CBF81830B7
:1013480009F0D2FE0AF1010ADFE700BF8F1B002077
:1013580090D003009C000020F56B0008596D000830
:1013680095F500085C240020396D0008D60200209D
:1013780089F50008496D0008900800207C010020CC
:1013880054260020EC340108D81C00203C11002011
:101398003C0B0020F0180020481900209419002068
:1013A8008E240020A8020020F60A0020C42600206F
:1013B800CC260020E8180020521300204C190020E9
:1013C800EC000020D0100020D21000208808002057
:1013D80000040048CA1300209C01002018190020AE
:1013E8004D19002035FA8E3C1BB208EE103AB6F9BA
:1013F8005A315FED047A344A09EE103AB6F95C3195
:10140800B8EEC88A08EE903A28EE278AB8EEC99A4C
:10141800F8EEE88A0021B0EE480A29EE279A68EE2D
:10142800A78A117008F09AF9F0EE409AB0EE480ACF
:1014380008F034F9B0EE408AB0EE490A08F08EF9A7
:10144800B0EE40AAB0EE490A08F028F9F0EE40AA3A
:10145800B0EE680A08F082F9B0EE409AB0EE680A79
:1014680008F01CF960EE296A68EE097AF0EE665A0F
:10147800E7EEAA5A154B29EE296A28EE007AC3ED41
:10148800035AF0EE465A2AEE400AE7EE6A5AE6EEAA
:10149800AA7AA6EE6A7A29EE0A9A83ED010A28EE5C
:1014A8004A8A2AEE290A83ED009AC3ED02AAC3EDFF
:1014B800045A83ED058A83ED067AC3ED077A83ED36
:1014C800080AFFF712BB00BF58000020241C0020A8
:1014D800804A2DE9F04F15687F4C05F59C43203371
:1014E8002DED028B23607D4B196889B011F4804F74
:1014F8000592984605D10EF097F810B92379013373
:101508002371774B1F78C7B1764A1268954240F22B
:10151800FF80013F1F70FBE0D9F800307248072DAB
:1015280098BF595D714B88BF29461B689847032DA2
:101538000BD904EB45050137E8806B4BDFF8C89100
:101548001E78FDB2AE42E7D820E0D9F8002005F1B8
:101558000E0302EB83039988DA880028E9D04FF458
:101568007A73401A5843531A90FBF3F040F6C903B4
:1015780000F57A70984205DC40F2EE239842B8BF35
:10158800184601E040F6CA0080B2D2E70F23277957
:1015980084F82A3094F82B300193032594F82C30E2
:1015A800B7FBF5F505EB45057D1B0393D9F800302E
:1015B8000293DFF858A1EBB204930025B54254DA40
:1015C8004B49019B31F815B04FEA450953B90EF064
:1015D8002BF828B1039B002B08BF4FF0000B01E04C
:1015E800DDF804B0029B988A584502D8D88A584535
:1015F8000ED2E8B20DF0CCFF032D8346DFBF94F87E
:101608002AE00120A8402EEA0000D8BF84F82A006A
:101618000EF00AF818B1374829F800B021E0049B09
:1016280094F876002AF813B028B9022F15D92A4958
:10163800012081F87600BAF80210BAF800000844D0
:10164800BAF8041008442C4980B229F8010000B205
:10165800032190FBF1F080B200E05846254929F8B3
:10166800010001350AF1060AA8E794F82A20234860
:10167800234BA2F10F0EDEF1000242EB0E0284F8BA
:1016880090206AB11F4A1268570109D40268D968C4
:101698009A60521AC82A3BD9012283F8212037E0E0
:1016A80002689868DA605B68121A9A4288BF144B1D
:1016B8004FF0000184F82B1088BF83F82110002513
:1016C800B54225DAE8B20DF063FF0A4B23F815009E
:1016D8000135F5E7AC260020500A0020302600200E
:1016E80078260020742600205C2400209C0000201E
:1016F800560A0020481B0020C80A00205426002053
:101708007C26002004110020702600207E0A00207C
:10171800D8F80030DE0405D58C4B1B68DD0701D4F2
:101728000DF049FB8A4B1A68937A2BB3013B894920
:10173800127B31F813301AB1C3F53B6308339BB2FF
:101748001BB2A3F57A73B3F57A7FA8BF4FF47A7307
:1017580023EAE37307EE903A9FED7F7A7F4AF8EE2B
:10176800E77AC7EE877A9FED7E7A67EE877AFCEE96
:10177800E77A17EE903A1380D8F80030794F13F4CF
:10178800807F00F00481059BDFF8E0911A68764BB2
:101798009A4205D999F8022012B9012289F8022043
:1017A80099F80220002A00F0F280704A3E7892F8F8
:1017B8002150664A681E454211684541002DC1F313
:1017C8008063C6F380060193924614BF4FF0000B66
:1017D8004FF0030B99F82020052A00F2D280DFE8A9
:1017E80002F0034D527584A1002E3AD0D4F894002B
:1017F800B4F8981005F0ADF8012809D15C495D4AA4
:1018080009681268C988642000FB0122C9F8102001
:10181800019B6BB1564A126812794AB10AF0AEFDC3
:10182800032289F820204FF47A72C9F81C20D1E7E6
:10183800002D40F0A6804F4AD9F8101010684B4A86
:1018480088420AD902920AF099FD029A032182F885
:10185800201040F6B831D161BCE7012182F8201090
:10186800B8E7019B4FF4806013B107F08FFF01E0E8
:1018780007F07CFF0022C9F8102082E0002D46D135
:101888000AF07CFDA6E725B1052289F82020012071
:1018980000E0284666B1D4F89420D1892D4A1180F9
:1018A80051809180324909684988D1804FF0020BF4
:1018B800304A1168D9F81420914201D8002E5DD120
:1018C80047F23052C9F81C20032221E03A7842F04E
:1018D80002023A700DF06FFA264AD9F81C10126805
:1018E8000A44C9F81820042212E0224A9DB111685E
:1018F800D9F81820914244D91F4A12781AB9DAF84F
:101908000020D1073DD43A7822F002023A7005222D
:1019180089F820205EE71268D9F81C100A44C9F833
:1019280018202EE01249134A09681268C9886420F1
:1019380000FB0122C9F810204FF48060002289F8CA
:10194800202089F8032007F011FF43E70411002045
:1019580070260020481B002000007A4458110020FF
:1019680000C07F44CC260020404B4C007C26002041
:1019780024220020542600200100002000287FF4A3
:1019880029AFBBF1000F02D0584605F03DF8AD4D28
:1019980005F5C470B5F84E1104F0DBFF834668B94D
:1019A8000AF0DEFCA84BC3F800B0C3F804B0C3F8D3
:1019B80008B0A64B00221A605A609A603B785A0712
:1019C80036D5D8F80030DB0632D5A14B1B78DE06B9
:1019D8002ED4A04B1B7893B195F8E031BBF1000FE2
:1019E80015D17BB19C4B1A68D4F89C309B1A002BFC
:1019F80008DA0DF0E0F9994B83F8A0B018E0BBF1D4
:101A0800000F0DD1102004F0FFFF01230EE03BB1C1
:101A1800914A12684FF47A7101FB0323C4F89C3091
:101A280094F8A03023B104F0D9FF002384F8A03043
:101A3800002295F8DEA195F8DF11B5F898E1B5F820
:101A48009AC11346864E019636F912009B087045D6
:101A5800C4BF63F07F03DBB201326045B8BF43F017
:101A68004003042AEED194F8A1207C489A4205D17B
:101A780090F8A220F92A04D8013200E0002280F868
:101A8800A22084F8A130734B764E1A789946E2B9B1
:101A98003368D80708D5BBF1000F16D13B78D907B2
:101AA80013D50DF005F810E03B785A070DD56B4BB0
:101AB80093F82B304BB16C4BDB7833B911B10DF087
:101AC8007AF902E0BBF1000FF9D094F8A230634A2A
:101AD800DFF8A4B1142B40F0898099F800301AF18E
:101AE800000A18BF4FF0010A6BB392F8A1305F2BC0
:101AF80011D13B7803F0040303F0FF0113B10DF09B
:101B08005AF908E00B200391029204F07DFF029A33
:101B1800039982F8A210BAF1000F14D094F8A130FA
:101B28007D2B10D13B7803F0040303F0FF0213B1BF
:101B38000DF041F907E00B20029204F065FF474BD6
:101B4800029A83F8A2203B7803F0040303F0FF0114
:101B5800002B4BD194F8A130404A572B11D1434B5D
:101B68004FF47A721A80D8F800301B0601D508F0B5
:101B780019FD3F4B1B6813F0080337D13D4A13800A
:101B880034E0D8F80000400717D55A2B15D192F841
:101B9800A3302BB1012382F8A31082F8A43025E0EA
:101BA80092F8A53083F0010382F8A5300BB10C2020
:101BB80000E00D2004F028FF18E05D2B00F0FA8407
:101BC8005B2B00F015855E2B00F01485562B01D198
:101BD80008F078F899F80030002B00F0BE8494F8EB
:101BE800A1306F2B40F0B3840CF062FFD8F80030BE
:101BF8005A0752D594F8A530184A93B13B785B0739
:101C08000FD5019BB3F90610B5F89831994208DD54
:101C1800336813F0010302BF3221A2F8A81082F83A
:101C2800A5303368D80329D594F8AA200B4B2AB9D4
:101C380093F8A32012B93222A3F8A820012384F82C
:101C4800AA302AE0D8110020901F0020EC1F0020A5
:101C5800001900200100002054260020500A00200E
:101C6800481B0020041100207C260020C4260020E8
:101C7800FC180020CC1100203C11002094F8A3305F
:101C8800B64A53B13B7803F0040303F0FF0123B9CC
:101C9800012382F8A31082F8A430DBF800A0002307
:101CA80033600AF17B090AF1CB0B99F8002099F807
:101CB800013019F8010C9A420BD2494604F012FE81
:101CC80038B119F8022C012303FA02F233681343DE
:101CD800336009F10409D945E7D1A14B1B7843B119
:101CE800A04BA14E1A6812F0020F994640F03883B3
:101CF8002FE30AF1CA060AF589793278737816F85B
:101D0800010C9A4225D2314604F0ECFD08B3B378B1
:101D180096F804E0954A96F803A090480C21013BF8
:101D280001FB0E4103EB43031344D1F8B0209A4260
:101D38000FD0C1F8B030002390F8DC20C1F8B430DF
:101D4800012303FA0EF322EA030381F8ACA080F81A
:101D5800DC3006364E45D0D1854B1E68854B1B6856
:101D6800039394F82B300493834B0193002302933D
:101D7800019B1B68002B00F0E18293F800A0BAF1E8
:101D8800000F00F0DB82019A039952688A1A002A30
:101D98000CDB01F5FA7201994A60029901228A4026
:101DA80094F8DC1021EA020284F8DC20049A002A64
:101DB80000F0C482019A597812F8042C0432D2B285
:101DC800002940F07A826D4931F91210B5F8962150
:101DD80002F1C800814202DD93F802B015E0C83A6A
:101DE800914203DA9978C1F1000B0EE0029A0123BF
:101DF800934094F8DC2022EA030384F8DC30039B48
:101E0800019A03F5FA73536098E294F8DC30029A69
:101E18001341D90700F19282BBF1000FCCBF022019
:101E2800012004F015FE0AF1FF33DFF83091132B7F
:101E380000F27C82DFE813F01400250037004B0025
:101E480064006B00E7004A01B101DF010F027A026A
:101E58004B005A006B00E7004A01B9001C018101E0
:101E680096F80090D944B9F1FA0FA8BF4FF0FA09D3
:101E780029EAE979304686F8009004F019FD012036
:101E88000FE096F80190D944B9F1640FA8BF4FF05C
:101E9800640929EAE979304686F8019004F008FDDA
:101EA80002204946D4E196F803A0DA44BAF1640F57
:101EB800A8BF4FF0640A2AEAEA7A86F803A03046F7
:101EC800D9F8E01004F0AAFC03205146C0E171796A
:101ED80059446429A8BF642121EAE17171710D2078
:101EE80004F068FDBAF10D0F00F0208231795944F1
:101EF8006429A8BF642121EAE17131710E20A7E1AC
:101F0800B179594481F30801B1710520A0E1D9F8EC
:101F1800E4301A78022A39D107EE90BAB8EEE70A07
:101F2800DFED187A93ED097A80EE270A30EE070A7A
:101F3800B5EEC00AF1EE10FA07D4B4EE670AF1EE76
:101F480010FAC8BFB0EE670A01E09FED0F0A83EDF3
:101F5800090A0F2004F018FD23E000BF500A0020F2
:101F6800CD26002004110020FC1800204C3901085F
:101F78005C11002054260020000B0020481B002084
:101F880000007A440000C8420000000099785944D3
:101F9800C829A8BFC82121EAE17199700F2004F06F
:101FA80009FDBAF10F0F00F0C181D9F8E4301A78B1
:101FB800022A1ED107EE90BAB8EEE78A5FED0F7AD3
:101FC80093ED080A88EE278A38EE000AB5EEC00AB3
:101FD800F1EE10FA07D4B4EE670AF1EE10FAC8BFB2
:101FE800B0EE670A01E01FED180A83ED080A122017
:101FF80056E159785944C829A8BFC82121EAE17196
:102008005970122024E1D9F8E4301A78022A20D134
:1020180007EE90BAB8EEE70A5FED267A93ED0C7AF0
:1020280080EE270A30EE070AB5EEC00AF1EE10FA84
:1020380007D4B4EE670AF1EE10FAC8BFB0EE670A2B
:1020480001E01FED2F0A83ED0C0A102004F09CFC20
:102058000AE0197B5944C829A8BFC82121EAE171BF
:102068001973102004F0A6FCBAF1100F00F05E817D
:10207800D9F8E4301A78022A1ED107EE90BAB8EEE1
:10208800E78A5FED407A93ED0B0A88EE278A38EEEF
:10209800000AB5EEC00AF1EE10FA07D4B4EE670AEA
:1020A800F1EE10FAC8BFB0EE670A01E01FED4A0A68
:1020B80083ED0B0A1320F3E0D97A5944C829A8BF45
:1020C800C82121EAE171D9721320C1E0D9F8E430BE
:1020D8001A78022A22D107EE90BA1FED570AF8EEB5
:1020E800E77A87EE800AD3ED0F7A30EE270AB5EE4D
:1020F800C00AF1EE10FA09D45FED5E7AB4EE670A11
:10210800F1EE10FAC8BFB0EE670A01E01FED620AEF
:1021180083ED0F0A112004F037FC0AE0997D594439
:10212800C829A8BFC82121EAE1719975112004F0D6
:1021380041FCBAF1110F00F0F980D9F8E4301A78AF
:10214800022A20D107EE90BA1FED730AB8EEE78A8B
:1021580088EE008A93ED0E0A38EE000AB5EEC00A42
:10216800F1EE10FA09D45FED797AB4EE670AF1EE70
:1021780010FAC8BFB0EE670A01E01FED7D0A83EDD3
:102188000E0A14208CE0597D5944C829A8BFC821DB
:1021980021EAE171597514205AE0D9F8E4301A7827
:1021A800022A1ED107EE90BAB8EEE78A5FED8B7A65
:1021B80093ED0A0A88EE278A38EE000AB5EEC00ABF
:1021C800F1EE10FA07D4B4EE670AF1EE10FAC8BFC0
:1021D800B0EE670A01E01FED940A83ED0A0A0920B0
:1021E8005EE0D9785944C829A8BFC82121EAE1711D
:1021F800D97009202CE0D9F8E4301A78022A1ED1C7
:1022080007EE90BAB8EEE78A5FEDA27A93ED0D0A71
:1022180088EE278A38EE000AB5EEC00AF1EE10FA09
:1022280007D4B4EE670AF1EE10FAC8BFB0EE670A39
:1022380001E01FEDAB0A83ED0D0A0A2030E0597B5F
:102248005944C829A8BFC82121EAE17159730A2055
:1022580004F0B0FB6AE0D9F8E4301A78022A22D1F7
:1022680007EE90BA1FEDBA0AB8EEE78A88EE008A40
:1022780093ED100A38EE000AB5EEC00AF1EE10FA36
:1022880009D45FEDC07AB4EE670AF1EE10FAC8BF60
:10229800B0EE670A01E01FEDC40A83ED100A0B20B7
:1022A80004F072FB42E0D97D5944C829A8BFC8216F
:1022B80021EAE171D9750B20CAE7012936D198784E
:1022C800BD4B33F91230B3F5617F05DB40F63302BD
:1022D8009342A8BF134601E04FF46173BAF10C0FA3
:1022E80024D14FF4966292FBF0F0B44AA3F56173DF
:1022F80093FBF0F35FFA83F913784B4516D0B9F1E5
:10230800040F34BF4B4602231370AD4A0AFB035334
:1023180003F2E663136007F015FB5046494604F0E4
:1023280049FB09F10100C0B204F092FB029A0123B3
:10233800934094F8DC20134384F8DC30029B01338B
:102348000293019B0C330193029B042B7FF410AD85
:10235800C6E4D8F80030DA0510D59A4BDB786BB1B3
:1023680033689B070AD5984B1B8813F0010A0AD1DA
:1023780009F0F6FF012007F009FA04E0012007F050
:10238800F5F9012300E00023D9F8002050070DD506
:1023980063B1012007F0EAF98B4B1B88990708D431
:1023A80009F0DEFF022007F0F1F902E0022007F051
:1023B800DDF933689A0609D4D9F800301B0540F1D5
:1023C80094804FF4807007F0E1F992E07F4BDFF8DA
:1023D800F8A11B7813F0020F53D07D4B1B78042B08
:1023E8004FD9D9F8003013F4007B0FD0BAF8003079
:1023F800DE063AD4102007F0C9F9202007F0B6F914
:102408007448011D08F022F802232AE0BAF8006097
:1024180006F01006B6B22EB1102007F0A7F9012673
:1024280084F8E8B0D9F80030580512D5D4F8EC3063
:1024380069495A89B1F90030002BB8BF5B42934211
:1024480007DAB1F90230002BB8BF5B429342C0F201
:10245800F880BAF80030990608D5202007F086F9E8
:10246800002384F8E830012600E0002694F8F030D4
:10247800BBB90E2004F0C8FA584B012283F8F020AB
:102488000FE0BAF8003003F03003002B94D010208E
:1024980007F06CF9202007F069F9002384F8E83088
:1024A80001E0002E88D04E4B002003F1280603F1EE
:1024B80050044C4A002122F810104B4A596022F867
:1024C80010100432716022F8101000221A609A600D
:1024D8003260B26022606160A26014331436143432
:1024E80000287FF469AF0120E3E74FF4807007F01C
:1024F8003DF96B79082B01D00E2B02D1402007F053
:1025080035F9D8F800305A0540F1B18095F80C3209
:102518001BB93B7813F0040F03E0D9F8003013F42B
:10252800002F0BD0314B00221A703C200CF068FAB7
:10253800002800F09C800BF02BF9F6E70AF0A8FBC6
:1025480009B0BDEC028BBDE8F04F0CF05AB9BAF1F6
:10255800000F02D07E2B3FF447AB94F8A130972BA5
:1025680006D11E4B4FF4C872A3F8A620FFF73EBB56
:10257800A72B06D1154A137843F004031370FFF70D
:1025880035BB0022BB2B079201D1022303E0B72BF6
:1025980004D14FF6FE73ADF81E303BE0BE2B01D1DF
:1025A800022304E0BD2B7FF421AB4FF6FE73ADF898
:1025B8001C302FE001201EE0481B002010230020C3
:1025C8005C1100207C260020C4190020001900207E
:1025D8000619002064110020D0110020500A0020A4
:1025E800440B0020C6260020BC0B002061240020DC
:1025F800022000E003205FFA80F909F1FF3385F833
:10260800E43607F005F907F0C1F9484604F020FA66
:10261800FFF7ECBADBF80030BDF81C10B3F858200F
:102628000A44A3F85820BDF81E10B3F85A200A44EB
:10263800A3F85A2007F046FB002384F8A230FFF7DE
:10264800D5BABAF800309B063FF510AF202007F046
:102658009DF80948094B011D1A685B6843600260D0
:1026680007F0F4FE064B012683F8E860FEE609B0A1
:10267800BDEC028BBDE8F08F6C110020081900201A
:10268800500A0020026BC168034610B5406942B188
:102698001A6C8C1A013A005D08BF0A46C0B21A6467
:1026A80010BD1A6A805C01328A4228BF0022C0B27B
:1026B8001A6210BD436B13B190F844007047836AE7
:1026C800406A1B1A584258417047036B13B15B6844
:1026D800016C01E0C369016A8B423CBFC2689B1868
:1026E800581AC0B27047836A8169426B1944D16035
:1026F800416A99429DBF0169CB1A5360CB1A96BFB4
:102708000023536083624FF0000380F8443013685D
:1027180088BF816243F0010313607047436A82698E
:10272800D154436A02690133934228BF00234362AC
:10273800436B1BB11B68DB0705D4D4E7026D136834
:1027480043F080031360704710F80A3C0133DBB292
:102758000A2B84BF10F8131C044A00F80A3C82BFF5
:10276800002322F8113000F80A3C70476C1B002047
:10277800334A136C90681944081A40F68C2398421F
:1027880070B513469160D06051603BD9127893F9C7
:1027980045108A4210460BD1111F082908D893F812
:1027A8004610182901D8013103E083F8442002E0DB
:1027B800002183F8461093F944402149A24219D1D7
:1027C80091F84740B4B10C310024944206DA1D4D0B
:1027D80051F8046F25F814600134F6E70C2805D089
:1027E8001849002421F810400130F7E7164801780D
:1027F8000131017083F84520002201211A7083F805
:10280800471070BD92F84710C9B1A0F2EF2440F20A
:10281800DA518C4208D811780B2905D80B1D0131E3
:10282800117042F8230070BD002283F84720074B3F
:1028380003F13002002143F8041F9342FAD170BD1E
:10284800C00800206C1B00206C010020CC08002070
:10285800024A136C0133194411647047C008002000
:10286800024B53F820301B68196070472020002065
:10287800064B53F820301A681B89A1F57A71594321
:102888004FF47A7391FBF3F1116070472020002018
:10289800F0B5046D8668236823F00103236083790B
:1028A800054613F0020F40790CBF4FF0000E4FF4AD
:1028B800005E13F0040F14BF4FF48067002710F078
:1028C800010F14BF042100218307206820F00100B4
:1028D8002060626822F440524EEA02026260226876
:1028E80022F4B05323F00C0348BF41F008013B43E6
:1028F8000B432360A36895B023F44073A360684634
:1029080004F00EFD284B9C4201D10C9B0EE0274B96
:102918009C4201D10D9B09E0254B9C4201D10E9BA5
:1029280004E0244B9C420CBF0F9B109B2268A879A3
:10293800170448BF5B00B3FBF6F206FB1233B3EB98
:10294800560F236828BF01321E0441BF4FF6F073AB
:10295800C2F34201134041EA03026B7992B213F0C9
:10296800020FA28100F0010114BF4FF400320022CF
:10297800DC0748BF42F480322B6D11B159680A4315
:1029880002E0596821EA02025A609A6801074CBFBE
:1029980042F0080222F008029A601A6842F0010226
:1029A8001A6015B0F0BD00BF003801400044004077
:1029B80000480040004C0040417169E7816067E7CA
:1029C800026D036B70B50446D5699BB9A90611D58C
:1029D800C36A1BB1908C80B298470BE0E169928C76
:1029E80040694E1CD2B2E6614254E169E268914204
:1029F80028BFE361616BA1B92A0612D5636AA26A8E
:102A08009A42236D09D0501CA669A062B25C1A854F
:102A18002369984205D3A16203E01A6822F0800274
:102A28001A602B0742BF236D08221A6270BD0D4B36
:102A38000D484FF400525A600C4A11684FF6FE7365
:102A48000B401360426B11684FF6FE730B40136026
:102A5800426A836A9A4200D045E6012380F84430EE
:102A6800704700BF000002402C1F002044000240B5
:102A78002DE9FF471D46B24B9DF8306098428846C5
:102A8800174640F08680AF4BAF4A1A60AF4A5A618A
:102A980002F580729A614FF48072DA601A61AC4A6A
:102AA8001A63143A5A63A2F54842203ADA640432A7
:102AB8009A649F601865A74B9A6942F480429A61AC
:102AC8005A6942F001025A6102238DF80C3003233F
:102AD80016F0010A8DF80D304FF000038DF80E3016
:102AE80014BF0223012331078DF80F301BD54FF097
:102AF80090444FF40079CDF808908AF001038DF8DE
:102B08000E30636A23F0F0036362636A43F0700374
:102B18006362204602A904F071FDBAF1000F28D1C2
:102B2800C4F8189025E0AA0710D504A94FF400733B
:102B380041F8083D4FF09040436A23F0F0034362A8
:102B4800436A43F07003436204F058FDEB0710D565
:102B580004A94FF4806341F8083D4FF09040436A60
:102B680023F470634362436A43F4E063436204F00E
:102B780045FD0E238DF804300022012301A88DF8AD
:102B880005308DF806208DF807306E4C0CF048F9AA
:102B980075E0714B984240F0F380704B6A4A1A60B6
:102BA8004FF48072DA601A616D4A5A6102F58072D8
:102BB8009A61684A9F601865D36943F40033D3610A
:102BC80002238DF80C30032316F0010A8DF80D301E
:102BD8004FF000038DF80E3014BF02230123340791
:102BE8008DF80F301AD55F4C4FF02009CDF80890BA
:102BF8008AF001038DF80E30236A23F470032362F0
:102C0800236A43F4E0032362204602A904F0F6FC99
:102C1800BAF1000F24D1C4F8189021E0A8070ED506
:102C280004A9202341F8083D4E48036A23F47003A1
:102C38000362036A43F4E003036204F0DFFCE9077C
:102C48000ED504A9402341F8083D4648036A23F0FD
:102C580070630362036A43F0E063036204F0CEFC2E
:102C680026238DF804300022012301A88DF80530B1
:102C78008DF806208DF807300CF0D2F8374CC4F8E0
:102C88002C80012384F8443000232362E361A3628B
:102C980063626571A760A6712046FFF7F9FDEA0730
:102CA80029D5206B00B3D4F84C80E668676904F036
:102CB800ABFA236B216D1A6822F4FF4222F07002EE
:102CC80042F48552B6B21A605E60C3F80880DF60CD
:102CD8001A6842F001021A608A6842F040028A606B
:102CE8005B689BB2236406E0236D20221A621A688F
:102CF80042F020021A60AB073BD5606B002833D046
:102D0800A66C256904F080FA636B1A6822F4FF4206
:102D180022F0700242F4845242F010021A60ADB2FE
:102D280000225D609E60DA60196841F00201196056
:102D38005A605A60226D936843F08003936018E0EC
:102D4800003801402C1F002088390108C40B0020DE
:102D5800580002400010024000440040D81E0020E5
:102D6800C40D0020000C0048226D136843F0800356
:102D78001360226D136843F001031360204600E0DE
:102D8800002004B0BDE8F0873D4B1B78012B30B51F
:102D980014BF00240324B1B9036A23F001030362BA
:102DA8008169036A21F0F30123F00A0341F001016C
:102DB80042F001021A4341EA041181610262836907
:102DC80023F00C031BE004291DD1016A4FF6EF73B1
:102DD8000B4003628169056A120121F473414FF6C1
:102DE8005F7342F0100241F480712B4092B213439A
:102DF80041EA043181610362836923F4406383619A
:102E08008369836130BD0829016A1AD14FF6FF63CF
:102E18000B400362C169036A9BB289B223F4206341
:102E280043F4807321F0F30143EA022241F00101E7
:102E380092B241EA0411C1610262C2694FF6F373AA
:102E480019E04EF6FF730B400362C369056A40F64A
:102E5800FF41194045F6FF732B4043F4805343EA82
:102E6800023241F4807192B241EA0431C1610262D6
:102E7800C2694FF2FF331340C361C369C36130BDF8
:102E8800BC08002038B510F80E2C50F8043C044655
:102E980052B9012200F80E2C20F80C1C997A1868F7
:102EA8000222BDE838406FE730F80C2C20F80A1CE5
:102EB800891A89B220F8081C074A10F80F0C002557
:102EC80022F8101004F80E5C1868997A2A46FFF761
:102ED8005BFF04F8065C38BD6C1B0020044B53F8FC
:102EE80020301BB107289CBF1B681960704700BFC2
:102EF800E8090020084A13689B050BD5074B0021F9
:102F08001970074908684FF6FE7303400B604FF4C9
:102F180000735360704700BF00000240CB260020BA
:102F28003000024073B506460D46002401232A8866
:102F3800A34013421AD0AA78009302F003038DF835
:102F48000430EB78022B03D0032B0CBF032301239F
:102F58008DF805303046C2F301136946C2F3810289
:102F68008DF806308DF8072004F048FB0134102C4A
:102F7800DCD102B070BD2DE9F743DFF81C9299F857
:102F8800004405468E460068114616469846724625
:102F9800631C89F8003407F0C7FB2B89ADF80430AF
:102FA80001A9022368688DF806308DF80730FFF70D
:102FB800B9FFAB7A2A6809F2044724012744494635
:102FC8000C2B00F2B780DFE803F007B5B5B53EB5C6
:102FD800B5B56AB5B5B59300136ADFF8C0C123F07B
:102FE80001031362136AD2F804E0906920F4803078
:102FF80020F07300624540F0700012D00CF5006CB0
:1030080062450ED00CF5406C62450AD00CF5806C18
:10301800624506D00CF5806C624502D043F003038C
:1030280007E023F00E032EF4407E43F003034EF432
:10303800807EC2F804E09061C2F83480136293691C
:1030480043F0080329E0136ADFF850C123F01003A6
:103058001362136AD2F804E0906920F0807020F4BB
:10306800E640624540F4E04006D00CF5006C62454D
:1030780002D043F0300307E023F0E0032EF4406E63
:1030880043F030034EF4806EC2F804E09061C2F859
:1030980038801362936943F4006393614AE0136ACA
:1030A800DFF8F8C023F480731362106AD2F804E0E2
:1030B800D369624523F0730343F0700306D00CF51F
:1030C800006C624502D040F4407007E020F4606074
:1030D8002EF4405E40F440704EF4805EC2F804E086
:1030E800D361C2F83C801062D36943F0080320E042
:1030F800136ADFF8A8C023F480531362106AD2F869
:1031080004E0D369624523F4E64343F4E04340F422
:10311800405003D00CF5006C624501D14EF4804E4E
:10312800C2F804E0D361C2F840801062D36943F466
:103138000063D3612B7B1BB1536C43F4004353648E
:1031480013889BB243F001031380AB7A0C2B19D878
:10315800DFE803F0071818180B1818180F181818B4
:1031680013000B1902F134000AE00B1902F13800C0
:1031780006E00B1902F13C0002E00B1902F14000D5
:10318800C3F804040C443846A4F80C64C4F80824B2
:1031980003B0BDE8F08300BFC40B0020002C014041
:1031A8002DE9F04FC14BB3F90610C14B2DED028B41
:1031B8001F687A8987B0914201930EDBB1F5FA6FE7
:1031C800FC79BDBF8B1A6343A2F5FA64C4F16404A9
:1031D800BCBF93FBF4F4643400E06424B54AB64BF6
:1031E800B2F896A192F95E211868049092B20592FD
:1031F800054600220293AD4B33F912300393CAEB14
:10320800030303F2F31640F2E63086424FEA420B1C
:1032180003D8002BB8BF5B4201E04FF4FA73022ACF
:10322800049E4FF064002FD096F811E1BEF1000F14
:1032380004D07345CCBFCEEB03030023DFF8C0E214
:1032480093FBF0FC6FF063093EF81C809B4E09FB72
:103258000C390CF1010C3EF91CE00FFA88FCCCEBA0
:103268000E0E0EFB09FE9EFBF0FEC64426F80BE090
:10327800BE1836797343924E93FBF6F364339BB2D0
:10328800634393FBF0F02EE096F812E1BEF1000FD5
:1032980004D07345CCBFCEEB03030023DFF84C8288
:1032A80093FBF0F06FF0630C0CFB003938F910E079
:1032B8000130002B38F91000CEEB000000FB09F9B3
:1032C800BDF8140099FBFCF9CEEB090919FB00F9CC
:1032D8007A48A0F80490B879B8BF5B42434378486D
:1032E80093FBF0F064306B78764E4FF0640E4343F6
:1032F80093FBFEF3B354744EEB7A434393FBFEF314
:10330800B3546B7D6D4E5843704B90FBFEF0022A10
:1033180098546F4B0FD183F802E0039B53450EDBA3
:10332800644CB4F89821914215DBB1F5FA6FA8BF47
:103338004FF4FA6110E09C54039B534504DA36F8C5
:103348000B305B4226F80B300132032A05F10105E8
:103358007FF451AFE4E71146891A4FF47A73DFF826
:10336800A4E1564D59436FF06303C2F5FA6264272E
:10337800B1FBF2F191FBF7F23EF8120003FB0211E8
:10338800013203B23EF91220D21A514391FBF7F3EE
:103398000344F3804F4B1B885B0635D54E4B4F4A91
:1033A8001B881288DFED4E7A9B1A1BB208EE103A82
:1033B800B8EEC88A28EE278AB0EE480A06F0CEF999
:1033C800F0EE408AB0EE480A06F068F9B5F9023026
:1033D80006EE903AB5F90030F8EEE66A07EE903A54
:1033E80020EE667AF8EEE77AA7EEA87A67EE807A9A
:1033F800BDEEC77AE6EEA87A17EE103AFDEEE77A48
:103408002B8017EE903A6B80364D2B689F0740F162
:10341800A180354B354F1A687B6945F20721D31ACD
:103428008B4240F397807A6104F0D6F9304BDFF88D
:10343800D8901A78032A9846B9F8003022D10A2B76
:103448002AD90023282088F8003007F058FE04F015
:10345800C3F9284B188804F0A9F9274B1A68D378C0
:1034680090FBF3F001300828244BA8BF08201870FF
:10347800537980B213FB00F33B83137913FB00F0FD
:10348800788309E00A2B07D803231C4A88F8003000
:10349800002313703B837B8398F80030144A012B78
:1034A8003DD033D3022B4CD054E000BF481B002042
:1034B8005C110020D81100203C110020D011002000
:1034C8000CFEFFFF00200020C61000201420002062
:1034D800801F0020C4190020CC1100208C2400205B
:1034E80035FA8E3C30260020AC260020B81000208B
:1034F8004C190020481C0020E8180020EC0000208F
:10350800321A00201A1A0020EC1800203A8BB9F859
:1035180000309A421EDD012388F800300FE0B9F828
:1035280000107B8B8B4202DD022313700FE09B4B54
:103538001B8B0133994202DD002313700AE0082037
:1035480006E07B8BB9F8002001339A42E3DC0720C0
:1035580003F05AFA2F683D0570D5914B8F4D1A68C4
:10356800EB69C3EB020845F20723984566DD8D4BEE
:10357800B6F906B0D3F80090EA6199F80A30B4F8C1
:103588004E11894E012B4FF47A70ABF57A7B98FB7C
:10359800F0F803D03BD3022B19D03AE02A6A08216D
:1035A80092FBF1F3D31A00222B62AA8493FBF1F366
:1035B80040F6E4429BB25343B9F80820C2EB1333F8
:1035C8005843B9F9063090FBF3F0306021E0774BAF
:1035D800B9F808A01B78C6F800A0580719D5744890
:1035E80003F0B7F920B917F0100F18BF4FF0000B10
:1035F80032220BFB0BF393FBF2F3B9F906205B4481
:103608005A434FF47A7392FBF3F3534400E00023D8
:103618003360D5E90A013368664A03FB08F84FF4BA
:103628007A7398FBF3F810EB080041EBE87100237C
:10363800C5E90A010CF04CFA5F4B18605F4E33681D
:10364800D90427D53A0622D55D4B1B789B071ED592
:103658005C4B187804281AD900225B4BD71805212F
:10366800951C4FF00A0E122AD154E9B287F801E0EE
:1036780004D0B0EB510F2A46EFD800E014215A18B5
:10368800322002F8010CFF225A540F2000E00A20D1
:1036980003F0BAF94D4D2A68002A50D04C4B4D4FD3
:1036A800186839688142984649D84B4BDFF83491FD
:1036B80019785268E1B94FF0010A83F800A0B9F807
:1036C8000030D35C23B3504607F032FD434B83F8F8
:1036D80000A00BF0B5FFB9F80030CBB92B681B7808
:1036E800053B534514D807F0E3FC3D4B18600FE049
:1036F8004FF0000A83F800A0B9F80030D35C3BB162
:10370800504607F015FD354B83F800A00BF098FFE5
:103718002A68B9F8003052683248D25CFE2A01D1D2
:1037280000230BE0FF2A02D103F058F907E0D8F88C
:1037380000500A2111FB02523A60013303801B4DED
:103748002B785F0704D5284B4FF480521A8561E027
:103758003268D0075CBF43F001032B70184B1B780D
:1037680019075EBF2B7823F001032B70D30242BFE9
:103778002B7823F001032B701C4B1A88174B1AB1B6
:103788001B4A1268970702D41A4A1288A2B3022267
:103798001A702B7823F001032B7032E0B810002048
:1037A800AC260020E8180020F4180020CC260020C1
:1037B80060130020407E0500F81800200411002046
:1037C80000190020061900203C2300204C1A002074
:1037D80054260020441A0020401A0020A026002069
:1037E80010260020481A002000040048F60A00208D
:1037F800FC180020C42600202978CE0758BF0222D2
:103808001A7007F055FCB14B1B68C01A002801DB81
:103818000BF016FF09F03CFAAD4B03931E78002E0F
:1038280000F0AD80AB4F3B68002B00F08A8638680B
:1038380007F08DFC002800F08486A64BA64C18687B
:1038480007F082FC092801D03F2852D14FF0000927
:103858002668DFF8C4824D4636B1A048D8F8001073
:1038680032460EF077FF10B9C14605B945469C4B64
:1038780008F110089845EFD3EDB1D5F800C0D9F894
:10388800008023681CF803E018F80300704512D183
:103898005A1C924958B92D2B09D8DFF83CE2CEF8CA
:1038A80000204FF0200E01F803E0885403E001F8EF
:1038B80003E02260E5E723680BB14D4510D0894845
:1038C8000AF05AF84D4507D855F8100B0AF054F885
:1038D80009200AF049F8F5E783480AF04DF8002670
:1038E80023689E42A3D27D4B985D0AF03DF80136CD
:1038F800F6E72368002B40F00886042840F0448649
:10390800764804F0B7F800F01CBED8F80000DFF8DD
:10391800E89107F01CFC40B3D9F8000007F014FC4C
:10392800DAF8003093F848208346002A35D1242855
:103938006CD1012283F84820DAF80030DFF8B4911E
:1039480093F848B0BBF1060FDFD193F8490000F0B7
:10395800A9FE8046002800F081803B68987909F02C
:1039680054FF3B68002283F84820604B93F83730B7
:10397800002B40F0B8854C36982E00F0E2855C4B61
:10398800F21892F84A100129F5D15A4FF3583A60C3
:10399800594ABA4613609046B7E7012A04D14D2820
:1039A80014BF00220222C5E7022A04D13C2814BF12
:1039B80000220322BEE7032A0AD140284FF0000262
:1039C8009FBF1A71DA715871987198BF0422B1E7D4
:1039D800042A08D19A7983F8490080EA020B83F80F
:1039E80006B00522A6E7052AA6D159791A79914287
:1039F800997906D941409971511C1971134418726B
:103A08009AE781420CBF0622002293E72B783B4AB3
:103A1800590791D42328D9F8003012D10492039A77
:103A28003748012111702B490B6030490B6309F0AD
:103A3800A3FF2D4809F0A0FF049A137843F002036E
:103A48001370304B1B681B785B4501BF2E4B2F4A08
:103A58001A602F4B04BF2F4ADA606DE7D9F80020AF
:103A680092F849304E2B00F09D8476D8352B00F023
:103A78004B821BD8292B00F0448409D8252B00F051
:103A88001B84272B00F01F84232B40F0798500E24C
:103A98002D2B00F04784332B00F0B0842B2B40F003
:103AA8006F8509F095FE607100F018BD3E2B00F09F
:103AB800D68033D8392B00F013843C2B00F0D98002
:103AC800372B40F05D8500F0CDBC00BFA426002058
:103AD800CD2600202C2300200C1D0020DC1C0020FB
:103AE8000C3D01086C57010871570108B8100020F7
:103AF800C0230020A4190020A8190020CC260020EB
:103B0800A157010864240020FC9F0020EFBEADDE11
:103B180000ED00E00400FA057C3B0108432B00F0AF
:103B28007E8406D8412B40F02B854FF0000800F02A
:103B38006ABC442B00F0CE844C2B40F0218509F060
:103B480047FE84F8D60109F043FE84F8D70109F04E
:103B580049FEA4F8D80100F0C1BCD12B00F06B835A
:103B68001AD8CC2B00F00E8209D8C92B00F03C8360
:103B7800CA2B00F08D80C82B40F0028542E0CE2B86
:103B880000F02583C0F01A83CF2B00F04F82D02B92
:103B980000F0098300F0F4BCD62B00F0808207D82F
:103BA800D32B29D015D3D42B00F0848200F0E8BCA5
:103BB800EF2B44D005D8D82B40F0E2844FF0000911
:103BC800F9E0F22B00F0C482FA2B00F0098300F030
:103BD800D7BC2B7803F0040303F0FF08002B40F058
:103BE8007D8409F0F5FD022884F8E40640F2E182BC
:103BF800D94B83F8E486DCE209F0F4FDD74B9886CC
:103C080000F06CBC92F805804FEA5808B8F1120F22
:103C180003D90AF0F1FE00F061BC4FF00009C1457C
:103C280007D209F0DFFDCE4B23F8190009F101098D
:103C3800F5E7CA4B012283F8362000F04FBCDFF8C5
:103C48002483D8F8009009F0CDFDA9F85A00D8F8D7
:103C5800008009F0C7FDA8F8580000F03FBC09F043
:103C6800B7FD84F8E00109F0B3FD84F8DF0100F046
:103C780035BCDFF8F082D8F8009009F0A9FD89F882
:103C88000000D8F80030187807F09DFC00F026BC3A
:103C9800B44B1A681278022A4FF0000998466FD17F
:103CA800D8F800A009F094FD07EE900AF8EE677ABC
:103CB800B2EE048AC7EE887A0AEB890ACAED087A56
:103CC800D8F800A009F084FD07EE900A9FEDA67AC7
:103CD800F8EE677A0AEB890AC7EE877ACAED0B7A9B
:103CE800D8F800A009F074FD07EE900A9FED9F7ABE
:103CF800F8EE677A0AEB890AC7EE877A09F10109B3
:103D0800B9F1030FCAED0E7ACAD1B9F1070FD8F885
:103D180000A01CD109F05CFD07EE900AF8EE677A66
:103D2800C7EE887ACAED117AD8F800A009F050FDDC
:103D380007EE900AF8EE677AC7EE887ACAED127A2B
:103D4800D8F800A009F044FD8AF84C0012E009F008
:103D58003FFDCA448AF80100D8F800A009F038FDF0
:103D6800CA448AF80B00D8F800A009F031FDCA440B
:103D78008AF8150009F10109B9F10A0FC5D1ADE3B7
:103D8800D8F800A009F024FDCA448AF80100D8F840
:103D980000A009F01DFDCA448AF80B00D8F800A05D
:103DA80009F016FDCA4409F10109B9F10A0F8AF8A8
:103DB8001500E5D192E3DFF8AC819FED6C8AD8F865
:103DC80000A009F00FFD07EE900AF8EE677A0AEBFB
:103DD800890AC7EE887ACAED087AD8F800A009F0EF
:103DE80001FD07EE900AF8EE677A0AEB890AC7EE3A
:103DF800887ACAED0B7AD8F800A009F0F3FC07EE30
:103E0800900AF8EE677A0AEB890AC7EE887A09F110
:103E18000109B9F1030FCAED0E7ACCD1B9F1070F38
:103E2800D8F800A01CD109F0DDFC07EE900AF8EEE6
:103E3800677AC7EE887ACAED117AD8F800A009F037
:103E4800D1FC07EE900AF8EE677AC7EE887ACAEDD9
:103E5800127AD8F800A009F0C5FC8AF84C0012E0E4
:103E680009F0C0FCCA448AF80100D8F800A009F09B
:103E7800B9FCCA448AF80B00D8F800A009F0B2FCD3
:103E8800CA448AF8150009F10109B9F10A0FC5D128
:103E980024E309F09DFC132882463FF6BAAEDFF80A
:103EA800C490D9F800B009F093FC0023304A0C21E3
:103EB80001FB0322117A814222D10FFA8AF80BEB17
:103EC8008808137888F8793009F082FC88F87A0035
:103ED80009F07EFC88F87B0009F07AFC254B264A1D
:103EE8001A6088F87C00254BD9F80000186000217A
:103EF800793002F01DFD224B80F001001870EDE2D0
:103F080001331C2BD2D184E609F062FC0B288046D1
:103F18003FF67FAE134BD3F8009009F059FC032805
:103F28003FF677AE0BFB089B8BF8CE0009F050FCF0
:103F38008BF8C90009F04CFC8BF8CA0009F048FC62
:103F48008BF8CB0009F044FC8BF8CC0009F040FC5E
:103F58008BF8CD00C2E200BFD8110020B8100020B5
:103F6800481B00203C1100200000C84200007A4491
:103F7800D8390108300B002018130020340B00201A
:103F8800010000205379092B7FF643AE019BD3F83B
:103F9800008009F01DFC019B88F80000D3F8008020
:103FA80009F016FC88F8010009F012FC019B64284E
:103FB8001B68A8BF6420187109F00AFC019B6428DB
:103FC8001B68A8BF6420587109F002FC019BFF28F8
:103FD8001B68A8BFFF20987109F0FAFB019B6428B1
:103FE800D3F8008028BF642088F8070009F0F0FBA8
:103FF800019B88F80200D3F8008009F0E9FB019BD7
:1040080088F80300D3F8008009F0ECFBD9F80030F9
:10401800A8F80A005B790A2B40F26082D34BD3F8E8
:10402800008009F0D5FB88F8080057E209F0DAFBB0
:104038006FF4AF6283189BB2C62B98BFA4F89601A1
:1040480009F0D0FBA4F8400109F0CCFBA4F8420128
:1040580009F0C8FBA4F8440109F0C4FBA4F8D8018E
:1040680009F0B6FB84F8ED0109F0B2FB09F0B0FBEA
:1040780084F8EE0109F0ACFB84F8850109F0A8FB8F
:1040880084F8920109F0A4FBB94BD3F8008009F039
:10409800A9FB00EB80004000A8F8560020E109F0D9
:1040A800A1FBB44B23F8180008F10108B8F1080F78
:1040B800F5D113E253790F2B7FF4ABAD09F088FBF0
:1040C800072880463FF6A5AD029BD3F8009009F07B
:1040D80089FB0E2303FB08F8C144029BA9F81901C8
:1040E800D3F8009009F07EFBC144029BA9F81B019C
:1040F800D3F8009009F076FBC144029BA9F81D0192
:10410800D3F8009009F064FBC144029B89F81F01B1
:10411800D3F8009009F05CFBC144029B89F82001A8
:10412800D3F8009009F054FBC144029B89F821019F
:10413800D3F8009009F04CFBC144029B89F8220196
:10414800D3F8009009F058FBC844C8F82301C5E12A
:1041580009F03EFB0F2880463FF65BADC8EBC80868
:1041680009F036FB04EB080303F1D00883F8D0000C
:1041780009F02EFB88F8010009F02AFB88F80200F4
:1041880009F026FB88F8030009F022FB88F80400F0
:1041980009F01EFB88F8050009F01AFB88F80600EC
:1041A80007F084F99AE12B785B0700F1978109F011
:1041B8001BFE05F02DFB05F0E9FB8FE12B78580776
:1041C80000F18C816C4B4FF4C8721A8086E12B7811
:1041D800590700F18381694A137843F0040328E002
:1041E8002B785A07E5D5CBE109F0F2FA634B1A7838
:1041F80010B142F0020201E022F002021A7009F046
:10420800E7FA5F4BDFF89881187009F0F5FAC8F8FB
:10421800000009F0F1FAC8F8040009F0E3FA594B74
:10422800188009F0DFFA584B584A1880137843F081
:104238000203137052E109F0CBFA834609F0DCFA65
:10424800824609F0D9FA814609F0D6FA804609F083
:10425800C9FA09F0C7FA09F0BBFABBF1000F14D18B
:104268004B4B1020C3F800A0C3F8049005F07EFA69
:10427800424A137843F001031370B8F1000F00F0BD
:104288002D81444BC3F8008028E1BBF1100F40F0AA
:104298002581414BC3F800A0C3F80490B8F1000F82
:1042A80002D03C4BC3F800803B483C4B0222011D26
:1042B8001A7006F0CBF811E1A06009F09DFAA36826
:1042C8001843A0600AE109F08DFAA4F8580109F032
:1042D80089FAA4F85A0109F085FAA4F85C01FDE00E
:1042E80009F076FA84F87A0109F072FA84F87E0106
:1042F80009F06EFA84F87D0109F06AFA84F87F0102
:10430800ECE009F06FFAA4F8800109F06BFAA4F860
:10431800820109F05DFA84F8840109F063FAA4F8CF
:104328008601DBE009F054FA84F8900109F05AFAA2
:10433800A4F89A0109F056FAA4F8960109F052FA7D
:10434800A4F8980109F044FAD9F8003084F89101EA
:104358005B79082B40F2C28009F044FAA4F89C016A
:1043680009F040FAA4F89E01B8E000BF5C110020F3
:104378003C11002012230020F60A0020001900201A
:1043880006190020041900200219002062110020DB
:1043980064110020741100206C110020380B0020DB
:1043A8000819002092F805900323B9FBF3F9B9F135
:1043B800120F3FF62EACDFF8E8A2C84580F08E80D9
:1043C80009F006FA8AF8A00109F00CFA40F2ED2388
:1043D800984205DD40F6CA039842A8BF184601E096
:1043E80040F2EE20A0F2EE20192308F1010890FB1C
:1043F800F3F00AF1020A8AF89F01DEE709F0E8F90A
:1044080084F892016AE009F0E3F904EB080308F183
:104418000108B8F1080F83F88801F4D15EE009F0CB
:10442800D7F9C4F80880607109F0E6F9A368184361
:10443800A06009F0CDF984F8900109F0D3F9A4F847
:10444800580109F0CFF9A4F85A0109F0CBF9A4F8FA
:104458005C0109F0C7F9A4F8800109F0C3F9A4F8D0
:1044680082013BE053794FF00709B3FBF9F9C9EB37
:10447800C9029B1A13F0FF0F7FF4CBAB5FFA89F9DF
:1044880009F1FF395FFA89F9B9F1FF0F26D009F070
:104498009FF95FFA80FA4FFA8AF002F0CFF8804667
:1044A80000283FF4B6AB80F800A009F09BF9A8F803
:1044B800020009F08DF988F8040009F089F988F8F4
:1044C800050009F085F988F8070009F081F988F8EE
:1044D8000600D5E7604B012283F83720002009F059
:1044E800C3F9FFF73ABA5D4B985906F027FE18B999
:1044F800322006F004FEF6E706F098FF05F05EF9B4
:10450800574B584ADA60FFF736BA0C283ED00A28CB
:1045180040D1554D554809F02FFA284623210EF071
:1045280002F908B1401B20602368002B35D14E48A2
:104538002360002130220EF0C0F8039B1B78002B6B
:104548005ED14B4B1B689B060FD54A4B42491B68F3
:104558008A6B9A1A002A08DB474A1278042A82BF13
:1045680003F5123303F5F8738B63444B9B68002BF8
:104578006DD0434807B0BDEC028BBDE8F04F18473B
:104588000AF03AFAFFF7E9B90C2847D13D4809F093
:10459800F3F935E00D2835D1BBE75A1EA95C20296F
:1045A80001D11346C1E7304A23600021D154364B6C
:1045B800364DD3F80090D5F800A0DFF8AC8050460F
:1045C8000EF0BFF806463246404651460EF0C2F895
:1045D8002F4A28B918F806304B445B78580703D09F
:1045E80010359542E7D306E0954204D2701CEB687B
:1045F8004044984702E0274809F0BEF9002396E7AF
:10460800254807E07F280DD1013B174A234823603E
:104618000021D15409F0B0F9FFF709B97F2804D176
:10462800FFF705B92F2B3FF602A9A0F12002D2B25D
:104638005E2A3FF6FCA813B920283FF4F8A85A1CB4
:104648002260094AD05409F08FF9FFF7F0B807B093
:10465800BDEC028BBDE8F08FB8100020C02300200D
:1046680000ED00E00400FA05DC1C00209F62010850
:10467800FC180020AC260020061900200422002087
:10468800CE11002076570108FC0000207C3B010871
:104698000C3D010881570108715701089D57010811
:1046A800D81100202DE9F04764282DED028B04462F
:1046B80000F0BF8100F2D580322800F05F8667D80D
:1046C800222800F08C8423D8032800F07E8114D897
:1046D800012800F06E81022840F09186042009F03C
:1046E800C3F8432009F091F84C2009F08EF84620D1
:1046F80009F08BF84C2000F047BE042800F06F81C9
:10470800052840F07C861A2009F0AEF8002477E1ED
:10471800282800F0EC8515D8242800F0CF85262815
:1047280040F06D86CB4C062009F09EF8B4F858018D
:1047380009F09DF8B4F85A0109F099F8B4F85C0149
:1047480000F033BE2A2800F0E5852C2840F0578673
:10475800C04C0C2009F088F894F8900109F055F83D
:10476800B4F89A0109F083F8B4F8960109F07FF8D3
:10477800B4F8980109F07BF894F8910109F045F82C
:10478800B4F89C0109F073F8B4F89E0100F00DBE6E
:104798003D2800F0E68224D8382800F0958512D804
:1047A800342800F03E84362840F02986AA4BA94CCC
:1047B80093F8C100C0EBC000C0B209F055F804F18D
:1047C800180500F000BE3A2800F099823B2840F016
:1047D8001686012009F048F89F4B5B6C187800F0AA
:1047E800D3BD452800F0F88527D8402800F0CF85AC
:1047F800422840F00486974C102009F035F860797B
:1048080009F003F8A06809F03BF894F8900108F063
:10481800FCFFB4F8580109F02AF8B4F85A0109F075
:1048280026F8B4F85C0109F022F8B4F8800109F020
:104838001EF8B4F8820100F0B8BD4B2800F070856E
:104848004D2800F07C85462840F0D9850D2009F0D8
:104858000BF8002008F0D9FF002009F011F800F04B
:10486800C6BD722800F05B8455D86A2800F09B8486
:104878002FD8672800F0B8811CD8652800F002817D
:10488800662840F0BC85754C122008F0EDFF2088A2
:1048980008F0EDFF608808F0EAFFA0886E4C08F089
:1048A800E6FFA08D08F0E3FFE08D08F0E0FF208E22
:1048B80000F0FABC682800F00482692840F09F855F
:1048C800674D2878400000F0FE0008F0CDFF002476
:1048D80003E26D2800F00C8213D86B2800F0838463
:1048E8006C2840F08C855F4C062008F0BDFF2088BE
:1048F80008F0BDFF608808F0BAFF5B4B188800F02D
:1049080054BD6F2800F05282C0F0FD81702800F07D
:10491800778200F074BD782800F0728119D8752864
:1049280000F0518309D8732800F03284742840F0CD
:1049380066854FF000080126A0E3762800F064841D
:10494800772840F05C85444D287C08F08DFF0024D2
:10495800DDE3A42800F07D8414D87B2800F0D982F8
:10496800A02840F04C850C2008F07EFF3F4B1868CB
:1049780008F086FF3E4B186808F082FF3D4B186828
:1049880000F039BDF12800F07681FE2800F0888417
:10499800F02840F03485304C042008F065FF636C43
:1049A800B3F85A0008F063FF636CB3F8580000F0DE
:1049B800FCBC032008F058FF002008F026FF204622
:1049C80008F023FF0D2000F0DFBC08F04DFF0120A8
:1049D80008F01BFF0A2008F018FF00F038BC06207A
:1049E80008F042FF412008F010FF462008F00DFFB4
:1049F800462008F00AFF332008F007FF00F05CBCEF
:104A08001D4B185D013408F000FF0B2CF8D1002471
:104A18001A4B185D013408F0F8FE082CF8D1002470
:104A2800174B185D013408F0F0FE072CF8D100F0A0
:104A3800E4BC072008F018FFE72008F0E6FE054B65
:104A4800587908F0E2FE002008F0DFFE042000F0AC
:104A5800D2BC00BFD8110020F8100020C6110020D9
:104A68005C24002026260020CC110020ACF7FF1F74
:104A7800B0F7FF1FB4F7FF1FCE530108DA53010840
:104A8800AF530108BC4C0B2008F0EEFE208808F05C
:104A9800EEFE6268B94B9A420CBF2089608980B2E9
:104AA80008F0E5FEB64B1B68C3F3C000C3F38002F1
:104AB800800040EA4200C3F340021043C3F34012AF
:104AC80040EAC20003F01003184308F0D0FEAD4BD3
:104AD8001A88E368247C02F0080103F4475949EA7C
:104AE800010903F4804149EA010903F4004149EA54
:104AF800010903F4803149EA010903F4003149EA64
:104B0800010903F4802149EA010903F4002149EA73
:104B1800010903F4801149EA010903F0007349EA25
:104B28000303DFF8849299F8009012F0010FC9F39B
:104B3800800914BF4FF002084FF0000843EA090348
:104B480012F0020F43EA080314BF4FF0040C4FF0B1
:104B5800000C12F0040F43EA0C0C14BF4FF0100EB7
:104B68004FF0000E12F0400F14BF202700274CEA28
:104B78000E0E12F0100F14BF4FF4007600264EEA06
:104B8800070712F0200F14BF4FF4806500253E433D
:104B980012F4807F14BF4FF400600020354312F4F4
:104BA800007F14BF4FF400110021284312F4806FD6
:104BB80041EA000114BF4FF080630023002019432D
:104BC8000346A3420AD2704A9D5C012202FA05F507
:104BD8000D421CBF9A4010430133F2E708F050FE23
:104BE8006A4B93F8E406CFE3102008F03DFE00245A
:104BF800674B185D013408F008FE102CF8D1FCE36F
:104C0800702008F031FE00265B4D0E246B6C744357
:104C180023440136B3F8190108F029FE6B6C2344CC
:104C2800B3F81B0108F023FE6B6C2344B3F81D0195
:104C380008F01DFE6B6C234493F81F0108F0E5FD96
:104C48006B6C234493F8200108F0DFFD6B6C234460
:104C580093F8210108F0D9FD6B6C234493F82201E5
:104C680008F0D3FD6B6C1C44D4F8230108F008FE4F
:104C7800082EC9D1C1E37020444C08F0F5FD04F1B9
:104C8800700594F8D00008F0C0FD94F8D10008F041
:104C9800BCFD94F8D20008F0B8FD94F8D30008F0F1
:104CA800B4FD94F8D40008F0B0FD94F8D50008F0ED
:104CB800ACFD073494F8CF0008F0A7FDAC42E0D172
:104CC8009BE3102008F0D0FD0024324B185D01341E
:104CD80008F09BFD102CF8D18FE32B789C4280F0D4
:104CE8008C832D4B33F8140008F0C1FD0134F4E730
:104CF800062008F0B9FD002008F0C2FDDCE204201F
:104D080008F0B2FD76E3072008F0AEFD234B1888C3
:104D1800FF28A8BFFF20C0B208F077FD204B186815
:104D28004FF6FF74A042A8BF204620EAE07080B288
:104D380008F09DFD104BB3F8600008F098FD134B88
:104D480093F88521174B18683AB10A235843A042B3
:104D5800A8BF204620EAE07001E000F30F0080B20F
:104D680023E30A4C022008F07FFD94F8E00108F0E4
:104D78004CFD94F8DF0107E3F810002000540040D0
:104D8800FC180020C419002009110020D8110020A7
:104D98002A11002040110020481B0020EC18002098
:104DA800F8180020F4180020CC260020C24C0B2054
:104DB80008F05AFD636E187808F027FD636E58787E
:104DC80008F023FD002625466B6EBB4C33440136A4
:104DD800187908F01AFD032EF6D1636ED87908F019
:104DE80014FD636E987808F010FD636ED87808F0AB
:104DF8000CFD636E588908F03AFD636E187AC3E2B9
:104E0800AD4C1E2008F030FD636C1B78022B4FF070
:104E180000056BD1636C03EB850393ED080AB2EED2
:104E2800048A20EE080A0DF057FE80F30800C0B28D
:104E380008F0EBFC636CDFEDA17A03EB850393EDDF
:104E48000B0A20EE270A0DF047FE80F30800C0B2D7
:104E580008F0DBFC636CDFED9A7A03EB850393EDD6
:104E68000E0A20EE270A0DF037FE80F30800C0B2C4
:104E7800013508F0CAFC032DCCD1072D636C23D172
:104E880093ED110A20EE080A0DF026FE80F30800C3
:104E9800C0B208F0BAFC636C93ED120A20EE080A5F
:104EA8000DF01AFE80F30800C0B208F0AEFC636C87
:104EB80093F84C3000EE103AB8EE400A0DF00CFEB4
:104EC80080F30800C0B20BE02B44587808F09DFC32
:104ED800636C2B44D87A08F098FC636C2B44587D9B
:104EE800013508F092FC0A2DC7D186E2636C2B4489
:104EF800587808F08AFC636C2B44D87A08F085FC53
:104F0800636C2B440135587D08F07FFC0A2DEDD1E8
:104F180073E23C2008F0A8FC0024674D9FED688AE6
:104F28006B6C03EB840393ED080A20EE080A0DF07E
:104F3800D3FD80B208F09BFC6B6C03EB840393ED0C
:104F48000B0A20EE080A0DF0C7FD80B208F08FFCAE
:104F58006B6C03EB840393ED0E0A20EE080A0DF048
:104F6800BBFD013480B208F082FC032CD5D1072C9C
:104F78006B6C16D193ED110A20EE080A0DF0ACFD0A
:104F880080B208F074FC6B6C93ED120A20EE080AEC
:104F98000DF0A2FD80B208F06AFC6B6C93F84C002F
:104FA8000BE02344587808F062FC6B6C2344D87AF1
:104FB80008F05DFC6B6C2344587D013408F057FC05
:104FC8000A2CD4D119E22F2008F04EFC3D4C14F8DD
:104FD800010F002800F0118208F017FCF7E75020B5
:104FE80008F042FC0025344B5C6C374B04EB85041D
:104FF8000C2194F8792001FB0233013593F838002D
:1050080008F003FC94F87A0008F0FFFB94F87B00A2
:1050180008F0FBFB94F87C0008F0F7FB142DE2D1B4
:10502800EBE1482008F020FC0025234B5C6C0623AC
:1050380003FB0544013594F8CE0008F0E6FB94F82C
:10504800C90008F0E2FB94F8CA0008F0DEFB94F807
:10505800CB0008F0DAFB94F8CC0008F0D6FB94F803
:10506800CD0008F0D2FB0C2DDFD1C6E1002E00F0F8
:10507800C4815FFA88F008F0F7FB002600270E4B82
:105088001A7C9742F2DA11330024FA5C0E4D0C2395
:1050980005F130016343595C914207D12B44586BA9
:1050A8000DF04FFB82462EB9B1460FE001341C2C9F
:1050B800ECD118E0804416E0F81000200000C84247
:1050C80000007A44A7390108A8390108D1450ADA4D
:1050D8000C2303FB04535B6B13F8090008F095FBE2
:1050E80009F10109F2E70137C9E701311C290DD09F
:1050F800C4480C2200F1300702FB01F3DA5DB2422A
:10510800F3D1034493F8380008F07FFB01342B7C7B
:105118009C4280F07281BC4B0021E65CE8E7BB4C06
:10512800162008F0A1FBB4F8960108F0A0FBB4F82B
:10513800400108F09CFBB4F8420108F098FBB4F871
:10514800440108F094FBB4F8D80108F090FB94F8F7
:10515800ED0108F05AFB002008F057FB94F8EE0127
:1051680008F053FB94F8850108F04FFB94F892017E
:1051780008F04BFB002008F048FBA54B5B6C0A20AD
:10518800B3F9563093FBF0F080B208F070FB9FE063
:10519800082008F069FB0124E0B2013408F035FB6F
:1051A800092CF9D129E1102008F05EFB994B9A4CA3
:1051B800187800F0020008F028FB984B187808F0DF
:1051C80024FB206808F05CFB606808F059FB944BEE
:1051D800188808F04CFB934B188808F048FB8C4B58
:1051E800B3F86800E1E0052008F03EFB8E4B188814
:1051F80008F03DFB8D4B188808F039FB844B93F879
:105208006A0000F00100BFE008F0E2FA0746122049
:1052180008F02AFB7E4C17B9E66E256F05E0102FC3
:1052280013BF0025666FA56F2E46384608F0EDFAC5
:10523800304608F025FB284608F022FBE06F08F00E
:105248001FFB002008F013FB002008F010FB0020D3
:105258009AE06F4D95F8800080000130C0B208F0E8
:1052680003FB95F8800008F0D0FA00242E4696F843
:1052780080309C4280F0C1806D4D285D08F0C5FAF1
:1052880005F11003185D08F0C0FA05F12003303568
:10529800185D08F0BAFA285D08F0B7FA0134E6E7B5
:1052A800082008F0E1FA002008F0E1FA002008F0F0
:1052B800DEFA002008F0DBFA002076E0042008F08F
:1052C800D3FA524B986896E0042008F0CDFA4F4C78
:1052D80094F87A0108F099FA94F87E0108F095FAA2
:1052E80094F87D0108F091FA94F87F014CE0474C5E
:1052F800072008F0B9FAB4F8800108F0B8FAB4F851
:10530800820108F0B4FA94F8840108F07EFAB4F83F
:1053180086014AE0012008F0A7FA3C4B587933E0AF
:105328003A4C042008F0A0FA94F8D60108F06DFA77
:1053380094F8D70108F069FAB4F8D80135E03D4C83
:105348003D4D207800EB4000C0B208F08DFA0026F1
:1053580023789E4205F102054FD215F8020C08F099
:1053680054FA15F8010C00EB800000EB800000F205
:10537800EE2080B208F07BFA0136E9E7012008F058
:1053880073FA224B93F8920108F03FFA35E00820AF
:1053980008F06AFA00241D4B2344013493F888016D
:1053A80008F033FA082CF6D127E008F060FA24E078
:1053B80092F90C10994245D092F918209A4241D09E
:1053C8000834AC4219D01D4A94F8F40192F900103F
:1053D80043B29942ECD135E0132008F045FA002495
:1053E800174B185D013408F010FA0B2CF8D1002087
:1053F80008F046FA002008F043FA012039E00020BE
:1054080037E000BFA839010809110020D811002091
:10541800F8100020001900200819002006190020A3
:1054280004190020021900207A1900207C19002094
:10543800791100205C2400207813002068240020C3
:10544800CE53010808F0E1F9B4F8F60108F00FFAB4
:1054580094F8F80108F0D9F994F8F90108F0D5F9A9
:1054680094F8FB0108F0D1F994F8FA0108F0CDF9A5
:10547800A6E7BDEC028BBDE8F08700BF2DE9F04739
:10548800D44CD54E237886B00746002B00F0FE8119
:1054980032686368D31A7C2B40F2F881237A626001
:1054A80001332372002505F12400DFF82883C0B2F8
:1054B80007F0DEFB08F10A039FEDC87A33F91530CF
:1054C80007EE903AFAEECC7A013567EE877AFDEE70
:1054D800E77ACDED037ABDF90C0007F0B7FB032D91
:1054E800E1D1302007F0C4FB002007F0AFFB07F044
:1054F800B7FB98F8085015F0030520D1D8F8042018
:1055080041F288339A420BD9102007F0B1FB2846A4
:1055180007F09CFB212007F0ABFB284607F096FB21
:10552800142007F0A5FBB4F9100007F08FFB1C202E
:1055380007F09EFB002007F089FB07F091FB237A18
:10554800DFF890825B0740F07E81022007F090FB35
:105558000A23B8F9120090FBF3F007F077FB032059
:10556800B8F91A50DFF8909207F082FB9C4B1B7831
:1055780013F0040F4FF0050A95FBFAF5ADB20DD004
:1055880008F5D270394601F0E4F928B9D9F80030A5
:1055980013F0100F18BF002528B205E0D8F82C37F3
:1055A8009889B0FBFAF000B207F050FBD9F8003048
:1055B8009F0740F18A80DFF84492B4F8327799F86F
:1055C8000030B4F83027834D3F014FF06408BFB274
:1055D80008FB02325B00B2FBF3F347EA0327BFB2D2
:1055E800C3F303231F43062007F042FB38B207F03A
:1055F8002DFBB4F8323799F8001001339BB293FBB6
:10560800F1F201FB1233A4F83237D4F834379B7B1C
:10561800012B05D1392007F02BFBB5F930071AE02B
:10562800B5F830576E233A205D43152707F020FB65
:1056380095FBF7F5AFB2B7FBF8F528B207F006FB14
:1056480008FB15753B2007F013FBA8B2451D0A207F
:1056580095FBF0F000B207F0F9FA282007F008FBF4
:10566800D4F838375B4D0A2093FBF0F000B207F00E
:10567800EDFA042007F0FCFAD4F82C37D5F83C07EB
:105688009A894FF6FF739842A8BF1846C2B10028FE
:10569800ACBF131A134607EE903A9FED527AF8EE14
:1056A800E77A67EE877A07EE102AB8EEC77AC7EE70
:1056B800877AFDEEE77A17EE900A6428A8BF64207F
:1056C80020EAE07000B207F0C1FAD4F84037414F41
:1056D8009D0640F1AD8097F8443798071DD51120F5
:1056E80007F0C6FAB7F846073F4B4FF4F36568432F
:1056F80090FBF3F000B207F0A9FA192007F0B8FA06
:10570800B7F846074543642095FBF0F595FBF0F3A1
:1057180000FB135000B207F099FA94F84437B4F834
:10572800485713F0020F08BF0025012007F0A0FA20
:1057380028B207F08BFA092007F09AFA002007F040
:1057480085FA2A4B94F84A571A88B2F5967F0AD9EF
:10575800204B1B7A03F00F03072B04D842F20F7576
:10576800954228BF1546052007F082FAD4F8343749
:105778005B7B0BB928B21CE0A5F1200307EE903A39
:105788009FED1B7AF8EEE77AF6EE006AC7EE877AA5
:10579800BEEE007AF5EEC07AF1EE10FA58BFB0EE20
:1057A800667A77EE877AFDEEE77ACDED037ABDF972
:1057B8000C0007F04BFA94F84427064B910703D4E2
:1057C80093F84B27012A1DD1012384F84B37094848
:1057D80035E000BFBC1100205426002000007A44A8
:1057E800CC2600200000C842A0860100EE00002060
:1057F8006666E63F0819002030260020EC000020ED
:105808008096184BD3F834375FED036A93ED017A2D
:10581800D3ED027A27EE267A67EEA67ABDEEC77A2E
:10582800FDEEE77A8DED047ACDED057A04A806E061
:10583800B74A92E8030004AB83E80300184603F074
:10584800C3FB07F00DFA237A282B1FD1B14B002296
:105858001A723C2733684FF47A70B3FBF0F81720BC
:1058680007F006FAB8FBF7F5B5FBF7F007FB1050A1
:10587800000200B207F0EAF9182007F0F9F907FB6F
:10588800158000B207F0E2F907F0EAF994F8543706
:10589800A04D002B00F05D8105F00AFCD5F85837C3
:1058A8009D4AC31A9342074640F2C680002385F8F2
:1058B8005E3785F86037B5F83037DAB21B0A85F8F5
:1058C8007A2785F87B3785F8702785F87137D5F8FA
:1058D800882733689A1AD5F88C37D97B4FF47A73AE
:1058E8004B439A420ED38D4B1B68C5F8883795F801
:1058F8009037013B012B9FBF102385F85E370223A9
:1059080085F860370A20D4F8382792FBF0F284F83B
:105918007827121284F8792794F84427D4F83C376A
:1059280093FBF0F384F87C371B1284F87D379207D9
:1059380094F84A37774984F8AB3703D42D2381F894
:10594800AC3777E0042BD4F84C97D4F85067DFF8DD
:10595800DC81734A8CBF3323322381F8AC374FF094
:10596800060C704B99FBF3F096FBF3F308FB0091E0
:1059780008FB036803EB83030CFB01F103EB8303D0
:1059880091FBF2FE642502FB1E119B0091FBF5F1D1
:1059980084F89D1709120CFB08FC84F89E179CFBE1
:1059A800F2F143FA81F39BB202FB11C292FBF5F2CA
:1059B80084F8A227121284F8A03784F8A3271B0AB8
:1059C800B4F8462784F8A1372423534393FBF5F50D
:1059D800B4F8BE3784F8A43700EB80001B0A00EB4C
:1059E8008000800084F8A5370A22B4F84837B3FB52
:1059F800F2F303F5FA739BB240FA8EF080B284F8A2
:105A0800A6371B0A4FEAD97984F89B07F60F000AD4
:105A180084F8985784F8A737C5F30725B4F8C03732
:105A280084F89A9784F89C0784F89F6784F89957B4
:105A380084F8AD37C4F8587794F8C287354DB8F173
:105A4800000F0DD1D5F8C80705F081FB012807D94B
:105A58000228354E00F0538203F0A8FA0123337070
:105A6800D4F8CC272B4D002A73D095F8C2673EB1E5
:105A7800D5F8D43740F6B731FB1A8B4219D868E00D
:105A88000123D5F8C80785F8C23700F07CFCD5F8A3
:105A9800D83793F9000002238DE8480008213246E0
:105AA8004FF4964300F08AFC85F8DC67C5F8C80710
:105AB8004DE095F8D067CEB9D5F8C807C5F8CC67DA
:105AC80085F8C26700F05FFCD5F8D83793F9000075
:105AD80001238DE84800082132464FF4964300F030
:105AE8006DFCC5F8C80703F061FA30E0013EF6B274
:105AF80085F8D06795F8DC1795F8DD37C6B94A1CE4
:105B0800013385F8DC2785F8DD37D5F8C8071CE0B0
:105B1800343B0108BC1100203F0D0300542600202F
:105B280040420F008096980002000020806967FFBD
:105B380012F8016BC5F8CC27701885F8DC0701331B
:105B4800D5F8C80785F8DD37314605F003FBC4F8FA
:105B5800D47794F8DE379D4DF3B1D5F8E037DBB153
:105B6800D5F8E437C3B1C5F8E8371B68984AC5F8D3
:105B7800EC37D5F8F0371344187AFEF793FDD5F8CB
:105B8800E837987907F041FED5F8F0370133092B4B
:105B980088BF0023C5F8F0378E4D94F8F4272E6897
:105BA8008A4B002A00F0E681D3F8F827002A00F093
:105BB800E18193F8FC37013B012B00F2DB81D4F83B
:105BC800F807824F05F0C3FAE0B1D7F8F80705F0F7
:105BD800BBFA97F8FD37D5F800907E2B80460ED19A
:105BE80002231B2887F8FC3709D1D7F8F80705F0F6
:105BF800AEFA20B90123C7F8009887F8043884F86A
:105C0800FD87DCE7D7F800282B689B1A41F6583245
:105C180093421ED9032387F8FC37ABE16E4A32F86A
:105C2800130010B903464FF403600133B0F5C06F99
:105C3800DBB271D01ED9B0F5006F77D033D9B0F58B
:105C4800036F40D184F80538D4F840375F4F9A067F
:105C580040D494F8041894F80538002900F04C81D1
:105C68002A68921B012AD9D984F80538002384F8B8
:105C780004387FE1B0F5007F44D008D8B0F5807FC4
:105C880000F08780B0F5887F00F08380E5E7B0F505
:105C9800806F00F0A580B0F5826F00F0EA80B0F563
:105CA800047FDAD123E0B0F5E26F00F08280B0F52E
:105CB800E46F00F08380B0F5E06FCED184F805384A
:105CC800B4F90A107EE0B0F5046F6BD0B0F5026F3E
:105CD800C3D1FAE097F844379B07BAD5B7F8461707
:105CE80024234B431233642193FBF1F1FEE084F843
:105CF80005383A4B354F1B689907AAD5B7F830379E
:105D08000A21F2E084F80538344B304F1B681A0535
:105D18009FD5D7F83817E9E084F805382F4B2B4F73
:105D28001B681B0595D5D7F83C17DFE0D4F840175A
:105D3800264A84F8053888068BD592F844178907CF
:105D480087D5DB0712D5D2F8503783EAE371002BE9
:105D5800A1EBE37101EB51014FF01902B1FBF2F134
:105D6800ACBF41F0004141F040410FE0D2F84C3760
:105D780083EAE371A1EBE371002B01EB51014FF0D2
:105D88001902B1FBF2F1B8BF41F080414FF4006055
:105D98008AE084F80538D4F840375F077FF559AFB3
:105DA80000215FE0B4F9101084F8053864235943E2
:105DB8007AE084F80538B4F90C1003E0B4F90E1051
:105DC80084F805382C2391FBF3F16DE0BC11002019
:105DD800343B010854260020BE5801083026002014
:105DE80084F8053894F80638644A0133DBB2032B8B
:105DF80088BF012382F8063894F8061842F2107317
:105E080059435F4B1B78D80748BF01319A0748BFF1
:105E180002315F07B4F8083848BF0431D80748BFD3
:105E28000A319A0748BF14311F0648BF2831D805E0
:105E380048BF28315A0748BF64311F0748BFC831D7
:105E4800980548BF01F5C8719A0648BF01F57A71EF
:105E5800DF0648BF01F5FA61580648BF01F57A61C7
:105E68004FF4806003F06EF8444B002283F8042856
:105E7800EFE6D4F84017DFF8048184F8053811F00C
:105E8800200717D098F8442712F0020F14BF4FF4D8
:105E98007A71002112F0010F14BF4FF4FA63002346
:105EA8000B4494F84A17194403F04CF8002384F87B
:105EB8000438CEE6334B1B6819067FF5CAAE39465F
:105EC80003F040F888F80478C3E684F80538D4F875
:105ED80040372A4F9A067FF5BCAE97F844379B07A0
:105EE8007FF5B7AEB7F848376421594303F02AF86D
:105EF800002387F80438ACE684F805383AE03378AC
:105F080023B1C5F8C47786F80080A9E5D5F8C43769
:105F1800FB1AB3F57A6FFFF4A3AD0123D5F8C807D0
:105F2800337005F011F90646D5F8C80705F00CF9E5
:105F380076067FF495AD8A2802D08E280DD08FE59D
:105F4800D5F8403799067FF58BAD95F8C237002B09
:105F58007FF486AD05F2917306E095F8C237002B01
:105F68007FF47EAD05F25C73C5F8CC372D2385F838
:105F7800D03775E506B0BDE8F08700BFBC1100203A
:105F8800CC26002030260020F8B504460E461746D9
:105F98000025204620210CF0C6FB0446D0B1013470
:105FA80020460CF025FCB0F5617F05DB40F6340394
:105FB8009842A8BF184601E04FF46170A0F56170DF
:105FC800192390FBF3F00DB9307000E070703B7846
:105FD80001333B700DB90125DBE72046F8BD7FB5DD
:105FE80004780646E4B9364B1B6803EB8403192191
:105FF80093F87B0093F87C6093F8792093F87A30D3
:106008004FF4617511FB005011FB0651009001918E
:106018002C482146013403F0B0FA142CE3D14CE0AB
:106028000CF0E6FB1328054641DC254B701C1C6868
:10603800202100238DF80F300CF075FB1E35064625
:1060480070B1013630460CF0D3FB1A289FBF04EB21
:10605800850358709DF80F30013398BF8DF80F30C5
:10606800304620210CF05FFB064670B10136304601
:106078000CF0BEFB0D289FBF04EB850398709DF8BC
:106088000F30013398BF8DF80F3004EB850430468C
:10609800E11C0DF10F02FFF777FF9DF80F30042B7D
:1060A8000BD0601C002104220CF007FB05E0064819
:1060B80006490022132303F060FA04B070BD00BF44
:1060C8003C110020DE580108F35801081259010854
:1060D800014807F051BC00BF18590108F0B5047811
:1060E80087B006461CBB524B1968062303FB0411F4
:1060F800192091F8CA5091F8CB7091F8CE2091F8F8
:10610800C9304FF4617610FB056510FB07600095F8
:10611800019091F8CC000290C83146484979039122
:106128002146013403F029FA0C2CDCD17DE00CF077
:106138005FFB0B28044672DC3D4B701C1D68202158
:1061480000238DF817300CF0EEFA064680B10136C0
:1061580030460CF04DFB03289FBF062303FB045376
:1061680083F8CE009DF817309CBF01338DF81730A7
:10617800304620210CF0D7FA074680B1013738465F
:106188000CF036FB0D289FBF062303FB045383F84E
:10619800C9009DF817309CBF01338DF817300626CB
:1061A8006643A9193846CA310DF11702FFF7ECFE0C
:1061B80020210CF0B8FA074670B1013738460CF0C8
:1061C80017FB14289FBF9DF817307619013386F8FE
:1061D800CC0098BF8DF81730384620210CF0A3FA70
:1061E80078B101300CF004FB0D289FBF062303FB98
:1061F800045383F8CD009DF817309CBF01338DF808
:1062080017309DF81730062B0FD0062202FB0450DA
:106218000021C9300CF051FAFFF75AFF05E0064893
:10622800064900220B2303F0A8F907B0F0BD00BF10
:106238003C11002026590108F35801081259010899
:106248002DE9F347047807464CB9204601A908F020
:106258007DFB0134FFF7F4FF122CF6D178E00CF047
:10626800C7FAC5B2112D6DD8781C20210CF05BFA45
:10627800394C3A4F05F1D006034614F8168030B968
:10628800A8F10202D2F1000848EB020843E000F14D
:10629800010A597838460CF046FA60B1032D8CBFD4
:1062A80003230023C01B3B4453FA80F090F804906A
:1062B800B9F1030F02D1FFF70BFF49E0A9F102037F
:1062C800D3F1000850464FF0200148EB03080CF0CA
:1062D8002AFAD8B1B8F1000FEDD001300CF088FAE5
:1062E80040F2ED2380B2984205DD40F6CA03984299
:1062F800A8BF184601E040F2EE2004EB4603A0F2E6
:10630800EE20192290FBF2F0587002E0B8F1000F6D
:10631800D1D104F8169014F81630FA5CB8F1000FD1
:106328000BD00D4B0E4803EB46062946737840F216
:10633800EE24192505FB034308E02946094803F024
:106348001CF905E0084809490022112303F015F952
:1063580002B0BDE8F08700BFD8110020503B01080B
:106368004659010858590108F3580108A56401085D
:1063780010B50446204604F0E1FE18B90A2004F0DE
:10638800BEFEF7E710BD0C4B5A6882421A4607D08A
:106398001B69834206D0D36983420BD1022302E0F2
:1063A800002300E001230021C1620C2000FB03232D
:1063B80019725960704700BF682400202DE9F04F1A
:1063C80006468B4890F9004087B0B44289469DF84C
:1063D800445011461A469DF840300AD090F90C40B6
:1063E800B44209D090F91840B4420CD14FF00208D9
:1063F80004E04FF0000801E04FF001080C2404FB12
:106408000800047A0CB10020EEE0012E00F0DA80DA
:10641800142E05D0002E40F0E68000957548D3E094
:10642800DFF814A2DAF8183043F00103CAF818307C
:10643800DAF814304FF0904543F40033CAF81430BA
:10644800012703224FF4805B04A94FF090408DF898
:1064580015200392CDF810B08DF814708DF81670D1
:106468008DF8174001F0CAF8A5F828B0C82004F044
:1064780046FEC5F818B0DAF81430039A43F400332E
:10648800CAF8143028464FF4C0534FF0020B04A941
:1064980004938DF815208DF814B08DF816408DF8FA
:1064A800174001F0ABF86B6A23F470436B626B6AB8
:1064B80043F460436B626B6A23F470236B626B6A0C
:1064C80043F460236B624C4B4C4D4FF480221A60AE
:1064D80002F18042A2F53F321223AB64082385F80B
:1064E8004D30136885F84E7023F480231360536889
:1064F80023F48023536095F84C3003F1804303F56F
:1065080082331A6842F480221A60AA6C3C4B22F04B
:106518001F0002F01F02C15807FA02F221EA020224
:10652800C250AA6C374922F01F0002F01F0250F82F
:1065380001E007FA02F22EEA02024250AA6C22F0A7
:106548001F0102F01F02C85807FA02F20243CA509C
:106558002D4B2E4A1C60DAF81C3043F40003CAF8AD
:106568001C302B4B04A8DA608DF810608DF811B040
:106578008DF812408DF8137008F052FC2A238DF81C
:1065880010309DF813308DF811708DF812401BB142
:1065980004A808F045FC04E01E4B4FF48062C3F8E1
:1065A80084201D4A1D4B136002221A721C4A1D4B7F
:1065B80013601D4A1D491B68116098471C4B2B60CE
:1065C8000E4806E01B480095FCF752FA00283FF4F5
:1065D8001AAF074B06710C2202FB083888F808909E
:1065E800C8F8040000E0204607B0BDE8F08F00BFFF
:1065F800682400200038014014040140C819002014
:10660800080401400C040140D80042420005FA0584
:1066180000ED00E000E100E05C23002060230020A2
:1066280034220020BC00002030220020040000207A
:106638005C3B010800440040001002400C4B1B6802
:1066480093F90220824209D093F90A20824207D0A6
:1066580093F91220824208D1022002E0002000E0D3
:10666800012003EBC000023070470020704700BFD4
:1066780064240020F0B5027887B0AAB94C4C04F124
:1066880018064C4B94F9F41193F900208A4272D001
:1066980093F90C208A426ED093F918308B426AD055
:1066A8000834B442EDD180E0002204920592451CE2
:1066B8000CF09EF8C4B260B2FFF7C0FF074618B1ED
:1066C8008DF81040012400E00446284620210CF0F3
:1066D8002AF8054638B1013528460CF089F8013406
:1066E800ADF81200E4B20026284620210CF01BF871
:1066F800B0B3451C28460CF07BF800222E4951F80F
:10670800223083425FFA82FE04D00132082AF5D192
:10671800002300E0734651F82320824220D1022E44
:106728000FD0032E12D05A1E012ED2B204D0042A42
:1067380013D88DF814300EE0042A0ED88DF81530D1
:1067480009E0052B09D88DF8173004E09A1E052AB0
:1067580003D88DF816300134E4B20136042EC3D1C3
:10676800052C03D807B0BDE8F040B1E404AB03CB77
:106778003860796019E094F8F9010F4B94F8F851F2
:1067880053F82000B4F8F621009094F8FB0153F870
:106798002000019094F8FA0153F82000029053F871
:1067A8002530064802F0E9FE7AE707B0F0BD00BFE1
:1067B800D811002068240020B85201086759010840
:1067C80038B1438811EA030003D08B420CBF012083
:1067D8000220704730B50B4B0B491C6891F85020CC
:1067E800022A0BD8134604EBC303551CEAB29D8852
:1067F8002842F5D081F85020981C30BD81F85020EF
:10680800002030BD64240020C8190020024B00225B
:1068180083F85020DEE700BFC81900202DE9F047B3
:10682800877890F803C0214DBBB2C7F1640E03EB23
:1068380083065C42C3F178005FFA8EFE7600CCF1E5
:106848006408A4B280B2A3B20FFA83F9B9F1000FB9
:1068580005DC002B14BFBA464FF0010A00E0F246EF
:1068680013FB03F303FB0CF21AFB0AF392FBF3F39B
:10687800434403FB09F30A2293FBF2F333449BB22C
:1068880025F8023FB1F800904A880A34C9EB020A99
:10689800A4B21AB202FB0AF24FF47A73844292FB52
:1068A800F3F34B442B80CED1BDE8F087181A0020B3
:1068B80010B544780078002202FB02F3193B6343C9
:1068C80003F6C413534340F6C411434393FBF1F357
:1068D800034921F812300132072AEDD110BD00BF5B
:1068E800321A00200430114B33F91000B0F5617FE3
:1068F80010B506DB40F6330398420246A8BF1A4695
:1069080001E04FF461720C78192340F2833013FBD5
:106918000404944207DA497813FB01039342B4BF95
:106928000020012010BD002010BD00BF481B002022
:1069380010B500F1500302788A4203D18478C278F6
:10694800944204D304309842F5D1002010BD0120B0
:1069580010BD0B4B1B6813F4805F0A4BB3F906306C
:1069680005D0C089421A934207DD084400E0008A36
:106978008342B4BF0020012070470120704700BF48
:1069880030260020481B00201FB5094B1B681B033D
:106998000AD58DF8040001230D2001A98DED030A05
:1069A8008DF8053001F068FF05B05DF804FB00BF05
:1069B800302600201FB5084B1B681B0309D58DF82E
:1069C8000400029100230D2001A98DF8053001F083
:1069D80053FF05B05DF804FB3026002010B50020F9
:1069E80004F0A6FB064B00241C7008F029FE054B9A
:1069F80083F87840DC67A3F88040C3F8844010BD72
:106A0800A0260020C819002010B510B9BDE8104014
:106A1800E4E700230C225A430B4C1119125D824201
:106A280003D00133102BF5D110BD084BD3F88400E7
:106A380018B14A784078824205D20022C3F88410FF
:106A4800A3F88020DA6710BD0C440108C81900209B
:106A580010B540001428A8BF14200023074A0221BB
:106A680099540B4499181424834201F8014CF5DB1E
:106A7800FF21D1540F20BDE81040C5E73C2300207A
:106A88002DE9F84307460B24013C36D01D4B4FF443
:106A980080529A617D1C32264FF00508DFF8649019
:106AA800B9F814309BB283F48053A9F8143001204C
:106AB80004F03EFB304604F022FBB9F814309BB2D8
:106AC80083F480530020A9F8143004F031FB3046D9
:106AD80004F015FBB8F1000F08D0B8F10108DDD1BA
:106AE8004FF4FA7004F00BFBFA26D7E7013DD5D135
:106AF8004FF47A7004F003FBC6E7034B034ADA60ED
:106B0800BDE8F8830004004800ED00E00400FA0541
:106B180010B5214A18B9136802221A8210BD1F48FD
:106B2800146800230380217811F07F0102460DD1FB
:106B3800637A990644BF0221017013F0400F03786D
:106B480014BF43F0010323F0010315E0012921D00C
:106B580002291ED1637913F0800F03F00F034FEA67
:106B6800830303F1804303F5B8431B6806D003F0A1
:106B78003003102B07D10123137004E003F44053B2
:106B8800B3F5805FF6E7064B1B681B699847034817
:106B980010BD184610BD00BF5C230020501A00200D
:106BA8003022002010B5064C18B9236801221A8239
:106BB80010BD044B1B689B68984720680C3010BDBB
:106BC8005C2300203022002010B5064C18B9236839
:106BD80001221A8210BD044B1B681B689847206865
:106BE8000A3010BD5C2300203022002003788B423D
:106BF80083BF034B03EB410148880020704700BF67
:106C0800501A002070B500221346244914180C4469
:106C1800A47E83EA0423082413F4004F4FEA4303B5
:106C280018BF83F4815304F1FF3418BF83F00103C4
:106C380014F0FF049BB2EFD10132192AE5D100F11B
:106C4800190200F11A050A440D44967EAA7E02EB49
:106C5800062292B29A421FD1104B93F83B50E2B2EF
:106C6800AA4216D2431C03EB4203DBB2CA18013313
:106C78000B44927E9B7E03EB02239BB24FF4AF62E0
:106C880053431B13064A03F5487322F814300134A2
:106C9800E5E7012381F83C3070BD00BF501A0020A1
:106CA800521A002003788B420BD9074B1A78074BEE
:106CB80089001944086C02B1400800F5777080B269
:106CC80070470020704700BF60240020501A002041
:106CD80007299DBF034B03EB8101B1F87000002029
:106CE800704700BF501A0020034B03EB4101B1F875
:106CF8009000C008704700BF501A00200A4BDFED13
:106D08000B7A03EB810191ED2C7AB8EE477AF6EE17
:106D1800046AE7EE267A82B0FCEEE77ACDED017AD6
:106D2800BDF8040002B07047501A002000005C440F
:106D3800024B03EB4101B1F8F8007047501A0020EC
:106D4800024B03EB4101B1F81C017047501A0020B7
:106D580070B5334C054604F0ABF9D4F83431C4F8B7
:106D68003401C31AB3F5FA5FC4F8383182BF00237F
:106D780084F83C3184F83D3194F83C312BB9A12D8D
:106D880002BF274A012182F83D1194F83D11244A97
:106D980029B1D118EDB201338D7682F83C3194F8DF
:106DA8003C5194F83E31AB4239D11D4B93F83F31F9
:106DB800052B02D0062B03D02CE00020FFF722FF82
:106DC800E37E1E2B26D100200246C1B26B1E9942DB
:106DD80019DA21448B7E0821DBB283EA0206F60722
:106DE80044BF83F01803C3F3460301F1FF3154BFD6
:106DF8005B0843F0800311F0FF01C2F34702ECD1B6
:106E080001301A46E1E723449B7E9A4202D10320CF
:106E1800FFF7F8FE002384F83D3184F83C3170BD5B
:106E2800501A002010B5044604F042F90F4BD3F86D
:106E38004021C3F84001821A41F288318A42C3F8DE
:106E4800442184BF002283F8482193F84821074948
:106E580013440F2AE4B218BF013283F8494112BF24
:106E680081F84821012381F8593110BD501A0020BA
:106E780010B5044604F01CF90F4BD3F85C21C3F895
:106E88005C01821A41F288318A42C3F8602184BFCA
:106E9800002283F8642193F8642107491344142AD3
:106EA80018BF013283F8654112BF81F864210123BC
:106EB80081F87A3110BD00BF501A002038B5044659
:106EC80004F0F6F8274A2749D2F87C31C2F87C0149
:106ED800C31AB3F57A6F84BF002382F8803192F821
:106EE800803133B9A82C3BD181F88131A1F88231A6
:106EF80006E0022B02D181F8844101E0242B02D85C
:106F0800D11881F8854192F88411164D0133023168
:106F1800DBB249008B4282F8803118DAB5F8823149
:106F2800E0B283EA0020082310F4004F4FEA400043
:106F380018BF80F4815003F1FF3318BF80F00100BF
:106F480013F0FF0380B2EFD1A2F8820138BD0131FE
:106F58008B4201BF002385F88031012385F88131F8
:106F680038BD00BF501A002010B5044604F0A0F840
:106F7800104AD2F8AC3140F6AC51C31A8B42C4BFA8
:106F8800002382F8B03192F8B031D11881F8B141BC
:106F980023B90F2C0DD10749C1F8AC010133DBB27D
:106FA800192B044982F8B0310CBF0123002381F862
:106FB800CA3110BD501A00202DE9F843324F3D6800
:106FC8002A8A2E7AB2B9042E14D1304C304823784C
:106FD800012B0BD12F4B19682F4B89B20B445B0047
:106FE80019681A6030230380227048E01023038058
:106FF800072644E0AC8AAB69A24294BF0426022665
:10700800944228BF14461FFA84F840469847214AFC
:1070180013689BB203F1005303F540535B0004F17E
:10702800010E1B689BB203F1005303F540534FEA6E
:107038006E0E5B000021714500F1020009D010F8C6
:10704800019C10F802CC4CEA092C23F821C001312C
:10705800F1E71268104B92B213445B001A681C6087
:107068002B8AC8EB03032B826B8A9844084BA5F83C
:10707800128030221A80094B4FF440521A803B6824
:107088001E72BDE8F88300BF5C230020CE260020D6
:107098002A220020505C00400230002028220020D4
:1070A8000E4B0F4A1B689BB203EBC00002443E29FB
:1070B8004FEA420209D94B09C80604BF03F1FF335E
:1070C8009BB29B0243F4004304E04B08C90748BF46
:1070D80001339B0211681360704700BF505C004089
:1070E8000630002010B5454B1A68107810F07F0064
:1070F80004D1537A23F02003537210BD02287AD1A9
:107108005388002B78D11379002B75D1537923F04C
:107118008000840004F1804101F5B84113F0800F2C
:10712800096814BF01F0300101F44051032862D806
:10713800002960D0927A002A5DD004F1804404F5D9
:10714800B8441906226825D502F03002102A4CD11D
:1071580003F07F039B0003F1804303F5B8431A68EB
:10716800510641BF196840F60F720A4042F40042C6
:1071780044BF42F0C0021A601A6822F4E04222F0CA
:10718800400292B282F0300242F4004242F08002A1
:107198001A602AE002F44052B2F5805F25D128B97E
:1071A800174B93F82C10FFF77BFF11E09B0003F1BE
:1071B800804303F5B8431A68520441BF196840F682
:1071C8000F720A4042F4404244BF42F080021A6003
:1071D800236823F4804323F070039BB283F4405365
:1071E80043F4004343F080032360064B1B685B694C
:1071F8009847002010BD022010BD00BF5C2300206E
:10720800BC0000203022002002684FF6FE731340B5
:1072180003600023036043608360C360284B984287
:1072280001D1284A27E0284B984201D1254A2AE073
:10723800264B984201D1234A2DE0254B984201D193
:10724800204A30E0234B984201D11E4A33E0224BBA
:10725800984204D11B4A536843F470032EE01F4B35
:10726800984204D1174A536843F0706326E01C4BD8
:10727800984204D11B4A536843F00F031EE01A4B8F
:10728800984204D1174A536843F0F00316E0174BAD
:10729800984204D1134A536843F470630EE0144BC8
:1072A800984204D10F4A536843F4704306E0114BE7
:1072B800984204D10B4A536843F4702353607047D3
:1072C80008000240000002401C000240300002405A
:1072D80044000240580002406C0002408000024016
:1072E80008040240000402401C040240300402402A
:1072F8004404024058040240084BDA68D10709D414
:10730800DA68D20608D4DB6813F0040F14BF032030
:107318000420704701207047022070470020024077
:10732800994A536803F00C03042B2DE9F04105D06A
:10733800082B06D095490160B3B916E0934B03605A
:1073480012E053685468C3F38343991CE30349BFAD
:10735800D36A8F4B8D4C03F00F0344BF0133B4FB4A
:10736800F3F34B43036000E000235168894FC1F3F6
:1073780003117D5C0168EDB221FA05F4446056689A
:10738800C6F30226BE5D24FA06FEC0F808E0566879
:10739800C6F3C226BE5DF6B2F440C460D2F82C80B3
:1073A800C8F3041808F00F0C07EB4C0C18F0100F7A
:1073B800BCF810C01FFA8CFC07D0BCF1000F04D039
:1073C800B3FBFCFCC0F810C000E00161D2F82CC08F
:1073D800CCF3442C0CF00F0807EB48071CF0100FF7
:1073E8003F8ABFB204D01FB1B3FBF7F7476100E093
:1073F8004161176BFF065ABF644F87618161176B44
:10740800BF065ABF614FC761C161176B7F065ABF7C
:107418005E4F07620162176BFF0506D5994204D1DA
:10742800AE4202D14F00476200E04462176BFF048E
:1074380006D5994204D1AE4202D14F00876200E0DE
:107448008462176BBF0506D5994204D1AE4202D1BA
:107458004F00C76200E0C462176B7F0506D59942EA
:1074680004D1AE4202D14F00476400E04464176B78
:107478003F0506D5994204D1AE4202D14F00876438
:1074880000E08464176BBF0406D5994204D1AE426C
:1074980002D14B00C36400E08464156B3A4BAD071E
:1074A80001D1046315E01C6B04F00304012C01D125
:1074B80001630EE01C6B04F00304022C02D14FF4AC
:1074C800004305E01B6B03F00303032B01D12F4B93
:1074D8000363146B2C4B14F4403F02D1C0F834E022
:1074E80018E01C6B04F44034B4F5803F01D14163CB
:1074F80010E01C6B04F44034B4F5003F02D14FF4A3
:10750800004306E01B6B03F44033B3F5403F01D161
:107518001E4B4363146B1C4B14F4402F02D1C0F86C
:1075280038E018E01C6B04F44024B4F5802F01D136
:10753800816310E01C6B04F44024B4F5002F02D1E1
:107548004FF4004306E01B6B03F44023B3F5402FD0
:1075580001D10E4B8363146B0B4B14F4401F02D103
:10756800C0F83CE020E01C6B04F44014B4F5801F24
:1075780001D1C16318E01C6B04F44014B4F5001F7A
:107588000AD14FF400430EE00010024000127A00C6
:1075980000093D00280000201B6B03F44013B3F5DD
:1075A800401F01D1134BC363126B134B12F4400FEE
:1075B80003D1C0F840E0BDE8F0811A6B02F4400244
:1075C800B2F5800F02D10164BDE8F0811A6B02F4B4
:1075D8004002B2F5000F02D14FF4004306E01B6BE6
:1075E80003F44003B3F5400F01D1024B0364BDE837
:1075F800F08100BF00127A0000100240F0B50023AD
:107608000E681C460125A54005EA060EAE452BD19D
:107618000F797A1E012A15D8856803229A4025EA2F
:10762800020282604D7982689D4015438560828898
:1076380092B222EA0E0282808A798588A2402A4381
:1076480092B28280032205689A40D24315400560B1
:1076580005689F402F430760C7681740CA7902FA38
:1076680003F547EA0502C2600134102C03F1020356
:10767800C8D1F0BD38B52DED048B4A4C0368C4F869
:10768800CC318388A4F8D031013A0D46072A42D874
:10769800DFE802F0040A101822292F35B4F8CC319B
:1076A8000B80B4F8CE3113E0B4F8CE310B80B4F8C7
:1076B800CC3105E0B4F8CC315B420B80B4F8CE3164
:1076C8005B4205E0B4F8CE315B420B80B4F8CC31B4
:1076D8006B80B4F8D0311DE0B4F8CC315B420B803C
:1076E800B4F8CE3112E0B4F8CE310B80B4F8CC3116
:1076F8000CE0B4F8CC310B80B4F8CE3105E0B4F826
:10770800CE315B420B80B4F8CC315B426B80B4F86D
:10771800D0315B42AB80244B93F83030002B3ED104
:10772800B5F9003094ED780AD4ED757A09EE103A7F
:10773800B5F9023008EE103AB8EEC88AB5F9043047
:10774800B8EEC99A28EE000A08EE903AA7EE890A20
:10775800F8EEE88AD4ED7B7AA7EEA80A0BF0BCF91C
:1077680094ED790AD4ED767A288028EE000AA7EEFF
:10777800890AD4ED7C7AA7EEA80A0BF0ADF994ED4E
:107788007A0AD4ED777A688028EE000AA7EE890A8B
:10779800D4ED7D7AA7EEA80A0BF09EF9A880BDEC7F
:1077A800048B38BD501A002028000020094B1A68A5
:1077B800137844F6FB7103EB431300FB0313507873
:1077C800C0EB0030B3FBF0F39078B3FBF0F080B27D
:1077D800704700BFE81800200748002108B50A22B2
:1077E800A0F8F81100F5007003F0B7FC80B2FFF7BD
:1077F800DDFF024B188008BD501A0020EC1800204D
:1078080038B500240B4D6059254406F0B5F8696871
:1078180011B1094801F0B1FEA96811B1074801F09A
:10782800ACFE0748103406F0A7F8B4F5C87FE9D1D4
:1078380038BD00BF7C3B0108585A01085E5A010850
:107848009F620108F0B585B004460AF07AFF08285F
:1078580026D1621EE01D1F4912F8013F096819442C
:10786800497801F00301022908BF203B82421370C6
:10787800F1D1254604F1080715F8016B1648314681
:107888000AF051FF20B1284631460AF04CFF10B1EA
:10789800FEF71EFC1CE0BD42EED1204607F038F88A
:1078A8000E4806F069F800230D4A1A4404A992F814
:1078B80088210A440849595C02F80C1C0133082B3A
:1078C800F2D1002307488DF80C3001A901F055FECC
:1078D80005B0F0BDFC000020C56D0108645A010820
:1078E800D8110020E16101081E4B1F4C1D6820685B
:1078F80080B5FEF73DFD2846FEF73AFD2068417940
:107908008B0704D4036841F002015B699847174B61
:107918004FF480529A61206803F019FCA0B1134E0D
:107928004FF480533385104B186803F00DFC07465D
:1079380002F037FA08B105F0ABFA2846394603F0E9
:1079480009FC4FF48053B361284603F000FC00287B
:10795800E1D02846266803F0F7FB0146304603F0DD
:10796800F9FBD8E72C230020D81C0020000400488D
:107978002DE9F04705460AF0E4FE314E0446D6F8F4
:10798800088090B92F4805F0F7FF2F4B53F82410C3
:1079980049B10123A34013EA080F02D02B4801F094
:1079A800ECFD0134F1E72A4822E02846294922461D
:1079B8000AF0D0FE58B92848284C05F0DDFF54F8E5
:1079C800041F0029EFD0214801F0D7FDF7E72B78F5
:1079D8002D2B03BF013504F1FF344FF0010A4FF09E
:1079E800000A4FF00009184B53F8297027B91C48B2
:1079F800BDE8F04705F0C0BF2846394622460AF0E0
:107A0800A9FEC8B9012000FA09F0830501D5154877
:107A1800EEE7BAF1000F03D001F0C8FE124803E008
:107A280040EA0800B060114805F0A6FF3946104842
:107A3800BDE8F04701F0A1BD09F10109D3E700BF96
:107A4800D81100206A5A01080C3D0108745A01082F
:107A58009F620108785A01087D5A0108083D01080B
:107A6800895A0108985A0108A65A0108AF5A01080C
:107A7800E061010810B5084805F07EFF074B0024B7
:107A88001C715C63064B1C7003F0F4FC06F058F99B
:107A9800044B1C6010BD00BFB75A0108D81C002059
:107AA800CD2600202C23002070B5064600240B4B61
:107AB800E518AA8816420AD0E158094801F05DFD88
:107AC8002846002105F0E5FE064805F055FF143468
:107AD80040F644439C42EAD170BD00BFAC45010862
:107AE800E35A01089F620108F0B504788BB0054697
:107AF8000CB1002436E04B4B19680E2303FB04112C
:107B080001F58C70B1F91D51B1F91921B1F91B3189
:107B1800009591F82051019591F82151029590F91D
:107B28000700039001F590713F4891F90210049104
:107B38002146013401F021FD082CDCD170E02D2B09
:107B480014D1072C1BDC28460AF052FE0AAB661C2F
:107B580003EB440424F8100C15F8013F303B092BC3
:107B6800FAD934462B78002BE9D104E0A3F130028E
:107B7800092A09D8E5E7082CBDF8182009D00BB068
:107B8800BDE8F040FEF7A4BA202BF8D1013526460F
:107B9800E7E7072AF3D8BDF81A00224BA0F2EE2136
:107BA80089B240F2DC55A9421B68E8D8BDF81C1020
:107BB800A1F2EE24A4B2AC42E1D8BDF81E6004B232
:107BC80037B2A742DBDB0DB2AF42D8DCA542D6DB29
:107BD800BDF8247007F16404A4B2C82CCFD8BDF84E
:107BE80026E00FFA8EF4112CC9DCBDF82050B42D14
:107BF800C5D8BDF82240B42CC1D812B24FF00E0C33
:107C08000CFB0233A3F81901A3F81B11A3F81D619B
:107C180083F8205183F8214183F81F7183F822E10A
:107C28000BB0F0BD3C110020ED5A01082DE9F041E0
:107C3800047806467CB9334DB5F8C421B5F8C63189
:107C480031482146013401F098FC042C05F1040563
:107C5800F2D1BDE8F0812D490AF038FDB0B9294BC1
:107C68004FF47A714FF4FA62A3F8C411A3F8C6214D
:107C7800A3F8C811A3F8CA21A3F8CC11A3F8CE2100
:107C8800A3F8D011A3F8D221BDE8F08130460AF05C
:107C9800AFFD032805462DD8304620210AF043FDC4
:107CA800044630B1013420460AF0A2FD01260746F9
:107CB80000E00646204620210AF035FD18B9BDE847
:107CC800F041FEF705BA01300AF092FD012EF6D117
:107CD800A7F2EE2240F2DC539A42F0D8A0F2EE224C
:107CE8009A42ECD8074B703503EB85039F80D88008
:107CF800BDE8F0810648074900220323BDE8F041AA
:107D080001F03BBCD81100200D5B0108205B010885
:107D1800F3580108A56401082DE9F0412DED048B05
:107D2800AB498AB004460AF0D1FCAA49002820468B
:107D38000CBF012607260AF0C9FCA74900282046DF
:107D480008BF02260AF0C2FC002808BF0426F10773
:107D580040F1E380A148A24C05F00EFE002005F09A
:107D680013FCA04805F008FE9F4805F005FE63795E
:107D78009E4A9F48013B254652F8231001F0FDFB1F
:107D88009C4801F0FAFB4FF00008274695ED048A5D
:107D9800B5EE408AF1EE10FA04D1974801F0EDFBF8
:107DA800002570E09548D5ED059A95ED069AD5ED34
:107DB800078A414601F0E1FBB5EEC08AF1EE10FA00
:107DC80002D5202005F0D0FDB0EE480A06A801F043
:107DD80069FA01468A4801F0D0FBF5EEC09AF1EE47
:107DE80010FA02D5202005F0BFFDB0EE690A06A8FA
:107DF80001F058FA0146824801F0BFFBB5EEC09A7F
:107E0800F1EE10FA02D5202005F0AEFDB0EE490AD9
:107E180006A801F047FA0146794801F0AEFBF5EEF5
:107E2800C08AF1EE10FA02D5202005F09DFDB0EED3
:107E3800680A06A801F036FA08F1010801467148F7
:107E480001F09BFBB8F10C0F05F110059ED1A4E7DA
:107E580049B294F8D02094F8D130009194F8D31016
:107E6800019194F9D410029194F9D510039194F8E2
:107E7800D610049164482946013501F07EFB102D87
:107E880004F1070403D094F8D2100029E0D15F4828
:107E98005F4C05F071FDD7F8088054F8041F19B13C
:107EA8005C4801F06AFBF8E70D465B4B53F8254048
:107EB80054B10123AB4013EA080F03D057482146B9
:107EC80001F05BFB0135F0E7554805F055FD21460B
:107ED8007B180AAA93F888311344524A8A5C03F83B
:107EE800102C01310829F3D1002306A94E488DF83A
:107EF800203001F042FB4D4805F03EFD4C48FEF7AE
:107F0800B9FB4C4801F039FB4020FFF7CDFD4A484A
:107F180005F032FD4648FEF793F9B20739D54748D0
:107F280005F02AFD464805F027FD414805F06CFBA1
:107F3800444805F021FD3E48FEF751F8424805F057
:107F48001BFD3B48FEF7CAF8404801F016FB3848CD
:107F5800FFF76CFE3E4805F00FFD3548FFF7C4FDFE
:107F680000270E257D4300243A4A926B2A440123B8
:107F7800D2F80A20A34013421ED101340E2CF3D1AB
:107F88000137082FEDD12B4801F0F7FA8020FFF7D1
:107F98008BFD730716D5304805F0EEFC2F4805F029
:107FA800EBFC234805F00AFB224801F0E6FA4FF4FF
:107FB8008070FFF779FD05E039462246284801F030
:107FC800DCFADAE70AB0BDEC048BBDE8F08100BF4B
:107FD800265B0108865F01082D5B0108335B0108F9
:107FE800D8110020415B0108535B0108F0510108DA
:107FF8005F5B01086A5B0108775B0108845B010825
:10800800615A0108E16101089C5B01088C5B010869
:10801800083D0108BB5B01080C3D0108C95B01086C
:10802800D65B0108C56D0108E25B0108EB5B01083E
:10803800A05701089F620108FA5B0108075C010864
:108048001A5C0108285C0108325C0108415C0108DF
:108058004F5C0108D81C00205B5C01086C5C0108BF
:108068007E5C0108F0B504468FB020460AF069FB33
:10807800C5B225BBAF48B04C05F07EFC94F8D210D1
:1080880009B9AE4854E049B294F8D02094F8D130F8
:10809800009194F8D310019194F9D410029194F9B5
:1080A800D510039194F8D6100491A54829460135B6
:1080B80001F063FA102D04F10704DFD1E1E720464F
:1080C800A04905220AF046FB0546B8B929469E484C
:1080D80070220AF0F2FA9D4B196828460E2303FB1A
:1080E800001301300022082883F8232183F8242173
:1080F80083F8252183F82621F0D119E120469449F7
:1081080004220AF027FB05462046002D4AD12021EB
:108118000AF009FB002800F00B81461C30460AF0E3
:1081280010FB2C4607468B4B53F824502DB98A4830
:108138000FB0BDE8F04001F020BA30462946FAB247
:108148000AF008FB01340028EDD17B4A02F17001E6
:108158001646002382F8D63082F8D23082F8D13021
:1081680082F8D03007328A42F3D17C4901EBC4014E
:1081780091F8E821934210DAD1F8EC71C3EBC3020D
:10818800B0183A4400F1D0011768C0F8D070908850
:10819800888092798A710133E7E72946704801F0AF
:1081A800ECF996E06F4907220AF0D4FA0546204612
:1081B800002D4AD120210AF0B6FA06460AF0C1FA83
:1081C800C4B274BB684801F0D8F921466748013445
:1081D80001F0D3F90E2CF8D1584801F0CEF900245B
:1081E8006348214601F0C9F90025584A61481168D9
:1081F8000E2202FB04120123D2F823215E49AB4070
:1082080013425E4B05F1010508BF194601F0B5F9A7
:108218000E2DEAD14948013401F0AFF9082CDFD11D
:1082280086E0304656490AF0E7FA2C46002852D034
:10823800022C55D00AF0DCFA06AB514943F8240069
:1082480000200AF0D9FA0134F0E74D490AF0D4FACF
:10825800002460B1082C3ED00AF0CAFA06AB48499F
:1082680043F8240000200AF0C7FA0134F1E7082C8B
:1082780031D1069B0F2B2ED8DDF81CE0BEF1070F7D
:1082880029D8089F0D2F26D8099E06F16402C82A0E
:1082980021D80A9DFF2D1ED80B9864281BD80C994D
:1082A800642918D8884216DA0D9C032C13D8224A60
:1082B800C3EBC303134483F8D0E083F8D17083F889
:1082C800D26083F8D35083F8D40083F8D51083F8AC
:1082D800D6402C4CC9E60FB0BDE8F040FDF7F8BE1B
:1082E800069B072B20D807990D291DD80278722ADA
:1082F8000DD06E2A18D1154A12680E2000FB0323F0
:1083080001228A40D3F8231121EA020209E00F4A28
:1083180012680E2000FB032301228A40D3F82311A0
:108328000A43C3F8232101E0FDF7D2FE0D4C9CE679
:108338000FB0F0BD9D5C0108D81100209F620108B4
:10834800C85C0108205B0108A81200203C1100202D
:10835800E45C0108F0510108895A01087C3B0108D6
:10836800E95C0108955C0108625A0108F55C01089E
:10837800F9610108FA5C0108D865010892660108EC
:10838800FE5C0108A05701082DE9FF410478054665
:10839800002C39D17348744D05F0EEFAD5ED047A06
:1083A800F5EE407AF1EE10FA00F0D98021466F48D8
:1083B80001F0E3F895ED040A684600F073FF014602
:1083C8006B4801F0DAF895ED050A684600F06AFF97
:1083D8000146674801F0D1F895ED060A684600F0B5
:1083E80061FF0146624801F0C8F895ED070A684642
:1083F80000F058FF013401465E4801F0BEF80C2C2D
:1084080005F11005CAD1AAE05B4905220AF0A2F9D4
:1084180040B9554B03F1C002002143F8101F9342A5
:10842800FAD19CE02846554904220AF093F90446FB
:108438002846002C40D120210AF075F9002800F0C8
:108448008E80451C28460AF07CF907464C4B53F8A9
:1084580024601EB94B4805F08FFA80E02846314663
:10846800FAB20AF077F901340028EFD13E4B03F154
:10847800C0029E46002143F8101F9342FAD1424B96
:1084880003EBC4029846D2F804C0BCF1000F04D133
:1084980031463E4801F071F857E0002718F83430AB
:1084A8009F42F5DA3B010EEB030563440FCB103511
:1084B80085E80F000137F1E70AF09AF90B2806461C
:1084C80047DC284620210AF02EF9054650B101352F
:1084D800284600F05DFE244B03EB061383ED040AE7
:1084E800012400E00446284620210AF01CF905462C
:1084F80048B10135284600F04BFE1B4B03EB061331
:1085080083ED050A0134284620210AF00CF90546B6
:1085180048B10135284600F03BFE134B03EB061328
:1085280083ED060A0134284620210AF0FCF810B928
:10853800FDF7CEFD13E0013000F02AFE0A4B032CB4
:1085480003EB061686ED070AF2D11148FFF71CFF68
:1085580005E01048104901220C2301F00EF804B080
:10856800BDE8F081005D0108D81100201B5D0108FD
:10857800215D0108E1610108205B0108E45C010854
:10858800F0510108895A010888590108E95C010875
:10859800A0570108F358010812590108284B294A25
:1085A8001B68126810B51A60274A1168596051682B
:1085B8009268DA60254A9960116819615168926871
:1085C8009A61234A59611168D961516892685A625F
:1085D800204A196211881985518859859188D2884D
:1085E800DA851D4A99851188198651885986928895
:1085F8009A861A4A1188D986518819871946928805
:1086080021F83A2F164A10780022824206DA154CD1
:1086180034F8124021F8024F0132F6E7124A128864
:10862800A3F86420114A1288A3F86620104A128819
:10863800A3F868200F4A5289A3F85E2010BD00BF36
:10864800A8240020AC260020C81F0020D41F00202A
:10865800E01F0020D011002024110020C6110020A6
:108668001720002040110020481C0020DC100020AA
:10867800581100202A1100202DE9F8430E4B93E8E9
:10868800800305460E460024B44213DA7B1933F9F9
:10869800140008EB050333F9142009EB050333F93B
:1086A80014301344022293FBF2F3C01A05F0F9FECA
:1086B8000134E9E7BDE8F883A824002070B5472015
:1086C80005F03EFE174B1B681B0307D5164B174AD0
:1086D8005B6810681B68C01A05F0D4FE144E154C70
:1086E800154D307805F0CEFE23682868C01A05F0CD
:1086F800D8FE63686868C01A05F0D3FE0F4B188867
:1087080005F0C0FE0E4B188805F0BCFE0D4B18880E
:1087180005F0B8FE337823742B68A3606B68E360B8
:1087280070BD00BFFC250020A8240020AC26002036
:10873800061900209424002008190020041900209C
:1087480002190020601100207FB5264C264E274DC7
:108758002749284A284B20B128480088B0F5805F6F
:1087680031D23088ADF8040028781E4D91F82010D9
:1087780012788DF806008DF807108DF808201B7800
:108788008DF8093001A82946062209F07BFF30B38D
:108798000198BDF808302860AB80532005F0D0FD63
:1087A800208805F06FFEA07805F06CFEE378019351
:1087B8002379029301A86379039305F0C9FD0F4B50
:1087C80000221A800BE03088208091F82010287849
:1087D80012781B78A070E17022716371DDE704B034
:1087E80070BD00BF141D0020C4190020001900200E
:1087F8007C2600207B0A0020E00A00201C2600209E
:10880800A0F17D03012B70B504460D460A4E05D82C
:1088180030687D2102F09EFC84F0200430682146F7
:1088280002F098FC35B12B881C4404EB142404F0A6
:10883800FF042C8070BD00BFB41900200A4A1388B9
:1088480001331380094A136801331360084A1388F7
:1088580001339BB2202B01BF00231380054A1388E4
:1088680008BF0133138070471C260020042600200F
:10887800082600200A26002038B53A4B1B78083B0A
:10888800012B05460C466BD8452005F059FD2846B6
:1088980005F056FD0C2D23D004D80A2D0AD014D883
:1088A80035B138BD0E2D4BD02ED3FF2D50D038BD4D
:1088B800206849E0207805F043FD62796378002A52
:1088C80014BF80200020184300E0207805F038FD10
:1088D800A07805F035FDE07805F032FD20793BE021
:1088E800B4F9000005F0C4FDA07805F029FDE07892
:1088F80005F026FDB4F9040005F0BAFDB4F9060048
:10890800BDE8384005F0B4BD637820788BB180F0BD
:10891800800005F015FDA468E0B205F011FDC4F370
:10892800072005F00DFDC4F3074005F009FD200EF2
:1089380012E005F005FD6068BDE8384005F0B1BDFE
:10894800206805F09FFD6068BDE8384005F09ABDD5
:10895800054805F0D3FC0020BDE8384005F0F0BC20
:1089680038BD00BF8E240020F76001082DE9F04FC4
:10897800B54BB64F1A888BB00193002A40F0968009
:10898800B7F80A07B24D42F20103C11A48424841FA
:10899800FFF7DAFEFFF702FE2C68492005F0D0FC4D
:1089A800AC4B2646186805F06DFD56F8040B05F02B
:1089B80069FD304605F018FF04F1100005F014FFBA
:1089C80004F11C094FF01008A34E0123326803FA82
:1089D80008F3134203D0D9F8000005F062FD08F14E
:1089E8000108B8F1130F09F10409EDD104F12800C9
:1089F80005F0EAFEB7F84031B4F92E00C01A05F0C8
:108A080041FD3368DA0408D5944BB4F864001B8838
:108A1800181AC0F30D0005F035FD33689B0403D523
:108A2800B4F8660005F02EFD3368180403D5B4F8D1
:108A3800680005F027FD04F13000A04605F0C4FEEB
:108A480004F1360005F0C0FEB7F8403138F93C0FA4
:108A5800C01A05F017FD0127814B1B789F4208DAE1
:108A680038F9020FB4F93C30C01A05F01AFD013785
:108A7800F2E73368990505D5B4F95E00A0F2DC5039
:108A880005F00FFD2A6877486A60AA60121A9110EB
:108A9800754A4A43531C032293FBF2F202EB42024B
:108AA8009A1A6C2303FB02032B60ABE16F4B704AED
:108AB8001B6811688B4206D00AA9002041F8203DA6
:108AC8001360FFF7D9FE019B97F80A171B8897F8E0
:108AD8000B070B44013BB3FBF0F200FB12338B4254
:108AE80080F05B815A4D0120FFF72EFEFFF756FDFF
:108AF80050202F686E6805F023FCAA682B68106860
:108B08001B686A6803441068A3EB400005F0C9FCC1
:108B180072687B689B1A0293B268BB689B1A0393BE
:108B2800F268FB6802A89B1A049305F05DFE32699F
:108B38003B699B1A029372697B699B1A0393BB6911
:108B4800B26902A89B1A049305F002FC07F11C0BFA
:108B580006F11C081024404901220B68A2401A4261
:108B68008A4606D0DBF80000D8F80030C01A05F0B5
:108B780098FC0134132C0BF1040B08F10408EAD11A
:108B880007F1260006F12601002331F9024F30F9DA
:108B9800022F121B02AC44F823200133042BF4D11A
:108BA80003214FF000094FEA89035FFA83F902AB0A
:108BB80053F821206AB102F108000F2802D849F0C1
:108BC800010906E08032FF2A94BF49F0020949F002
:108BD800030911F1FF31E6D2484605F0B1FB002444
:108BE8000DF1080BA04609F00302022A16D0032A49
:108BF8001DD0012A4FD1B8F1000F05D1DBF8004094
:108C08002401E4B2904646E0DBF8000000F00F00D3
:108C1800204305F095FB4FF000083CE0B8F1000F49
:108C28000CD0DBF80000C0F3031020432DE0B8F1AE
:108C3800000F1FD19BF8010005F082FB9BF8000094
:108C480005F07EFB27E000BF08260020D811002091
:108C5800A824002004260020FC250020F825002058
:108C680017200020B424002013DA4B6810260020B7
:108C78000C260020DBF80000C0F30330204305F089
:108C88005FFBDBF80000C0F3071005F059FBDBF8C9
:108C980000402401E4B20BF1040B06AB9B454FEAFC
:108CA8009909A0D1B8F1010F02D1204605F048FB7F
:108CB800DAF8003013F480541FBFB7F86420B6F810
:108CC8006410521A029218BF01249A040AD50AAAFB
:108CD80002EB8401B6F86600B7F86620121A41F86C
:108CE800202C013418040BD50AAB03EB8402B6F828
:108CF8006810B7F868305B1A42F8203C013400E08D
:108D0800FCB1012C03D1029805F0CBFB19E0631EDE
:108D1800002002AA400052F82320C0B20AB140F055
:108D28000100013BF5D505F00BFB4FF0000802AB45
:108D380053F8280008B105F0B4FB08F10108A04574
:108D4800F5DB30200321FFF797FC36200321FFF7DE
:108D580093FC2F4B3C201978FFF78EFCDAF8003093
:108D6800990506D5B7F95E00B6F95E30C01A05F068
:108D780098FB2A6827486B686A60121A9110264A7D
:108D8800AB604A43531C032293FBF2F202EB42020C
:108D98009A1A6C2303FB02032B60204B1B681A06EC
:108DA80030D51F4C1F4D22682B689A420BD1626840
:108DB8006B689A4207D1019B1B88102B11D11A4B63
:108DC8001B885B060DD1482005F0BAFA206805F02B
:108DD80068FB606805F065FB23682B6063686B605F
:108DE8000EE0124A0F4B11782A7C914208D1104AA2
:108DF80099681068884203D15268DB689A4201D0AA
:108E0800FFF75CFC05F06CFA0BB0BDE8F08F00BF13
:108E180017200020B424002013DA4B6830260020E5
:108E280064110020942400200A260020061900203E
:108E3800081900202DE9F84F0C9E3A4CC2EB030BA1
:108E48000B9BF61A6368002914BF4FF0060A4FF00F
:108E5800040A01330546904613D1236853455ED270
:108E6800314A324852F82320032B98BF294605F08F
:108E780055FA6368013363602D4B002205469A71E9
:108E880013E0002511E02B4A1278954240DA0B9B3B
:108E9800E3B109FB06F2995C01228A402649096878
:108EA8000A4213D1636801336360D4F804900A9BC3
:108EB8001C4F9945E7DB2BD10A2005F041FA3B68A6
:108EC80001333B604FF0FF337B6021E0184A917912
:108ED80021B12C2005F034FA013501E0012191710E
:108EE800226809FB0BF308EB030752B958F8030093
:108EF80005F004FA97F904104B1C0544D2D00F482A
:108F080002E03A440E48117905F008FA0544C9E729
:108F1800206850452CBF00200120BDE8F88F0020B4
:108F2800BDE8F88F14260020B44301080261010847
:108F3800141D0020F8000020FC2500201161010804
:108F4800F961010830B585B004AC002524F8025D4C
:108F58000091ADF8060021461020FFF751FC9DF85E
:108F680006002146FFF74CFC9DF807002146FFF755
:108F780047FC9DF800002146FFF742FC9DF80100E0
:108F88002146FFF73DFC9DF802002146FFF738FC1B
:108F98009DF803002146FFF733FC9DF80E00C043FF
:108FA800C0B22946FFF72CFC05B030BD10B5054C02
:108FB800206802F0CCF818B1206802F0C5F8F6E78E
:108FC80010BD00BF8419002013B5044601A900682C
:108FD80003F012FE132003F04BFEBDF9040003F06A
:108FE80035FE1B2003F044FEBDF9060003F02EFEFB
:108FF800232003F03DFE2368002BB4BF53204E20EE
:1090080003F024FE01A9606803F0F6FD122003F0C6
:109018002FFEBDF9040003F019FE1A2003F028FE04
:10902800BDF9060003F012FE222003F021FE63685A
:10903800002BB4BF5720452003F008FE02B010BD36
:10904800F0B50124B0FBF4F58D4201D34C43F9E7A8
:109058000026D4B1B0FBF4F504FB1500B4FBF1F421
:109068001EB9002D01DC002CF3D1092D03F1010EEE
:10907800EFB204DD002A14BF3725572500E030255C
:109088003D441D7001367346E3E71C70F0BDF0B532
:109098000124B0FBF4F58D4201D34C43F9E70026D7
:1090A800D4B1B0FBF4F504FB1500B4FBF1F41EB920
:1090B800002D01DC002CF3D1092D03F1010EEFB2D4
:1090C80004DD002A14BF3725572500E030253D442C
:1090D8001D7001367346E3E71C70F0BD2DE9F843B7
:1090E800089E002B07468846144614BF4FF03009E7
:1090F8004FF02009334613F8012B0AB9254603E03F
:10910800002CFBDD013CF6E7002D04DD384649461E
:10911800C047013DF8E724EAE4743546A01B28441B
:1091280015F8011B11B13846C047F7E7BDE8F883C9
:10913800014B186802F00EB8E810002090ED017A93
:1091480007EE901AB5EE407AF1EE10FA01BFF8EE8C
:10915800E77A9FED0E7A67EE877AB7EE007A04BF5A
:10916800C7EE277AC0ED017A90ED017AD0ED007A4A
:1091780030EE877A30EE670AC0EE870AE0EE807A32
:10918800B0EE670AC0ED007A704700BFDB0FC94038
:1091980010B50278202A034600F10100F9D0092A07
:1091A800F7D02D2A03D10346BFEE000A04E02B2A8C
:1091B80008BF0346B7EE000ADFED387A1A461346B1
:1091C80012F8010BA0F13001CCB2092C0AD807EE35
:1091D800101AB8EEC77AF2EE046AA7EEA67AF0EE95
:1091E800477AECE72E2816D1F2EE046A1146B0EE63
:1091F800666A0B4611F8012B303AD0B209280AD812
:1092080007EE102AB8EEC77A87EE267A66EE866AE7
:1092180077EE877AEDE71A7802F0DF02452A35D132
:109228005A782D2A02D10233012004E02B2A14BFD8
:10923800013302330020013B002213F8011F3039AB
:10924800CCB2092C03D80A2404FB0212F5E7B2F5C4
:109258009A7F28BF4FF49A721346B7EE007A072B0D
:1092680005D9DFED0F6A083B27EE267AF7E702F00B
:1092780007032BB1F2EE046A27EE267A013BF8E7E2
:10928800F0EE476A20B1C7EE877A03E0F7EE006A8E
:1092980067EEA67A20EE270A10BD00BF0000000086
:1092A80020BCBE4C30B52DED028B87B0B0EE408AA5
:1092B8000C220021054603A809F0FFF9B5EEC08A83
:1092C800DFED2A7AF1EE10FACCBF38EE278A38EEB5
:1092D800678ADFED277A28EE278A6946FDEEC87A85
:1092E80017EE904A84EAE470A0EBE47005F02EFBD8
:1092F800002CACBF20232D2368468DF80C3009F0D4
:1093080020FA012807D130238DF80D308DF80E3062
:109318008DF80F300CE0022805D130238DF80D3080
:109328008DF80E3004E0032804BF30238DF80D308B
:10933800694603A809F0E8F903A809F002FA033816
:10934800C4B2224603A9284609F028FA00232B555F
:109358002846084909F0D8F903AB2846191909F035
:10936800D3F9284607B0BDEC028B30BD6F12033A23
:1093780000007A443561010870B50646154608466E
:10938800B6FBF2F414B12046FFF7F6FF05FB1464B0
:10939800024B1B5D00F8013B70BD00BF376101083F
:1093A8002DE9F04F814689B08A4616461C460025AD
:1093B8003178002900F0DD80252902D001364846A1
:1093C80075E07278302A08BFB278A2F1300319BF6D
:1093D800B71C4FF0000BF71C4FF0010B092B4FF097
:1093E800000819D8A2F13003D9B2092905D80A22F0
:1093F80002FB083817F8012BF4E7A2F16103052BEB
:1094080002D8A2F1570305E0A2F14103052B03D8C6
:10941800A2F137030A2BEADD6C2A31D13A78642AA3
:1094280007F1010600F083800BD8252A3DD003D828
:10943800002A00F09E80BBE7582A0CD0632A19D076
:10944800B6E7732A22D002D86E2A37D0B0E7752A39
:109458005CD0782AACD1271D2068A2F1580462425A
:109468004FF01001624155E02CD9582A32D0632AB6
:109478002AD13E4648462178271DD04701350FE0BE
:10948800642A64D00ED9732A14D13E462368009307
:109498004846514642460023FFF720FE271D054453
:1094A8003C4685E7252ADFD13E4648462521D04758
:1094B80001357DE70AD86E2A06D13E462368043472
:1094C8001D6075E7002A54D03E4671E7752A26D0FC
:1094D800782AF9D1A2F1580304F1040C5A42206801
:1094E800CDF80CC04FF010015A4105ABFFF7A8FDAD
:1094F800DDF80CC03E46644605AB0093484651462D
:1095080042465B46FFF7EAFD054451E72068271D00
:109518000A21002205ABFFF7BAFD3C46ECE704F14F
:10952800040CCDF80CC020680A210022DDE7206871
:10953800002804F1040708DA2D238DF8143040427E
:109548000DF115030A210022E5E705ABFAE72068CB
:10955800002804F1040C0ADA2D238DF81430404257
:109568000DF11503CDF80CC00A210022BEE705ABAA
:10957800F8E7284609B0BDE8F08F0FB413B50B49DA
:1095880004AB08680A4953F8042B09680193FFF7EC
:1095980007FF0446074B186801F0D0FD0028F9D0F2
:1095A800204602B0BDE8104004B07047940800207F
:1095B80090080020E8100020B0EEE06AF0EEC05AF3
:1095C800B4EEE56AF1EE10FAD4BFF0EE656AF0EE9B
:1095D800466AF5EE406AF1EE10FA0BD0B4EEE56A91
:1095E800F1EE10FA54BFF0EE657AF0EE467AC7EE67
:1095F800A66A01E0DFED1F6ADFED1F7A9FED1F7A93
:109608009FED1F5AA6EEA77ADFED1E7AE7EE267ABF
:109618009FED1D7AA7EEA67ADFED1C7AE7EE267A93
:10962800F4EEC65AB1EE677ADFED197AA6EEA75ABC
:10963800F7EE007AE5EE267AF1EE10FAC7EE277A11
:10964800C8BF9FED147AF5EEC00AC8BF77EE677AF7
:10965800F1EE10FA48BF9FED107AB5EEC00A48BF88
:1096680077EE677AF1EE10FA48BFF1EE677AB0EE5E
:10967800670A70470000000039094E3DE3B59EBEF9
:1096880069A2163E88FA16BE45FE7FBFA7DFA8B4BA
:1096980099FB243FDB0FC93FDB0F4940FDEEC07A41
:1096A80017EE903A2033402B43D8DFED237AB4EEFF
:1096B800E70AF1EE10FA04DDDFED207A30EE670AF2
:1096C800F3E7DFED1F7AB4EEE70AF1EE10FA04D5FE
:1096D800DFED1A7A30EE270AF3E7DFED1A7AB4EEF7
:1096E800E70AF1EE10FA04DD30EE670A37EEC00A39
:1096F8000AE09FED157AB4EEC70AF1EE10FA44BFFE
:1097080030EE270A37EE400A60EE007ADFED0F6A86
:109718009FED0F7AA7EEA67ADFED0E6AE7EE876A6D
:109728009FED0D7AA7EEA67A20EE276AA6EE070A25
:1097380070479FED060A7047DB0F4940DB0FC940B1
:10974800DB0F49C0DB0FC93FDB0FC9BF00000000BA
:1097580092E741B99730083C15A82ABEDFED027A96
:1097680030EE270A9AE700BFDB0FC93F064B1A887D
:1097780022EA0000904210B518801C4602D0012051
:10978800FDF766F9208810BDC4190020064B1A8819
:109798001043904210B518801C4602D00120FDF7F6
:1097A80057F9208810BD00BFC4190020024A9368E9
:1097B80023EA000090607047D811002008B5104BCC
:1097C8001A780023D9B2914207D20E4951F82310D2
:1097D8000968002008600133F4E7322001F08FFCAB
:1097E800094B1B685A0309D5084B9B685B0305D4D2
:1097F80040F2DC50BDE8084001F081BC08BD00BF64
:10980800172000202020002030260020D81100201A
:109818002DE9F34105F0F6FE454A6C2313704FF429
:10982800E2635380BE231371EF2382F80D370023C0
:1098380082F80E3719461646F25C0133B3F5E26F2B
:1098480081EA0201F8D13A4B83F80E17394B1A69AD
:10985800120604D5384A5A6002F188325A60042741
:109868000020013F17F0FF074FD0324B3422DA6057
:10987800002444B1002356F80480019305F036F81B
:109888000428EED117E005F031F80428E9D1294D74
:109898002B6943F002032B61284B6B612B6943F062
:1098A80040032B6105F022F82B69042823F00203FA
:1098B8002B61DFD0D5E71F4D2B6943F001032B61E6
:1098C80004F1006303F57E331FFA88F21A8005F06D
:1098D8000DF8042810D11A4B23440193019B4FEA39
:1098E8001848A3F8008005F001F82B69042823F034
:1098F80001032B6105D0B4E72B6923F001032B6129
:10990800AFE70434B4F5E26FB3D10A4A1369042807
:1099180043F08003136102D104F044FA10B9052022
:10992800FDF7AEF805F05CFE02B0BDE8F08100BFBF
:10993800D8110020002002402301674500F80308E1
:1099480002F8030810B50E4C2068FCF7B1FF206838
:10995800047A002202FB02F3193B634303F6C413A3
:109968005343192193FBF1F3064921F812300132D0
:10997800072AEFD10449BDE81040FCF74FBF00BFEC
:109988005C110020B8100020181300202DE9F041C8
:1099980004F008FA10B90420FDF772F8AB4CAC4D8E
:1099A80005F030FEAB494FF4E262204608F07AFE3B
:1099B80094F8E436022B84BF002384F8E43694F844
:1099C800E4264FF4CC7101FB02F3E018234400F5C0
:1099D8000770286093F8700203F51A73022801FBD8
:1099E800024284BF0020187292F870329A4A1370AB
:1099F8000C2202FB0343994A03F2E6631360A3684F
:109A080046F209021A401AB9904A43F40053936087
:109A1800A368D80703D54FF40050FFF7C7FEA36823
:109A2800590409D50820FFF7C1FE4FF40050FFF78D
:109A3800BDFE0120FFF7BAFEA3681A0706D54FF44A
:109A48000050FFF7B3FE0120FFF7B0FEA3689B04A8
:109A580002D54020FFF7AAFE012284F80D2294F8CF
:109A6800DE217A4B2AB193F8E22112B1002283F861
:109A7800E2217B4B7B4E1E604FF0000C674604EBE7
:109A88000C03B3F8F6E14FEA5E0101F077314FEAD3
:109A98009E0303F03333C1EB0E00C11A4FEADE0315
:109AA80003F01133CB1A03EB23131EF0010803F064
:109AB8000F324FF0FF0392FBF3F3C3EB032318BFFE
:109AC8000137A2EB030318BFFFB2012B0ADD022BFB
:109AD80040F0B980B8F1000F00F0B5801EF0BC0F5F
:109AE80000F0B1800CF1080CBCF1180FC7D1013F90
:109AF800012F00F2A880FFF725FF302200215A48E5
:109B08005A4F08F0DAFD5A4BD5F800801F60594BC0
:109B1800002108F17900C3F80080FCF709FF564BD3
:109B280080F001001870554B07F128021A60544B59
:109B380007F1CC021A6098F8000001F044FD28688B
:109B4800504B00F5C5721A6000F0CAFC4E4B94F8F1
:109B5800D601DFED4E6A07F196021A6064214C4B7C
:109B6800C82211FB00225A6000229A60DA601A614A
:109B78005A619A61DA6183F8202083F82120454BE5
:109B880007F12E021A602A68434B92ED187A02F206
:109B980019111960414B02F289111960404B07F104
:109BA800080119603F4B1F603F4B07F1A201196084
:109BB80067EE266A3D4B07F1AC01B6EE007A1960F4
:109BC80087EE267A3A490E60B4F86411181D07EE3C
:109BD800901AB4F86611F8EE677AC3ED027A07EEC8
:109BE800901A92F85C10197192F87810597194F8DB
:109BF800E1111974F8EE677AB2F81611C3ED037A19
:109C080007EE901A2B49F8EEE77A08605A6183ED5F
:109C1800077A9FED297A1A62C7EE277A02F1640162
:109C280099612649DF62BDE8F0419FED257A67EE2C
:109C3800877AC1ED007A02F1680102F211125962C5
:109C48009A6205F0CDBC04F01DFE54E7D81100203F
:109C58003C11002000F80308102300205C110020AC
:109C68007026002060130020FC0A00201813002032
:109C7800300B0020340B002001000020A40100203C
:109C88002C0A00203C0B002024220020DB0F494036
:109C98007C2600200C020020101D0020400400201B
:109CA800682100206C210020540300201C1D002086
:109CB80018040020800200200000614450030020A6
:109CC8004C3D0F4408B5FFF7A3FDFFF75FFE0120E9
:109CD800BDE80840FCF7BCBE07EE900AF8EEE77A4C
:109CE800DFED0C6A9FED0C0AF5EEC07AF1EE10FA82
:109CF800D4BFB1EE677AC7EEA67A08B5D8BFC7EE6B
:109D0800267A27EE800AFFF729FD044B83ED000A27
:109D180008BD00BF8096184B35FA8E3C5C000020C9
:109D28002DE9F0410369C76805460E461F40002F1C
:109D380035D0B7FA87F24FF00043D340DB432B61AD
:109D48001F40A2F11B03042BF1D8DFE803F0221F08
:109D58001C190300746A24B1013C0023A4B2736285
:109D680001E0EC6AA4B2D6F82080B8F1000FDED08A
:109D7800D8F80030404621469847D8F80480F4E7E0
:109D88003068696B07E07068A96B04E0B068E96B3C
:109D980001E0F068296C036889B29847C7E7BDE815
:109DA800F081F8B5994B1B680546187818B1012859
:109DB80000F06181D9E2242D954C0CD006D80A2DEB
:109DC80000F0D7800D2D00F0D4803FE12A2D06D079
:109DD8002C2D04D03AE120706070A07047E18D4BC3
:109DE800617827788A4A002058542FBB1978D77091
:109DF800472921D1597850291ED19978472907D167
:109E0800D978472904D11979412901D10121D17083
:109E18009978804A522903D1D1784D2900F0A78238
:109E280099787C4A472907D1D178532904D11279E6
:109E3800562A04BF0322E270E278754E022A38D00F
:109E4800032A4BD0012A40F08380BA1E072A7FD804
:109E5800DFE802F004080F131A257E2A05F0B8F986
:109E6800606075E01B78532B72D163685B42636056
:109E78006EE005F0ADF9A0606AE01B78572B67D15A
:109E8800A3685B42A36063E01B78302B624B1A78AF
:109E98008CBF42F0020222F002021A7058E0002041
:109EA80005F0F6F9207353E0002005F0F1F9E081A0
:109EB8004EE0072F06D0082F4AD1012005F0E8F917
:109EC800708245E0012005F0E3F941F21843584358
:109ED8004FF47A73B0FBF3F0308239E0022F07D0E9
:109EE800032F0AD1002005F0D3F94C4B18702FE04E
:109EF800002005F0CDF930752AE029D93A1F9210D3
:109F0800337D0132D2B2013B02EB8303DBB2102B6B
:109F18001ED8F91EC2F1010201EB8202D2B2012A57
:109F28000BD0042A11D100205E1E05F0B1F93C4B7C
:109F380098553C4B00229A5507E05E1E3A4A00208D
:109F4800935505F0A5F9394B9855A3690133A361D9
:109F58002F4B2A2D18BF9A7807F101074FF0000000
:109F68000CBF01225540277060700CBF1A779D7096
:109F78007DE0207F002846D02D4B13F8012D2D4978
:109F88005A708B42F9D1234A214D13785278402BCD
:109F980085BF373B1B011B01DBB298BF03F0F00301
:109FA800402A8CBF373A303AD2B21344A278DBB297
:109FB8009A4225D121230B70E8782B6A1D4A013378
:109FC80001282B620AD002281CD1722313701A4B65
:109FD8002A8A1A80194B6A8A1A8013E06723137039
:109FE8000D4B1B789F070ED5154B6A681A60AA6837
:109FF8005A60144B2A7B1A70134BEA891A8002E0C4
:10A008003F230B7000200023237730E09C010020C1
:10A018004C1D00205C26002000190020781100202B
:10A02800A911002099110020791100208911002020
:10A03800280A0020140A00200219002060110020BC
:10A048000819002006190020041900206378207FD1
:10A058000E2B9FBFAA4A591C5170AA4A98BFD554C3
:10A06800A74A18B993785D40957000E00020003049
:10A0780018BF0120F8BDA24B93F82410002208292C
:10A0880000F27381DFE801F0050C101A2B3B5F7BAF
:10A098008800B52D40F0698183F8252001224FE022
:10A0A800622D08BF02224BE0032283F8242083F8A4
:10A0B800265083F8275083F8285056E1042283F865
:10A0C800242093F8272093F8281083F829502A444D
:10A0D800D2B283F827200A4483F8282045E10522D4
:10A0E80083F8242093F8272093F828105D852A44C4
:10A0F800D2B283F827200A4483F8282035E10622C3
:10A1080083F8242093F8272093F828102A44D2B201
:10A1180083F827200A4483F828205A8D02EB052566
:10A12800ADB2B5F5AC7F88BF754A5D8584BF0121A6
:10A1380082F8251000229A85002D40F0168107220A
:10A1480083F8242011E193F8272093F828102A4453
:10A15800D2B283F827200A4483F828209A8DB2F5D2
:10A16800AC7F3CBF6649891802F1010238BF81F80B
:10A178003050598D92B291429A85E0D9F5E0082283
:10A1880083F8242093F82730AB4200F0EE805C4B34
:10A19800012283F825200FE05B4C83F8242014F873
:10A1A800012D6270594A9442F9D193F82810544A03
:10A1B800A94206D03F232370554A536801335360A0
:10A1C800D3E0116A92F825000131116210B13E23E3
:10A1D8002370CAE02121217092F82910062941D064
:10A1E80004D8022907D0032923D0F8BD122959D051
:10A1F800302967D0F8BD502121704649546B4C6016
:10A20800946B0C60116C4FF47A7491FBF4F1424C2E
:10A21800218092F88811414A19B1117841F0020160
:10A2280002E0117821F002011170012283F88921DE
:10A238008DE05321217092F83510CE0705D592F89C
:10A248003420D51E6A426A4100E0024602F001014C
:10A2580083F88811002A7AD130490A7822F002025C
:10A268000A7074E04F21217092F83B10CC0705D595
:10A2780092F83A20D11E4A424A4100E0024602F0D2
:10A28800010183F8881122B924490A7822F00202D0
:10A298000A70234A93F85F101170224AB3F85C10D1
:10A2A800118054E0562121701F49546C0C8042F2F1
:10A2B8001074916C91FBF4F11C4C2180012182F8FF
:10A2C8008A1144E04921217092F83410184A102963
:10A2D80088BF10211170174914780022A24233D286
:10A2E800154D0E7A5655154D4E7A5655144DCE7A53
:10A2F8005655144D11F80C6F56550132EEE700BF54
:10A308004C1D00205C260020280A0020140A00208A
:10A318007C010020081900200419002000190020E1
:10A3280006190020EE00002002190020601100200C
:10A33800781100207C1D002079110020891100204F
:10A3480099110020A91100209A6901329A6193F8A5
:10A3580089310B4A93B192F88A317BB1002182F896
:10A36800891182F88A111846F8BD0020F8BD1279C3
:10A37800432A7FF455AD0222E27051E5F8BD00BFD3
:10A388004C1D00200449054B0968187000225A61C9
:10A3980099611A77704700BF542600207C0100207D
:10A3A80010B5121A07EE902A5B1A2DED028BF8EE03
:10A3B800E78A07EE903A184B059CB8EEE78AD3ED8A
:10A3C800007A28EE278A28EE080AA8EEA80A08F0DC
:10A3D8005BFCDFED127A049B20EE270AF0EE480AB8
:10A3E800BCEEC00A83ED000AB1EE680AFFF7E4F894
:10A3F800DFED0B7A9FED0B7AE0EE077ABDEC028B6E
:10A40800FDEEE77A17EE903A002BBCBF03F50C433C
:10A41800A033236010BD00BF5C0000202C7D8E3F60
:10A4280000A00C46A00CB34544F25063984203DDEB
:10A43800A0F50C40A0387047034B9842BCBF00F50C
:10A448000C40A030704700BFB0B9FFFF73B51A4C7D
:10A45800036823600B686360184D0068184EFFF7A7
:10A468003BFC184B009395E8030094E80C00019618
:10A47800FFF796FF144B32681A60686863681349DF
:10A488001B1A07EE903A124B286893ED007A23685E
:10A498001B1A0B600F4BF8EEE77A1A600E4B67EE4B
:10A4A800877A1B68FDEEE77ADA880C4BC1ED017AF2
:10A4B8001A8002B070BD00BFB02200200819002029
:10A4C800BC220020B8220020F8220020C022002050
:10A4D8005C000020F02200203C0B0020EC22002031
:10A4E8004279DFED2A5A2A4B9FED2A5A07EE902A25
:10A4F800F8EE677AC27BC7EEA57AB2EE047AC3EDAE
:10A50800007A07EE902AF8EE677A234ADA60C7EEF7
:10A51800A57AC3ED017A8179204B07EE901AF8EEFF
:10A52800677A017CDA60C7EE877AC3ED007A07EEB6
:10A53800901A817E06EE101AF8EE677AB8EE466A2F
:10A54800C7EEA57A86EE056AC3ED017A83ED026A45
:10A55800C179134B06EE901A417CDA60F8EE666A10
:10A56800C6EE876A07EE101AC17EC3ED006A07EED1
:10A57800901AB8EE477AF8EE677A87EE257AC7EE32
:10A58800857A83ED017AC3ED027A70470000C842EC
:10A59800C822002000007A440000FA44D822002093
:10A5A800FC22002010B50C4C23789B0713D50B4BCD
:10A5B8001B78042B0FD90A4A0A4B106852685A6054
:10A5C8001860FFF789FB084B1A88084B1A80237814
:10A5D80043F00103237010BD001900200619002064
:10A5E8000819002064110020CC1100200C23002041
:10A5F8001C4B1B681B0307B530D51B4A1B4BD2ED00
:10A60800007A1B788DF80030B2EE047A67EE877A0C
:10A61800174B9FED187A1B788DF80130FCEEE77A1E
:10A628000A2017EE903AD2ED017A8DF8023067EEE3
:10A63800877A6946FCEEE77A17EE903AD2ED027A0D
:10A648008DF80330FCEEE77A17EE903A8DF8043077
:10A65800094B1B788DF80530FEF70EF903B05DF84D
:10A6680004FB00BF302600204426002020260020BE
:10A678004026002000007A4424260020054A13784A
:10A6880083F001031370044A00231360034A136024
:10A69800AEE700BF242600203C26002038260020F4
:10A6A80001480249FFF73CBB004801404021002017
:10A6B80001480249FFF734BB00400140F020002068
:10A6C80001480249FFF72CBB00080040C8200020C1
:10A6D80001480249FFF724BB00040040A0200020E5
:10A6E8004FF080400149FFF71BBB00BF78200020D6
:10A6F80010B5064C06482146FFF712FB04F1C801C5
:10A708000448BDE81040FFF70BBB00BF50200020F5
:10A71800002C01400044014001480249FFF700BBFA
:10A72800002C014050200020224B10B5224C5A43E7
:10A73800224BB3FBF2F203880139013AA04289B2F5
:10A7480092B29BB20ED004F50064A0420AD0B0F1D8
:10A75800804F07D0A4F59834A04203D004F5806454
:10A76800A04202D123F070039BB2154CA04206D040
:10A7780004F58064A0421CBF23F440739BB203809D
:10A788000D4BC162984202850FD003F500639842D1
:10A798000BD003F54063984207D003F580639842D5
:10A7A80003D003F58063984201D100230386012377
:10A7B800436110BD40420F00002C014000A24A0432
:10A7C80000100040134B800A984220D00AD84A3B18
:10A7D800984212D00133984211D0B0F5801F14D19D
:10A7E800012070470C4B98420BD0013398420AD095
:10A7F800023B984209D10420704702207047032089
:10A8080070470520704706207047FE2070470020DB
:10A81800704700BF4B00100051001000F8B50468E5
:10A82800064620460F461546FFF7CCFF06284BD8AC
:10A83800B27A910847B902238B40D4F80CE0DB4385
:10A848009BB203EA0E03E3600A23204A03FB0013CA
:10A8580042F82370043342F8235015463FB1B17AC9
:10A86800E268890802238B409BB21343E3602822E5
:10A8780002FB00522032EFF31286502383F3128832
:10A8880003B203EB8303DB0003F10C011C332944FF
:10A898002B4451F8047F17B117600A6804329942B3
:10A8A800F7D100231360F3B283F31188282303FB45
:10A8B8000050036A1BB1E36843F0010303E0E26858
:10A8C8004FF6FE731340E360F8BD00BF5020002030
:10A8D8000148F8F775B800BFD81E00200148F8F7FE
:10A8E8006FB800BF2C1F0020034B4FF4806208B1E3
:10A8F8009A6170471A85704700040048034B4FF46B
:10A90800806208B11A8570479A6170470004004850
:10A918002DE9F04F2DED028B87B0074603938C4B42
:10A928001B889807934636D5129B8A48DC89B0F96C
:10A9380000301B1B03F2F31540F2E632954203D8B0
:10A94800002BB8BF5B4201E04FF4FA73B0F9022064
:10A95800121B02F2F31440F2E630844203D8002AB4
:10A96800B8BF524201E04FF4FA729342B8BF13469F
:10A97800C3F5FA73052293FBF2F33A7F0A25643B89
:10A988006B43D2105343642593FBF5F5643525EAF0
:10A99800E575EBB200E064230193CB1C0293B84643
:10A9A8000025029BDFF8CCA113F8016F0293022D5A
:10A9B8004FEA450905D1BAF904201B3656437611EA
:10A9C80046E065483AF8151030F91500022411FBE5
:10A9D8000400CBF10001884203DB58450146A8BFBB
:10A9E80059465E48039B30F909400C1B33F9151092
:10A9F8000C4400F00DFE88B107EE904A5849B8EEB5
:10AA0800E70AB2EE048A485D80EE080A04F052FABA
:10AA180020EE080AFDEEC07A17EE904A4C490988E4
:10AA2800CA0712D43AF909201B3656438B074FEA56
:10AA380026160DD5BA7C54439DF90420544364224C
:10AA480094FBF2F406EB241602E03E7A74432611D6
:10AA5800444A98F8011032F90920042492FBF4F4CE
:10AA6800414A341BAE5C614371436420022D91FB63
:10AA7800F0F14FEAE11308EE103A09D1B8EEC80A2E
:10AA8800101D1E21D2ED030AFEF758FBBDEEC08A49
:10AA9800354B364803F110014FEA850C51F8252053
:10AAA800B2F5001FA8BF4FF400128242B8BF024699
:10AAB80041F8252003F11C01521351F8250041F8F3
:10AAC8002540201A00214FF6FF74B4FBF1F189B23A
:10AAD8004143891100EE101A97F8501089B103F11B
:10AAE8002800B8EEC00A00EBC500D3ED030ACDF884
:10AAF80014C00492FEF722FBDDF814C0049ABDEEE0
:10AB0800C00A98F8151010EE103A594318EE103A8A
:10AB18004E439818642196FBF1F6154936123044D5
:10AB280021F8090001F1080001354CF8003001F165
:10AB380014002031032D4CF800204CF8016008F176
:10AB480001087FF42EAF07B0BDEC028BBDE8F08F93
:10AB5800C4190020481B0020C626002026260020F5
:10AB6800CC43010824110020801F00200000E0FFD2
:10AB7800C01F0020D01100202DE9F04F2DED0A8BC9
:10AB880085B08246039390F85030029190461BB1ED
:10AB9800322BA8BF322300E0012307EE903AB8EE2B
:10ABA800E7BADFEDD97AD94BDFEDD9BA1B88D94C92
:10ABB800019487EE8BBA002B08BF0123D64D07EE10
:10ABC800903AF8EEE79A238869EEABBA13F0020FD1
:10ABD8003BEE2BBA8BEE8BBA26D0B5F90030B5F91F
:10ABE800022083EAE37182EAE270A1EBE371A0EB51
:10ABF800E27088420646B8BF0E46B6F5E17F16DA1F
:10AC08008842DFEDC6AA05DD002AD8BF524207EE0A
:10AC1800902A04E0002BD8BF5B4207EE903AF8EE8A
:10AC2800E77AC7EEAAAA04E0DFEDBDAA01E0F7EED5
:10AC380000AA9FEDBB9ABB4C56464FF0000BB0EEF6
:10AC480049AADFF8189339F91B300CEE103AB8EE20
:10AC5800CCCAF5EE047A35F91B302CEE27CA08EE7B
:10AC6800903A019BBDEECCCA1988F8EECC7A9FEDDC
:10AC7800AECA89074FEA4B0727EE8CCAF8EEE88A76
:10AC880000F08580A94931F91B3007EE903AF8EEBB
:10AC9800E77AB0EE007AE8EE877AC8F10000FDEEB8
:10ACA800E77A17EE901A814203DB4145A8BF414677
:10ACB80008469F49039B795E401A33F91B100844E4
:10ACC80007EE900AB8EEE78A00F0A2FC50B1994965
:10ACD800B2EE049A88EE090A11F80B0004F0EAF8BB
:10ACE80020EE098A9AF81C30DFED936A0AEE103AD2
:10ACF8009AF8083007EE903AF8EE677AB8EE4AAA62
:10AD080068EE277AB1EE047A67EEA67A2AEE077A19
:10AD1800FDEEE77A17EE901AF1EE477ABDEEE7AA54
:10AD28001AEE103A994208DBBDEEC7AA1AEE103A9D
:10AD38008B42A8BF0B460AEE103A804901EB8B0103
:10AD4800D1ED007AE8EE2B7ABBEE0E7AF4EEC77AF4
:10AD5800F1EE10FAB8EECAAA09D4B3EE0E7AF4EE00
:10AD6800477AF1EE10FAC8BFF0EE477A01E0F0EE4C
:10AD7800477AC1ED007A9AF8123009EE103AB8EE27
:10AD8800499A67EE897A9FED6E9A27EE899A019B18
:10AD98001988CA0750D439F907000028B8BF4042BB
:10ADA800B0F5206F02DD0020206025E09FED657A78
:10ADB800737868EE877A07EE103AB8EE477A87EE2E
:10ADC800877AD4ED007A37EE4C7AE7EE2B7A9FED4E
:10ADD8005E7AF4EEC77AF1EE10FA09D49FED5B7A49
:10ADE800F4EE477AF1EE10FAC8BFF0EE477A01E0C8
:10ADF800F0EE477AC4ED007AF37AD4ED007A08EEE3
:10AE0800103AB8EE488A8B0768EE277A9FED508A89
:10AE180027EE888A14D578EECA8AF0EE4A7AEAEEE6
:10AE2800A87A38EE498AF0EE678AF0EE497AEAEEB7
:10AE3800887AB0EE678A03E0B0EE498AF0EE4A8A73
:10AE4800DFF81C919FED437A09F1800109F1840034
:10AE58001BF8013007EE903AF8EEE77A4FEA8B01DB
:10AE680067EECC7A0844E7EE878A0434013690ED21
:10AE7800007A80ED00CA3CEE477A09F18C0087EE33
:10AE88002B7A0144D1ED007A37EE677AF0EE68CA82
:10AE9800EBEE077A3CEE880AC1ED007A09F19401DD
:10AEA8001BF8013008EE903AF8EEE88A67EEA87AC7
:10AEB800DFED298A67EEA88A30EE680A07F00CFEF3
:10AEC80009F14001FDEEECCAC8531CEE903A09F1B5
:10AED8004801BDEEC88AF1EE688A41F82B30FDEED4
:10AEE800E88A09F1540118EE103A41F82B3009F1BB
:10AEF800600118EE903A4F4641F82B30BBF1000F35
:10AF080030D14FF0010B9CE683F9223EF810002067
:10AF1800BD378635C4190020D01100200000E14358
:10AF280000000000EC1F0020CDCC4C40C6260020BD
:10AF380026260020CC4301086F12033CF81F00208E
:10AF48000AD7A33D0000A043000040C300004043CF
:10AF58000AD7233CA69B443BF7CC92382411002007
:10AF6800801F0020029AB5F90430947964002834CF
:10AF78005C434B4BB3F9043000EE103ABAEECF0AFB
:10AF880007F0AAFD6411201A002C07EE900AB8BF3A
:10AF98006442322CF8EEE76A03DD0023C9F8183062
:10AFA80029E0FDEEE99A19EE903A23F0030307EE43
:10AFB800903AF8EEE79ADFED3B7A9AF80D30C9EE51
:10AFC800A77A07EE103AB8EE477AD9F8183026EE85
:10AFD800877A67EE277AFDEEE77A17EE902A134410
:10AFE800314A9342A8BF1346304A9342ACBFC9F8CE
:10AFF8001830C9F81820BB695B13B3F5807FA8BF68
:10B008004FF480736FF0FF029342B8BF134607EE08
:10B01800903AF8EEE78AFDEEE67A9AF8032017EE02
:10B02800903A53439B1107EE903A97F89730032BC9
:10B03800B8EEE78A14D9BAF84E20B2F5FA7F0FD2E3
:10B04800FDEEC87A534217EE901A994204DB9142FA
:10B0580017EE903AA8BF134607EE903AB8EEE78A83
:10B0680038EE280ABDEEC00A8DED010ABDF904309C
:10B0780000EE103AB8EEC00A07F02EFDBDEEC88A01
:10B08800FDEEE88A0023A7F8440087ED148AC7ED8F
:10B09800178ABB6605B0BDEC0A8BBDE8F08F00BF10
:10B0A8002411002000803B45FEFFFF0F020000F046
:10B0B80010B50A4A0A4B11689B6800BF1268914292
:10B0C800F7D1084AD2F898404FF47A7000FB04F29E
:10B0D800D31AB3FBF4F300FB013010BD5426002053
:10B0E80010E000E0801F002038B50446FFF7E0FFBD
:10B0F8000546FFF7DDFF401BA042FAD338BD10B567
:10B1080004462CB14FF47A70FFF7EEFF013CF8E7E4
:10B1180010BD024A1368013313607047542600209B
:10B12800024BD3F89C3003B118477047801F0020AA
:10B13800014B1B68184700BFB026002003681B6935
:10B1480018470368DB68184703689B681847036853
:10B158005B68184703681B6818472DE9F84FB0F972
:10B168000230934218BF00232DED048B18BF0370E3
:10B17800057804460E469146002D40F0978007EE6C
:10B18800902ADFED7D8AF8EEE77AB6EE009A67EE50
:10B19800A88ADFED7A7A68EEA78AA04668EE898ADF
:10B1A8002746B0EE680AFEF779FAB0EE408AB0EEAC
:10B1B800680AFEF7D3FA88EE000A40F2DC536365AA
:10B1C8001023A4F852301823A4F85030DFED6C6A2D
:10B1D80060EE266AB7EE006AB0EE667AA0EE007AF4
:10B1E800D0EE006A37EE067A76EE866AC6EE077A01
:10B1F80084ED046A27EE807AB0EE498A27EE007A59
:10B2080077EE075A84ED017AC4ED025A70EE005ABF
:10B2180084ED037AB8EE007AA5EE807A27EE877A75
:10B2280067EEA67A84ED057AC4ED067ADFED557AE5
:10B2380098ED047A27EE277AF0EE678AB5EEC07AA1
:10B24800F1EE10FA4CBF77EE487A77EE087A0135BE
:10B2580017EE900A04F058FCD8ED017A67EEA87A48
:10B26800C7E90E01F5EEC07AF1EE10FA4CBF77EEA1
:10B27800C87A77EE887A08F1040817EE900A04F085
:10B2880043FC032DC7E9080107F10807CED1A6F250
:10B29800DC531B042367E3676367C4F88030A36744
:10B2A800C4F884300123A4F802902370D4F8549091
:10B2B800B4F95280636A276A206FE26FD4F840C0FD
:10B2C800D4F88010C4F88020C9EB060606FA08F600
:10B2D8004FEAE67B734307FB0B332667A7FB06673A
:10B2E8001F44636C656F60674FEAE27B53430CFB56
:10B2F8000B3EACFB02237344B61A67EB0307E36A01
:10B30800A26AC4F884104FEAE07B434302FB0B3E79
:10B31800A2FB00237344B6185F41E36CA06CB4F938
:10B328005020A5674FEAE17B4B4300FB0B33A0FBA2
:10B3380001011944636B361A206B4FEAE57B05FB64
:10B3480003F300FB0B3367EB0107A0FB050119446E
:10B358008019794104F0A6F908F1FF3201239340DE
:10B36800E067C01841EBE371424604F09BF9BDEC7D
:10B37800048B4844BDE8F88F6F12833ADB0F4940CD
:10B38800F404B53F0000804B2DE9F8430024244B1A
:10B3980093F89760E0B2B0420DD203EB8003214AE4
:10B3A800D3F8A03032F810101BB10B2801D8DB6895
:10B3B80098470134EBE71C4B1B685B032DD5002431
:10B3C8002346E2B2B24228D2DFF8549009F1A0072E
:10B3D8004FEA840857F8242055689D4215D028461E
:10B3E800FFF7F0F9EFF31283502282F31288282135
:10B3F8006A6A01FB00900132C0F8F4206A6942F0E1
:10B4080001026A61DBB283F3118857F808301B68C0
:10B4180000221A6001342B46D3E7BDE8F88300BF49
:10B42800801F0020401100203026002008B50E4B58
:10B438001B6813F4805F0D4B14BFD3F8E821D3F8D1
:10B44800EC2193F8971092880023D8B2884204D24E
:10B45800074820F813200133F7E7FFF795FF32205C
:10B46800BDE808404BE600BF30260020801F0020C2
:10B47800401100200A4B1A680A4B30B502F480527A
:10B48800D3F8E841D3F8EC5100230AB1A18800E0D1
:10B49800A988054820F8131001330C2BF5D130BDCD
:10B4A80030260020801F00201223002070B5124D86
:10B4B8000024214605F2F110702285F8F04107F0CA
:10B4C800FCF82146D5F864320B4A0B4493F9020084
:10B4D80080B102F2F1141E680E5108199C8884800C
:10B4E8009B79837192F8F03107310133702982F822
:10B4F800F031E7D170BD00BF801F0020094B1A68EA
:10B508000E2303FB0020437AFF2B07D0064A12784C
:10B518009A4203D9054A32F8130000E0808800B245
:10B52800704700BF101D00205C240020481B00202D
:10B53800D0ED024A91ED016A90ED015A91ED027A3F
:10B54800D0ED005AD1ED007A66EE646AE5EE076A3E
:10B5580027EE657AC2ED006AA4EEA77A67EEC57A8F
:10B5680082ED017AE5EE867AC2ED027A7047D0ED77
:10B57800017A91ED017AD1ED026A91ED006A37EE18
:10B58800877AD0ED027A77EEA67AD0ED006A82ED5E
:10B59800017A76EE866AC2ED027AC2ED006A7047D9
:10B5A80090ED017AD0ED027AD0ED006A20EE077AAC
:10B5B80060EE277A26EE800A81ED017A81ED000A95
:10B5C800C1ED027A704701380A4B042804D8DFE835
:10B5D80000F00507090B0D00074A08E0074A06E0D6
:10B5E800074A04E0074A02E0074A00E0074A1A60EF
:10B5F800704700BFF0000020A1BC000819A900088E
:10B60800A5BF000899B900083DB6000881AB00083D
:10B61800064B1B7803F0040303F0FF001BB1044B37
:10B628001888C0F3C01000F001007047CC26002035
:10B63800C41900202DE9F04F2DED028B87B00026AC
:10B648000493BD4B0391B3F90270B3F90030019232
:10B65800002FB8BF7F42002BB8BF5B429F42B8BFE4
:10B668001F46B7F5FA7F8046A8BF4FF4FA770090D7
:10B67800B246B446B3463446B04D2B8899075AD0E3
:10B68800AD4BAF4A33F8143032F91420022013FBC3
:10B698000022019B5B429A424FEA440103DB019B73
:10B6A8009342A8BF1346A74A31F90290049A32F987
:10B6B8001420C9EB030303EB0209FFF7A9FF88B1C4
:10B6C80007EE909AA04BB8EEE70AB2EE048A185D2E
:10B6D80080EE080A03F0EEFB20EE080AFDEEC07AC1
:10B6E80017EE909A98F80830642203FB09F393FB4D
:10B6F800F2F398F81C206FF0040B0BFB02FB5B4580
:10B7080004DB02EB820B9B45A8BF9B468F4A52F88D
:10B71800241009EB010342F210718B42A8BF0B46BB
:10B728008B498B42B8BF0B4642F8243098F8122058
:10B7380053434FEA233C2D8805F00303012B38D0EF
:10B748007D4B844933F914A0009B51F824E093F809
:10B758000190814B33F9140080EAE073A3EBE073A6
:10B76800B3F5206F4FEA840616DC0AEB8A031A0148
:10B7780092FBF9F3042290FBF2F0181A8644BEF506
:10B788007A5FA8BF4FF47A5E744B9E45ACBF41F810
:10B7980024E041F8243002E0002341F824308B599A
:10B7A8007D2693FBF6F6009BDB7A7343402693FBDA
:10B7B800F6F6AA0710D5C7F5FA7307FB0AF907FBCF
:10B7C80006F54FF4FA7103FB0B9903FB0C5599FB33
:10B7D800F1F295FBF1F505E0EB0759BF3546524606
:10B7E80065465A46630002935D495B4B615C33F8DA
:10B7F80014004FF0040E03B293FBFEF909FB01F1AC
:10B808006FF04F0991FBF9F99144564A32F9141037
:10B8180022F814005B1A98F8501093FBFEF300EE20
:10B82800103A79B1504B5148D3ED000ACDF814C005
:10B83800B8EEC00A00EBC400FDF780FCDDF814C0C8
:10B84800BDEEC00A4A4A029912F804E0494810EECF
:10B85800103A09EB05020EFB03F34FF0200E93FBA1
:10B86800FEF3D21A0A524449444A41F82450444D3E
:10B8780042F824905B4245F82430009B0133009342
:10B888000CB90124F8E62C4B98F80D70B3F9044074
:10B89800039B9B790F335B0063435B112E4C002B9A
:10B8A8004FF00406B4F9044094FBF6F4294EA3EBD8
:10B8B8000404B8BF5B42322BD6F808E00BDC314BEE
:10B8C80007FB04E7BB42A8BF3B462F4FBB42ACBFB8
:10B8D800B360B76001E00023B36098F803305C43BD
:10B8E8002A4B1B78032B4FEAA4140CD9B8F84E3016
:10B8F800B3F5FA7F07D25F42BC4203DB9C42A8BF84
:10B908001C4600E03C46B368946043F34F33B3F5FC
:10B91800807FA8BF4FF480736FF0FF06B342B8BFB3
:10B928003346E6188B6000238680AB6007B0BDEC19
:10B93800028BBDE8F08F00BFD0110020C419002091
:10B94800C626002026260020CC430108EC21002032
:10B95800F0D8FFFF901F00202411002080C1FFFFB6
:10B9680000200020F42100208C1F0020A81F0020A8
:10B9780014200020C01F0020D41F0020C81F002052
:10B98800E01F0020FEFFFF0F020000F0172000203C
:10B998002DE9F04F2DED028B85B080460293A84B20
:10B9A80001911C88009204F00204A4B294B1A54B42
:10B9B800B3F90240B3F90030002CB8BF6442002B41
:10B9C800B8BF5B429C42B8BF1C46B4F5007FA8BF15
:10B9D8004FF40074C24600259A4B9B4833F8152053
:10B9E8009A4B50F8256033F9153083EAE377A7EBD3
:10B9F800E37711B2B7F5206F4FEA450B4FEA4101E3
:10BA08004FEA850911DC042793FBF7F3CB1A1E4490
:10BA1800B6F57A5FA8BF4FF47A568D4B9E42ACBFFD
:10BA280040F8256040F8253002E0002340F8253032
:10BA380050F809609AF80B309AF80170F6115E43D5
:10BA48007F4B1B884F439B074FEAA6164FEAA71761
:10BA580056D0804B33F90B30022112FB0132009B88
:10BA68005B429A4203DB009B9342A8BF13467A4A83
:10BA78003BF902209A1A029B33F91530D31808EEC5
:10BA8800103AFFF7C5FD68B1B8EEC80A734BB2EEBD
:10BA9800048A80EE080A585D03F00CFA20EE080AC2
:10BAA800BDEEC08A6E4918EE102A59F8013042F2EC
:10BAB800107013448342A8BF03466A4898F80820C8
:10BAC8008342B8BF034649F8013018EE101A4A43BA
:10BAD80098F81C1001EB8101D2114842824203DB25
:10BAE8008A42A8BF0A46104698F8122053431B13EF
:10BAF800F61A3F1A6643674303EB662600EB67278F
:10BB0800524ADFF890C13BF802001CF805C003B2A6
:10BB18004FF0040E93FBFEF101FB0CF1A7EBA1170C
:10BB280051493BF901C02BF8010098F85010CCEBB3
:10BB3800030393FBFEF300EE103A69B14B4B4C48FC
:10BB4800D3ED000A0392B8EEC00A00EBC500FDF77A
:10BB5800F5FA039ABDEEC00A4649474811F805E0D0
:10BB680010EE103A0EFB03F3B9195B11C91A2BF842
:10BB78000010424949F80170414F49F80760414EA9
:10BB88005B4249F806300AF1010A0DB9012523E79D
:10BB98002C4BB2F90420B3F90440019B9B790F3375
:10BBA8005B0063435B11002B4FF00405264C92FBAE
:10BBB800F5F5A3EB0505B8BF5B42322BD4F808E0D6
:10BBC80098F80D200BDC304B02FB05E29342A8BF2E
:10BBD80013462E4A9342ACBFA360A26001E0002343
:10BBE800A36098F8032002FB05F3294A1278032A78
:10BBF8004FEAA3130CD9B8F84E20B2F5FA7F07D252
:10BC08005542AB4203DB9342A8BF134600E02B46E4
:10BC1800A2688B6042F34F32B2F5807FA8BF4FF421
:10BC280080726FF0FF04A242B8BF22469C1800231E
:10BC38008480BA60B36005B0BDEC028BBDE8F08FBC
:10BC4800C4190020D0110020901F002024110020CA
:10BC580080C1FFFFC626002026260020CC4301080D
:10BC6800EC210020F0D8FFFFF82100208C1F0020D5
:10BC7800A81F002014200020C01F0020C81F00207B
:10BC8800D41F0020E01F0020FEFFFF0F020000F07D
:10BC980017200020002000202DE9F04F2DED028B09
:10BCA80085B000260293A94B0192B3F90270B3F94B
:10BCB80000300090002FB8BF7F42002BB8BF5B4216
:10BCC8009F42B8BF1F46B7F5FA7F8146A8BF4FF419
:10BCD800FA77B246B346B04634469D4D2B8899074D
:10BCE8005DD0022C5BD0994B9A4933F8143031F966
:10BCF80014104FF0020E13FB0E11019B5B42994288
:10BD08004FEA440003DB019B8B42A8BF0B469249D4
:10BD1800029A30F901B032F91410CBEB030303EBAC
:10BD2800010BFFF775FC88B107EE90BA8B4BB8EEA4
:10BD3800E70AB2EE048A185D80EE080A03F0BAF842
:10BD480020EE080AFDEEC07A17EE90BA99F808308E
:10BD5800642103FB0BF393FBF1F399F81C106FF0CC
:10BD6800040808FB01F8434504DB01EB810898450A
:10BD7800A8BF98467A4951F8243042F210705B44C3
:10BD88008342A8BF0346774899F812B08342B8BFE8
:10BD980003460BFB03FB41F824304FEA2B3B2B886F
:10BDA80003F00301012901D1022C42D16E4D674AEB
:10BDB80035F9145032F914A06C48009A85EAE576F2
:10BDC800A6EBE576B6F5206F92F801E050F824204E
:10BDD8004FEA840120DC022C18D00AEB8A0000010B
:10BDE80090FBFEFE042095FBF0F5C5EB0E0E02EB72
:10BDF8000E0CBCF57A5F5D485D4DA8BF4FF47A5CC8
:10BE0800AC45ACBF41F800C00D5007E08AEAEA76BD
:10BE1800A6EBEA76642EE0DD002545505348009AEB
:10BE280009587D2691FBF6F6D17A7143402691FB9D
:10BE3800F6F69A0712D5022C10D0C7F5FA7307FB4D
:10BE480006F507FB0AF103FB08114FF4FA7003FB30
:10BE58000B5391FBF0F193FBF0F508E0DB0704D5F9
:10BE6800022C02D05D46414601E0354651463E4B24
:10BE780033F91400042390FBF3F33E48205C022CB2
:10BE880003FB00F36FF04F0093FBF0F30B444FEA12
:10BE9800440C08EE103A0ED1374B3848D3ED000A5F
:10BEA800CDF80CC0B8EEC80A1E21FDF747F9DDF839
:10BEB8000CC0BDEEC08A2C4B31493CF803003CF95C
:10BEC80001302CF8010099F850100FFA80FEC3EBEE
:10BED8000E034FF0040E93FBFEF300EE103A79B117
:10BEE800254B2848D3ED000ACDF80CC0B8EEC00A9F
:10BEF80000EBC400FDF722F9DDF80CC0BDEEC00A66
:10BF0800214B22481B5D10EE102A534318EE102ACD
:10BF180051194FF0200E93FBFEF3C91A2CF80010AC
:10BF28001B4941F824201B4941F824501A495B4217
:10BF380041F82430009B01340133032C00937FF433
:10BF4800CCAE05B0BDEC028BBDE8F08FD01100205F
:10BF5800C4190020C626002026260020CC4301084C
:10BF6800EC210020F0D8FFFF24110020901F0020B2
:10BF780080C1FFFF002000208C1F0020841F0020AC
:10BF8800FC210020A81F002014200020C01F002032
:10BF9800C81F0020D41F0020E01F00202DE9F04F0B
:10BFA8002DED088B83B00AEE102A0093D14B019334
:10BFB8001A8812F0020F0546F7EE009A4CD0149B2F
:10BFC800CD48DC89B0F900301B1B03F2F31640F2B0
:10BFD800E632964203D8002BB8BF5B4201E04FF42B
:10BFE800FA73B0F90220121B02F2F31440F2E630A1
:10BFF800844203D8002AB8BF524201E04FF4FA72D3
:10C0080095F84C0058B39342B8BF1346C3F5FA737A
:10C0180007EE903A9FEDB97AF8EEE77A6423C7EE17
:10C02800877A93FBF0F307EE103A77EEE97AB8EEE9
:10C03800C77AB0EE699AA7EE879AF7EE006AB5EE6E
:10C04800C09AF1EE10FA0AD4B4EE669AF1EE10FA3C
:10C05800C8BFB0EE669A04E0B0EE699A01E09FEDC1
:10C06800A89AA84ECF1C2C464FF00008B8F1020F32
:10C0780017F801BFDFF8DC924FEA480AF2EE04AA8B
:10C088000ED1B9F904109FEDA07A0BF10A0B01FB50
:10C098000BF307EE903AF8EEE77AC7EE877A68E096
:10C0A800F8EE4A7A9FED956A39F91830C7EE867A24
:10C0B80006EE903A954B33F9183007EE103A1AEE1F
:10C0C800103AF8EEE66AB8EEC77A5B42A6EEA77AAF
:10C0D80007EE903AF8EEE77AB4EEE77AF1EE10FA66
:10C0E80008D4F8EECA7AB4EEE77AF1EE10FAD8BFBF
:10C0F800F0EE477A864B33F90A3008EE103A009B87
:10C10800B8EEC88A33F9183077EEC87A08EE103AD4
:10C11800B8EEC88A37EE888A88EE2A8AFFF778FA56
:10C1280040B17C4B13F80800B0EE480A02F0C2FE9A
:10C13800B0EE408A019B1988CA0704D5D5ED117A5B
:10C1480068EE277A15E039F90A309FED6F7A0BF11E
:10C15800140B03FB0BF307EE903AF8EEE77A8B0724
:10C16800C7EE877A42BF95ED127A28EE078AE8EE85
:10C17800097A694BDFF8E0B133F90A3094ED08BA6F
:10C188009FED668ADFF8D49107EE103A644BB8EE5B
:10C19800C77AD3ED0A6A18F80B30E7EE667AB8F179
:10C1A800020FF0EE48BAF0EE678A67EE8B7A0BEE74
:10C1B800103AB8EECBBA27EE8BBA8BEE08BA09D193
:10C1C800B0EE4B0A5748D9ED000A1E21FCF7B6FF1E
:10C1D800B0EE40BAD9ED000A94ED0B7A68EEA07A79
:10C1E80067EE877A96ED007AA7EEAA7ADFED4E7AA7
:10C1F800B4EEE77AF1EE10FAF0EE47AA09D4DFEDD3
:10C208004B7AB4EE677AF1EE10FAC8BFF0EE67AA7F
:10C2180001E0F0EE67AA89EEA08A45494FEA88094D
:10C22800494491ED000AC6ED00AAC1ED008A38EE36
:10C23800C00A95F8501020EE080A21B13D4800EBDD
:10C24800C800FCF77BFFD4ED0E7A1BF8083060EECF
:10C25800277A00EE103AB8EEC00A27EE800ADFED22
:10C26800367A80EE2B8AB4EEE78AF1EE10FA09D41A
:10C27800DFED327AB4EE678AF1EE10FAC8BFB0EE9D
:10C28800678A01E0B0EE678A3BEE2A0A08F10108E6
:10C2980030EE080A06F020FC2949B0F57A7FA8BFDD
:10C2A8004FF47A708842B8BF0846BDEECBBA25492C
:10C2B8001BEE103A21F80A00FDEEEAAA2249BDEE6B
:10C2C800C88A49F8013021491AEE903A49F80130F4
:10C2D8001F4918EE103AB8F1030F49F8013004F17C
:10C2E800040406F104067FF4C1AE03B0BDEC088B6C
:10C2F800BDE8F08FC4190020481B00200000FA4355
:10C3080000000000EC1F002000004842C626002064
:10C3180026260020CC430108241100200000C84232
:10C32800EC210020841F002000007AC300007A431B
:10C3380018220020A81F0020000096C30000964382
:10C3480018FCFFFFC01F0020C81F0020D41F0020BA
:10C35800E01F0020D0110020801F00208C1F00202B
:10C36800044B00221A605A60034B00221A605A607C
:10C37800704700BFEC210020F81F002010B50B4CBF
:10C388000123E3704FF48060022384F82030FDF726
:10C39800FDF9074A074B926B1B685178642212FB20
:10C3A8000133636123880133238010BD7C2600207C
:10C3B800EC21002054260020704708B50B4B0020C4
:10C3C80093F82C10FAF76CFE094B1B68187A0828AA
:10C3D80001BF084B4FF480521A80102208BF5A80C0
:10C3E800A0F109035842584108BD00BFBC00002015
:10C3F8005C23002028220020704770477047FEE722
:10C40800FEE7FEE7704730B50024E3B293420DD251
:10C41800030F092B94BF3033373301F8143001EB85
:10C428004403002500015D700134EEE730BD30B5EE
:10C43800002202F1805303F5B8539B0042F40044F4
:10C448001D6840F60F7144F08004294001322143F1
:10C45800042A1960EDD1024B40F08000186030BD0D
:10C468004C5C00402DE9F347884D894C2B68894E78
:10C478009BB2A380A28831880A40970507D54FF65A
:10C48800FF53854A2B6013780133DBB21370A388FE
:10C498000B40180440F100830023ADF802302B68EC
:10C4A8007B4F9AB21804A28040F1F682BB8803F051
:10C4B8000F03BB71002B40F0C182784A13689BB20E
:10C4C8003B803B8803F030037B803B8803F4405378
:10C4D8003B8011684BF6BF730B4083F4005383F025
:10C4E800200343F4004343F080031360BB88D9065C
:10C4F80021D4116848F60F730B40694913600B6823
:10C508001A7A022A884601D0042A02D1FAF754FD81
:10C518005AE2062A40F06B825A78052A08D11A781E
:10C52800520605D1D878FFF782FFBB681B6A984787
:10C53800E3689B685AE213689BB2ADF80230BDF815
:10C5480002301F0540F1D0811168554F40F68F73B6
:10C558000B40544913600A68534B92B213445B0072
:10C5680088461A683B68187A092817D092B2520090
:10C5780002F1804202F5C042117819705178597061
:10C588009188C8B2090A41EA002159801189C8B2C4
:10C59800090A41EA002199809289DA8001221A72F7
:10C5A800DA8893F80190002A40F0DC801A7812F0BB
:10C5B8007F024AD1B9F1090F0FD1DA78012A00F2C6
:10C5C800B8809978002940F0B4809988002940F013
:10C5D800B0809A72A3685B68A9E0B9F1050F10D121
:10C5E80093F90320002A01DA0823B9E09A78002A8F
:10C5F800FAD19A88002AF7D19B7A002B00F0A28002
:10C60800F2E7B9F1030F0ED1DA78012A40F09180F0
:10C618009A88002A40F08D805A7A42F020025A7295
:10C62800A368DB6983E0B9F1010F40F08280DA7812
:10C63800012A7ED19A88002A7BD15B7A980678D520
:10C64800FAF750FD00287DD073E0012A2ED1B9F108
:10C658000B0F6ED1E26858799269D97890473B6898
:10C668009A7A002A65D0002863D11A79002A60D105
:10C678009B78002B5DD1064B9B68DB689847084B7D
:10C688001B685A79DA72DA781A735BE0445C004006
:10C69800282200206C260020CF260020005C0040C5
:10C6A8005C230020505C004004300020022A40D166
:10C6B800B9F1010FC4D0B9F1030F3AD1587920F07C
:10C6C800800E4FEA8E0202F1804101F5B84110F068
:10C6D800800F096814BF01F0300101F44051BEF128
:10C6E800030F26D8B3F802E0BEF1000F21D101B341
:10C6F8009B7AF3B102F1804202F5B8420106136851
:10C708004BBF23F4E04323F4804323F0400323F09A
:10C7180070034BBF9BB29BB283F0100383F480532A
:10C7280043F4004343F080031360A3689B69984770
:10C7380008E0E36848465B69984703280FD000285B
:10C748007FF452AFD8F80020A14B92B213445B009B
:10C758001A6800221A6030236380062300E0092348
:10C768003A6847E1B9F1060F12D11A78520678D122
:10C778009B78012B02D1E368DB6967E0022B02D1C9
:10C78800E3681B6A62E0032B6BD1E3685B6A5DE0D8
:10C79800B9F1000F38D15988002962D15A6822F4BA
:10C7A8007F42B2F5003F5CD11A7812F07F0204D1C3
:10C7B8009B88002B00F0D58153E0012A08D1E2685C
:10C7C80058799269904700284BD13B689B7A17E0CB
:10C7D800022A46D15A7902F00F010BB29B0003F1ED
:10C7E800804303F5B84312F0800F1B6814BF03F0B1
:10C7F800300303F44053032933D812F0700F30D1BB
:10C80800002B40F0AE812CE0B9F1080F04D11B7861
:10C818005B0600F0A88124E0B9F10A0F21D11A784B
:10C8280002F07F02012A1CD19A7AD2B15988C1B983
:10C838005A6822F47F42B2F5803F12D1E2685879F3
:10C8480092699047002800F090810AE04BB13A685D
:10C858004FF00008A2F8128093614046984740467E
:10C868000BE0E3683A681B6950789847032804D1BD
:10C87800584B1B6809221A72BDE03A68138A4FF6B2
:10C88800FF718B4201D10923B4E0022800D00BB913
:10C898000823AFE092F9001000291FDAD18801912E
:10C8A8000198834202D9019B138210E08B420ED279
:10C8B800E16891F82C00834201D2002105E093FB46
:10C8C800F0F100FB113313B90121434B1970E368F0
:10C8D80093F82C309382FAF76FFB8CE003231372E2
:10C8E8004FF44053238086E0BDF802301BB2002B82
:10C8F800BFF6D5AD116840F68F730B401360354A0B
:10C9080017683B7A022B904671D0042B6FD0032B0B
:10C9180001D0052B66D1BB693A8A8BB9398A0029BF
:10C928003BD04FF4405323802C4B1A68284B92B2CB
:10C9380013445B001A6800221A60302363802CE0DD
:10C94800002AEBD0B7F81490914528BF91461FFAFA
:10C9580089FA504698473B8ACAEB03033B827B8A95
:10C9680053447B821D4B1A681D4B92B213445B00E3
:10C9780009F101021B689BB203F1005303F5405310
:10C9880052105B004FF0000E9645C7D053F82E109A
:10C9980020F81E100EF1010EF6E7BB8A8B42D8F87C
:10C9A800003001D8032201E011B105221A720BE010
:10C9B80006221A72094B1A68054B92B213445B009F
:10C9C8001A68196030236380D8F800301B7A0FE0AA
:10C9D800023000205C230020CE260020505C00405E
:10C9E80004300020072B02D1E368DB68984708234E
:10C9F800D8F800201372FFF7E0FC5E4B1A684BF67C
:10CA0800BF7313402288D704228848BF83F4805319
:10CA18009004628848BF83F40053D106628848BFF7
:10CA280083F01003920648BF83F0200343F40043C9
:10CA380043F080034F4A9BB213602DE09A0002F145
:10CA4800804202F5B842116889B2ADF80210BDF80B
:10CA5800021009B2002909DA106840F68F71014006
:10CA68001160013B444A52F823309847BDF8023020
:10CA78001F067FF514ADA1798B0003F1804303F500
:10CA8800B84348F60F72186802401A603A4B03EB35
:10CA980081039B69984702E5A288338813405905AA
:10CAA80005D54FF6FF332B60344B5B689847A28857
:10CAB80031880A40920444BF4DF6FF732B60A38867
:10CAC8002F4A0B40DB0452D54EF6FF732B60002330
:10CAD8001374137C052B41D8DFE803F0030D1418F9
:10CAE800222D6369264D1BB901F0C6FF062300E01D
:10CAF80005232B743BE001F0BFFF042323740123BB
:10CB0800636134E002236374032328E0637C013B00
:10CB1800DBB26374637C53BB194B04221A7426E09E
:10CB2800184A13689BB243F010031360052323745B
:10CB38000A2363741BE0637C114A013BDBB2637414
:10CB4800637C03F0FF0093B90E490C684FF6EF734E
:10CB580023400B6006231374506108E006232374F6
:10CB680005E0094B73E6094B71E6094B6FE602B025
:10CB7800BDE8F087005C0040D0430108BC000020FD
:10CB880028220020405C0040196B0008D16B000887
:10CB9800AD6B0008022803D0431E58425841704725
:10CBA800064B1B681B7823B1054B1868C0F3C040BF
:10CBB8007047044B1878C0F3800070472C0A002097
:10CBC80004110020CC26002010B50A4C5E2801462E
:10CBD800206805D15D21FEF7BDFA20683E2105E0F9
:10CBE8005D2903D1FEF7B6FA20683D21BDE8104063
:10CBF800FEF7B0BA4022002030B50028104C114A88
:10CC0800B8BF40423C2590FBF2F304FB03006843A5
:10CC18000D4D90FBF2F22D682D7B25B903EB8303B4
:10CC280003EB830301E0C3EB031302EB83030B80E5
:10CC380004FB02024FF47A7392FBF3F24A8030BD90
:10CC4800806967FF80969800F018002010B50446A8
:10CC5800C0B2FFF7B9FFC4F30720BDE81040B3E73F
:10CC6800024B5E211868FEF775BA00BF402200200B
:10CC780038B5064C05465E212068FEF76BFA206839
:10CC88002946BDE83840FEF765BA00BF40220020BB
:10CC9800674B73B51878674DFFF77CFF2B78834295
:10CCA800044620D0C8B1644B1B68E3B193F9000077
:10CCB80002230093614B1B685B78003318BF012384
:10CCC800019304214FF416530022F9F777FB5C4BCC
:10CCD800186040B101232B7005E0594E3068F9F710
:10CCE80052FB34602C70574B574D1878FFF752FFA2
:10CCF8002B788342044618D088B1544B1B68A3B1E3
:10CD08000022012493F9000000944FF49643019205
:10CD18000821F9F753FB4E4B186028B905E04C4E33
:10CD28003068F9F730FB34602C704A4B4A4D18785C
:10CD3800FFF730FF2B78834204462E4642D0002866
:10CD480037D0464B1A68002A3CD0D37992F90000B4
:10CD5800434C002B08BF022302220092002254F801
:10CD6800233001921021F9F729FB3E4B0546186044
:10CD780040B33D4C94F84A30022B0BD094F89620DF
:10CD8800022A01D14C3405E023B1002A04F14C04F5
:10CD980018BF0024354B1C6044B1204600214C22AA
:10CDA80005F08BFC0223256084F84A300123337098
:10CDB80008E02C4E306800F0EBFC3068F9F7E3FA35
:10CDC80034602C702A4B2B4D1878FFF7E3FE2B7834
:10CDD8008342044629D000B3274B1B682BB3274A4C
:10CDE80093F9000012685278002A0CBF0822092221
:10CDF8000323009301924FF4614320210022F9F7A5
:10CE0800DDFA1F4B186080B11E4A012313702B7086
:10CE18001D4B1A681D4B1A6007E0194E3068F9F768
:10CE2800B2FA184B34601C702C7002B070BD00BF91
:10CE3800340A0020BC110020300A0020F01800201D
:10CE480040220020350A00201019002094190020E3
:10CE580084190020400A00209A1900203C0A00206A
:10CE6800B85201089C190020C0230020A0190020F6
:10CE78004C0A0020B0190020480A0020440A00206B
:10CE8800B4190020B819002054260020BC1900202D
:10CE98002DE9F04FC34BDA682DED028B1A61C24AB7
:10CEA8001168D960C1490B6843F020030B60C04B7F
:10CEB8001978012990460CBF002201221A70BD4B37
:10CEC8001A78910789B040F13F83BB490978042952
:10CED80040F23A83B949097801F0040101F0FF00F2
:10CEE80011B922F001021A701B78DB0702D408B1CD
:10CEF800FDF758FBB2490A79531C052293FBF2F25D
:10CF080002EB82029A1AAF4B0A711B7803939200C4
:10CF18000023AD4CDFF8D0C2DFF8DC925CF82310B8
:10CF280091FBF9F504F1080004F1100640F82350CC
:10CF3800A64844F8231000FB051142F2107091FB3B
:10CF4800F0F080B226F813004FF0140E04F1140626
:10CF580004F13C0A0EFB036E5AF823605EF8027077
:10CF68004EF80210F61B314444344AF823100526C3
:10CF780091FBF6F109FB051144F82310039C012CE1
:10CF88004FEA830BE24605D10238B0F5797F98BFA6
:10CF98004BF80C100BB90123BBE7894CD8F80030CB
:10CFA800626D9FED8B7A8B4E8B4D9B1A07EE903AF4
:10CFB800F8EE677AD8F800306365C7EE877A7D4B5C
:10CFC8001B78B7EE008AF4EEC87AF1EE10FA58BF73
:10CFD800F0EE487A13F00103C4ED167A12D005AAD0
:10CFE80000927E4B06AA01920CCB9AE80300FDF74B
:10CFF800D7F96421059A069BB2FBF1F293FBF1F392
:10D00800328000E033802B8094F85C306C48002B31
:10D018003BD0D0ED167A026EDAF80030C8EE276AF7
:10D028009B1A426E022507EE103AB8EEC77ADAF874
:10D03800043027EE267A9B1AFDEEC77AB0F96A20EB
:10D0480017EE901A07EE903A654BB8EEE77AD3EDF3
:10D05800007A67EE277A67EEA67AFDEEE77A17EE92
:10D06800903A02FA83F3B0F9682093FBF5F302FAD9
:10D0780081F29BB292FBF5F292B2A0F86E30A0F862
:10D088006C20A0F86A30A0F86820012384F85C308E
:10D09800544BDAF804101B88DAF80000484D524E59
:10D0A800616603F030032066002B00F04D8205F125
:10D0B8007803009305F17C0301932A6F6B6FFDF7EA
:10D0C8006FF972686B6F9B1A07EE903A444B32689F
:10D0D80093ED007A2B6FF8EEE77A9B1AC5F880304B
:10D0E800384B67EE877A1B78FDEEE77A012BC5EDA2
:10D0F800217A03D0022B00F0E08025E2D5ED297AD1
:10D108003A4BD5ED225A95ED265A95ED166A95EDCE
:10D11800274AD5ED284A36491D68B1EE677ABDEE33
:10D12800C77AFDEEE77A17EE10EA17EE90CA0020EC
:10D13800304A91ED007A52F8207007EE907AF8EEB6
:10D14800E77AA2F1140367EEA57A33F81060FDEED2
:10D15800E77A283217EE903A9B1B9BB222F81030E0
:10D168001BB207EE903AF8EEE77A3B4467EE857A11
:10D178004400FDEEE77ACDED037A07EE903AF8EE3B
:10D18800E77ABDF80C8067EE847AA7EE867AFDEE22
:10D19800C77A17EE902A724532DB6245A8BF62460D
:10D1A8002FE000BF7C01002054260020FC1800203E
:10D1B800621100200019002006190020CC2600204A
:10D1C80040220020380B002048220020806967FF99
:10D1D80000007A447A1900207C190020641100208C
:10D1E8005C000020C4190020081900203C0B002016
:10D1F8006C0B0020C022002080969800DB0FC940ED
:10D20800724607EE902AF8EEE77A5FED046AC1ED00
:10D21800007AFDEEE77A313617EE903A43449AB237
:10D22800AB78D1ED027A07EE103AB8EE477A4B6840
:10D238004F6027EE267AFB1A88EE077AB6B2622E7E
:10D2480006EE903AF8EEE66A37EE067AC6EE866A99
:10D2580086EE077A76EEE76AE7EE267AC1ED047A7B
:10D26800C1ED027A0FD964EEA77ABA4EFDEEE77ADD
:10D2780017EE903AB3F5FA6FA8BF4FF4FA63B342CA
:10D28800B8BF334600E0002313441BB240F6B8325F
:10D298009342A8BF1346B04A9342B8BF1346AF4A59
:10D2A800A352AF4A142303FB002351F8142B1A602E
:10D2B800002840F0498101203AE7AA4BD5F8788048
:10D2C8001F68D4F87C903E89DFEDA78A4FEA58039F
:10D2D8009E4228BF1E46B5F8AC301AB29642C3BF6C
:10D2E800D5ED167A9FEDA17A67EE877AB6B2C1BFFF
:10D2F800FDEEE77A17EE906AF618B6B2C8BFA5F841
:10D30800AC60D4F8B050C5EB09052846FDF78CF899
:10D318000028D8BF404241F293129042CCBF00206F
:10D32800012088B307EE905AB8EEE70A20EE280AE3
:10D33800FCF7B4F907EE908AF8EE677A40F6B8334E
:10D3480020EE270AFDEEC07ACDED037ABDF80C2059
:10D35800A4F8B42012B29A42A8BF1A467E4B9A4249
:10D36800ACBF09EB02034B4448F6A042934203DDED
:10D37800A3F50C43A03B04E0002BBCBF03F50C4312
:10D38800A033C4F8B83001E0C4F8B890D4F8B85065
:10D39800C5F50C53283307EE903AF8EEE77A67EEB6
:10D3A800A88AB0EE680AFCF7D9F98DED070AB0EE45
:10D3B800680AFCF773F9D4ED327AD4ED2F4AD4ED2C
:10D3C800165A94ED304A94ED315A65498DED060AA6
:10D3D800B1EE677ABDEEC77AFDEEE77A0DF1180E69
:10D3E80017EE10AA17EE90BA0020614AFEEC016A07
:10D3F80032F91030DFF88C9107EE903A07EE106A98
:10D40800F8EEE77AB8EEC77A3C32D6EE877A4FEA7A
:10D41800400CFDEEE77ACDED037ABDF90C30B3F59B
:10D428007A7FA8BF4FF47A734B45B8BF4B461FFAB3
:10D4380083F922F810900FFA89F207EE902AF8EE95
:10D44800E77A27EEA47ABDEEC77A8DED037A27EE48
:10D45800847AD1ED007ABDF80C90E7EE257AFDEEDE
:10D46800E77A17EE902A524503DB5A45A8BF5A4679
:10D4780000E0524607EE902AF8EEE77A9FED3D6A03
:10D48800C1ED007ABA7891ED027A06EE902AF8EEAC
:10D49800666A4A684B6066EE866A9A1AC8EE266A19
:10D4A800143106EE102AB8EEC66A76EEA56A86EE44
:10D4B800256AC5EEA66A36EE476AA6EE867A01EDBB
:10D4C800017A01ED037A25EE077ABDEEC77A17EEE9
:10D4D800103ABDEEE77A4B4417EE102A13441BB2FC
:10D4E80040F6B8329342A8BF13461B4A9342B8BFCE
:10D4F80013461A4A2CF802301F4A142303FB002350
:10D50800C3ED007A08B901206FE73B7923B16423A2
:10D5180095FBF3F5194B1D803B8898450DD9D4F838
:10D52800B030E06FC01AFCF77FFF80EAE072A2EB30
:10D53800E07242F210739A4206DD114B01221A7012
:10D548000E4BB4F8CC201A8009B0BDEC028BBDE8B4
:10D55800F08F00BF30F8FFFF48F4FFFFC00B00203A
:10D56800940B00203C0B0020D30237390000C8423E
:10D57800AC220020DB0FC9406C0B0020EC1000200F
:10D58800380B002018FCFFFF07B5064B0093064B2D
:10D5980001930649064A074B0748FBF7EEFF03B01D
:10D5A8005DF804FBDA530108AF5301087F610108F5
:10D5B80089610108CE5301085C61010808B5037848
:10D5C80033B90C4B0C481978BDE80840FBF7D5BFB8
:10D5D80005F00EF902280CD8064B1870074B0C22E0
:10D5E80002FB0030064B06301860FCF7ABF9054823
:10D5F800E5E708BD1023002090610108B818002055
:10D608005C110020A057010808B503783BB90B4B03
:10D618000B4893F8E416BDE80840FBF7AEBF05F0E9
:10D62800E7F8022808D8054B83F8E406FCF7F0F879
:10D63800FCF7ACF90348E8E708BD00BFD8110020A3
:10D6480094610108A057010838B5037803BB214B42
:10D658001B6801330F2B07D81F490C2202FB03124A
:10D668001C4695682DBB00E01C4601340F2C01DDDB
:10D67800002400E005D818490C2202FB0412956822
:10D68800BDB99C42F1D11548BDE83840FBF775BFDC
:10D6980005F0AEF80F28044605D80F4A0C2303FB03
:10D6A80000239D682DB921460D48BDE83840FBF799
:10D6B80064BF084B1C60F9F791F921462A460948CE
:10D6C800FBF75BFF0C235C43034B185DBDE8384058
:10D6D800F9F79AB9600000200C440108A16101081B
:10D6E800B7610108CF61010873B5037813B9F8F77A
:10D6F800EFFC3FE001AA204905F0DBF800240246D0
:10D70800264625469AB134B1012C08D1104605F0B9
:10D718006FF8064603E0104605F06AF8054601AAC8
:10D728000020154905F0C5F801340246EAE70B2D3B
:10D7380003D9124812490C230CE0022C11D1A6F58A
:10D748007A73B3F57A7F08D90C480E494FF47A7288
:10D758004FF4FA63FBF711FF0CE00B4B03EB4503A7
:10D768005E80094B094803EB45032946B3F90220BB
:10D77800FBF703FF02B070BDFE5C0108F358010817
:10D7880012590108B75E010810230020E66101085C
:10D7980038B50D4C23688342054606D1F8F7F3FDEA
:10D7A800204600214C2204F088FFE36CAB4209D1EB
:10D7B8002846F8F7E8FD054800214C22BDE8384026
:10D7C80004F07BBF38BD00BFC02300200C2400201C
:10D7D800034B1A68D379591C1344D171187A7047CE
:10D7E800A419002010B5FFF7F3FF84B2FFF7F0FF8C
:10D7F80004EB002080B210BD10B5FFF7F3FF04461C
:10D80800FFF7F0FF04EB004010BD064B10B50446CF
:10D8180021461868FDF79EFC034B1B689879604009
:10D82800987110BDA8190020A419002038B5044625
:10D8380024200D46FFF7E9FF4D20FFF7E6FF002CF7
:10D84800084C14BF21203E20FFF7DFFF2368002289
:10D8580028469A71FFF7D9FF236893F84900BDE875
:10D868003840D2E7A419002001460020DEE710B5B1
:10D878000446C0B2FFF7C9FF200ABDE81040C4E75C
:10D8880010B5044680B2FFF7F2FF200CBDE8104047
:10D89800EDE737B582888368044610060D4641BF18
:10D8A8002B4991F8E4164FF4CC7000FB0133D105F5
:10D8B80044BF2849097802F03F0244BF01EB410107
:10D8C80003EB8103042A12D006D8012A0DD0022ABC
:10D8D80032D193F9001030E0102A0AD0202A0AD059
:10D8E800082A29D1B3F9001027E0197825E019880A
:10D8F80023E0196821E093ED000A6846FBF7D2FCA3
:10D9080001461548FBF739FE05B3D4ED037A68469E
:10D91800B8EEE70AFBF7C6FC01461048FBF72DFEF8
:10D9280094ED040A6846B8EEC00AFBF7BBFC014652
:10D938000A48FBF722FE09E000210948FBF71DFE13
:10D9480025B10848E1682269FBF717FE03B030BD2E
:10D95800D811002010230020615A01085A5A0108E2
:10D96800F9610108F5610108024B0146D869FDF724
:10D97800F1BB00BF1023002010B5441E14F8011F8E
:10D9880021B1034BD869FDF7E5FBF7E710BD00BFF0
:10D9980010230020F7B52B492B4B08782B4D1C681A
:10D9A8002B4B05EB80001A882A4BD0F8C0101B7847
:10D9B800294800914FF47A71B4FBF1F1FBF7DDFDD2
:10D9C80026484821FBF7D9FD254B1F680026F3B2EE
:10D9D80005EB8302D2F8D010E9B101249C403C4207
:10D9E80017D0220715D01F4AD25C0B2000FB032357
:10D9F800164A1D4802EB8303D3F8F020FBF7BDFD60
:10DA0800022C06D1194B93F8281011B11848FBF7CE
:10DA1800B4FD0136DBE71748FFF7AEFF164B174892
:10DA28001A68174B9A420CBF164B174B1A88174B9C
:10DA3800198892B24FF4E26303B0BDE8F040FBF7F7
:10DA48009CBD00BF4C190020542600200C4401083E
:10DA5800EC180020EC000020FC6101083F6201087E
:10DA6800FC180020F40000204F6201081023002059
:10DA7800576201089F620108FC1000205B620108E0
:10DA8800005400400011002002110020F81000206E
:10DA98002DE9F0410024804625460F4EA7594146FE
:10DAA800384604F08DFE58B139460C48FBF765FD41
:10DAB80030190021FFF7EDFE0948FFF75DFF01353A
:10DAC800143440F644439C42E7D11DB90548BDE8EB
:10DAD800F04151E7BDE8F081AC450108E75A01087B
:10DAE8009F620108895A01082DE9F04F2DED028B3C
:10DAF80083B0054604F025FE064620B1012818D15A
:10DB08002B782A2B15D15C48FFF736FF00245B4D94
:10DB18005B486159FBF731FD28193146FFF7B9FE1B
:10DB28005848FFF729FF143440F644439C42EED18D
:10DB38009CE028463D2104F0F6FD002800F08F8087
:10DB48000346994613F8012D202AFAD0441C204692
:10DB580004F04EFE80462046FBF71AFBC5EB090988
:10DB6800B0EE408A0026DFF834A1142202FB06F446
:10DB78000AF5D07B54F80B70384604F0E2FD0346F2
:10DB88001A4628463946019304F0E4FD019B002813
:10DB98005BD15FFA89F29A4257D10AEB0402D2EDBF
:10DBA8006B7AF8EEE77A0BEB0405B4EEE78AF1EE50
:10DBB80010FA48DBD2ED6C7AF8EEE77AB4EEE78A31
:10DBC800F1EE10FA3FD8B2F8A431D2F8A82113F038
:10DBD800200F08BF08EE108A1C0641BF2A4991F899
:10DBE800E4164FF4CC7404FB0122D90544BF27493D
:10DBF800097803F03F0344BF01EB410102EB8102C6
:10DC0800042B18EE100A0BD004D8013B012B0ED8B8
:10DC180010700CE0102B05D0202B06D0082B06D155
:10DC2800108004E082ED008A01E082ED008A394626
:10DC38001748FBF7A2FC2846002103B0BDEC028B75
:10DC4800BDE8F04F25E6134803E001369D2E8AD142
:10DC5800114803B0BDEC028BBDE8F04F8CE62846B6
:10DC680003B0BDEC028BBDE8F04F11E703B0BDEC8B
:10DC7800028BBDE8F08F00BF8D620108AC4501083A
:10DC8800E75A01089F620108D811002010230020DC
:10DC9800A2620108AD620108895A01080C44010812
:10DCA80070B50546284604F04CFD064658B9194B90
:10DCB80019485A79194B03EB8203BDE87040D3F831
:10DCC800E01DFBF75ABC28461549324604F042FDD0
:10DCD80060B91448144CFFF74FFE54F8041F19B1EB
:10DCE8001248FBF74AFCF8E7114805E00024114BFD
:10DCF80053F8241019B91048BDE870403CE628468E
:10DD0800324604F027FD01340028F0D1014B0B4DB9
:10DD18005C71C7E7D8110020CD6201080C440108E6
:10DD2800785A0108D9620108EC510108745A0108AF
:10DD38009F620108F0510108895A0108A05701089B
:10DD480008B50748FFF718FE064BD869F8F710FB27
:10DD5800FDF76CFBFBF732FD034B044ADA6008BDA4
:10DD6800EC6201081023002000ED00E00400FA0531
:10DD780008B50548FFF700FE00F036F8FBF748FD48
:10DD8800BDE80840DCE700BFF862010808B50448B0
:10DD9800FFF7F2FDFBF73CFDBDE80840D0E700BF08
:10DDA8000E6301080E4B1A786C2A16D15A88B2F500
:10DDB800E26F12D11A79BE2A0FD193F80D27EF2AF4
:10DDC8004FF000000BD113F8012B5040054A934245
:10DDD800F9D1B0FA80F040097047002070477047C9
:10DDE80000F8030810FF03082DE9F04F2DED028B12
:10DDF800EB4D00214FF4E26285B0284604F05DFC4B
:10DE0800E84B05F507721A60E74A00231370E74AE2
:10DE180005F2E66111606C222A7003226A714FF4E0
:10DE28008072AA604FF41672A5F86421FA22A5F848
:10DE380066214FF4FA722021A5F86C21012285F899
:10DE48005E2185F8681185F869216E2185F86A21B7
:10DE580085F87C2185F88421052285F87A1185F8D2
:10DE68001B220A2140F2DC5285F87B11A5F8962185
:10DE78002B2140F24C4285F87D11A5F898212121EB
:10DE880040F26C7285F87E11A5F89A21232140F2A0
:10DE9800753285F87F11A5F89C214FF4C87140F6BA
:10DEA8004302A5F89E21A5F880112A462C46032B8B
:10DEB800CCBF0121002103F1010382F8A01114BF96
:10DEC8001E217521122B82F8A11102F10202EED156
:10DED80040F27E414FF4FA63A4F8401140F23A71DF
:10DEE800A4F8C631A4F8CA31A4F8CE31A4F8D231C6
:10DEF800A4F84211052340F27E5184F8E031A4F8D9
:10DF08004811C82340F2EA5101274FF47A794FF0BB
:10DF1800320A40F2DC50A4F8E431A4F84A114FF474
:10DF2800C87340F2B4511E224FF0190BA4F8E8311F
:10DF3800A4F84601A4F84C11A4F84EA1A4F8C49181
:10DF4800A4F8C891A4F8CC91A4F8D09184F8E2710F
:10DF580084F8E37184F8E671A4F8449184F8932175
:10DF6800019284F8E1B10390A4F85031A4F852A1C9
:10DF780084F8DF7184F8EC7184F8EF7100F082FCAA
:10DF88008849019A0B68029100262673DA721A737F
:10DF98005522DA700F225A7122229A710E221A74AF
:10DFA80035229A7621225A745322DA764FF0780C69
:10DFB8005A224FF028084FF02D0E83F807B01A7236
:10DFC8004FF0640B0A2283F80AC0DFF800C283F816
:10DFD8000DE083F804A09A74019283F814E01E708F
:10DFE80083F8018083F8158083F8028083F816800F
:10DFF800DE759E731E76DE735E7683F81CB083F83A
:10E0080009809F77C3F838C0C3F83CC0DFF8C0C1A7
:10E01800C3F828C0DFED667ADFF8B8C1C3F834C0AA
:10E028004FF4FA7EDFF8B0C19FED628AA3F84EE0A4
:10E03800C3ED0B7AC3ED0C7AC3F848C04FF0140E49
:10E04800B7EE087AF1EE047A039883F850E04FF0BF
:10E058004B0C83F84CC083ED087A83ED097A83ED85
:10E06800108AC3ED117A4FF0460CA4F8F00604208C
:10E0780084F8E7C684F8E8A684F8EEE684F8E6B6FD
:10E0880084F8E96684F8ED6684F8EA6684F8EB6655
:10E0980084F8EC6683F85C00152083F8680046482D
:10E0A800A3F85860A3F85A60A3F85660C3ED187A2D
:10E0B80083F8648083F86580D866404818674048CC
:10E0C800586783F878703F4800F022FC0299019A5B
:10E0D800D1F800A04FF44873AAF81631C8238AF87B
:10E0E80011618AF812618AF813818AF814718AF822
:10E0F800186184F8D62184F8D731A4F8D89184F827
:10E10800DA61A4F8DCB152460E2303FB06A36FF0D4
:10E11800170183F81911032183F81A116FF02F01E1
:10E1280083F81B11072183F81C116FF0230183F872
:10E138001D11052183F81E1101365A2182F820117C
:10E1480082F821116423FF21082E82F81F3182F8FA
:10E15800221102F10E02D7D100228AF88921C822A1
:10E16800AAF88A21AAF8903114224FF496738AF8F3
:10E178008C21AAF892311E2228238AF88D21AAF828
:10E1880094310122104B8AF88E2118EE102A45F896
:10E19800102F9D42F9D1024C0023012551461DE064
:10E1A800D81100203C110020102300205C11002011
:10E1B800CDCCCC3E000000009A99193FF6287C3F50
:10E1C8003D0A773FAA6D0108981200208FC2F53CDE
:10E1D800000060406666663F0000404004F56D70D0
:10E1E8004FF4CC7284F80C3784F80A5784F80B572C
:10E1F80004F058FA04F24C5051464FF4CC7204F033
:10E2080051FA0F4B1B681A68C4F8F2265A68C4F80A
:10E21800F6269A68C4F8FA261A68C4F8FE265A68D8
:10E22800C4F802279A68C4F80627022384F8085419
:10E2380084F8A03505B0BDEC028BBDE8F08F00BFB7
:10E248005C1100201549D1F8883043F47003C1F8F7
:10E258008830134B1A6842F001021A605868114A54
:10E2680002405A601A6822F0847222F480321A60DE
:10E278001A6822F480221A605A6822F4FE025A6050
:10E28800DA6A22F00F02DA62186B074A02401A6350
:10E2980000229A604FF000638B60704700ED00E049
:10E2A800001002400CC07FF8CCFC00FF38B5094BC9
:10E2B80093F80C5765B9084C2068F8F764F8074BD1
:10E2C80025601B78022B03D1BDE8384000F099BACD
:10E2D80038BD00BFD8110020902400208F240020D2
:10E2E800044B93F80C371BB9034B1868FCF726BF8F
:10E2F80000207047D81100209024002038B505462A
:10E308000446204614F8011B21B1034B1868FCF79A
:10E3180021FFF6E7401B38BD902400200FB407B555
:10E3280004AB064953F8042B01930020FBF738F897
:10E3380003B05DF804EB04B0704700BFB3E4000815
:10E34800024B01461868FCF705BF00BF9024002067
:10E35800F8B5011F06460023083051F8042F02F1D2
:10E3680020043F2C3AD802F108040F2C06D80232B8
:10E37800032A04D9002B08BF012300E002238142AD
:10E38800EBD1012B30680ED0022B1AD0736803F042
:10E3980003039B0000F0030043EA0010B36803F096
:10E3A8000303184317E000F00F0040F04000FFF7A8
:10E3B800C7FFB068736800F00F0040EA0310C0B2EE
:10E3C80009E000F03F0040F08000FFF7B9FF307926
:10E3D800FFF7B6FF307ABDE8F840B1E706F10C0761
:10E3E80034463A46002552F8043D03F18001FF29DE
:10E3F8004FEA850510D903F50041B1F5803F02D2F7
:10E4080045F0010508E003F50003B3F1807F34BF50
:10E4180045F0020545F00305B242E4D165F03F003E
:10E42800C0B2FFF78DFF05F00303022B207807D059
:10E43800032B0CD0012B13D1FFF782FF60780FE07C
:10E44800FFF77EFF6078FFF77BFFA07808E0FFF713
:10E4580077FF6078FFF774FFA078FFF771FFE07827
:10E468000434FFF76DFFBC424FEAA505DBD1F8BDC8
:10E4780010B50446C0B2FFF763FFC4F30720BDE838
:10E4880010405DE710B504467F2C06D964F07F0084
:10E49800C0B2FFF755FFE409F6E7E0B2BDE8104067
:10E4A8004EE7430083EAE070ECE7084648E700BF20
:10E4B800012380F8453070472DE9F04390F8441067
:10E4C800002380F84430002953D02E4C2268002ABB
:10E4D80052D02268052A52D12B4C20290D4628BF3C
:10E4E80020256E1C27687610DFF8A8E0DEF80030DB
:10E4F8009BBBDFF8A4C000F13203324613F8019C3D
:10E5080013F8028C013A48EA09282CF8048C03F124
:10E5180002030CF1040CF1D11C4B1A681C4B92B28B
:10E5280013445B002A46D3F800C01D60DEF80030B3
:10E538002B44CEF80030DFF864E0DEF8003023F436
:10E54800E04323F040039BB283F0300343F40043DD
:10E5580043F08003CEF8003000E000228A4203D066
:10E568002368DB1B312BBFD9531A58425841BDE8E9
:10E57800F0830120BDE8F0831046BDE8F08318461B
:10E58800BDE8F083B426002054260020505C0040EB
:10E598000A3000205423002084610040045C0040BD
:10E5A800002280F8452087E790F84420531C024455
:10E5B800DBB280F8443082F8301090F845200AB178
:10E5C800132B00D978E77047014B5868C0B27047E1
:10E5D80054230020012070477047704720B9034B2F
:10E5E8009B6808221A82704701487047542300200C
:10E5F8006400002020B9034B9B6808221A827047E8
:10E6080001487047542300206400002021B90128E4
:10E618008CBF0220002070470220704710B5094BBC
:10E628009A68D378042B0BD8074C518ADB00234413
:10E6380018B99B895B1A138210BD9B68581810BDC6
:10E64800002010BD5423002064000020054B996869
:10E65800054B4A8A18B99B8D9B1A0B827047986A9A
:10E66800104470475423002064000020054B99682B
:10E67800054B4A8A18B99B8E9B1A0B827047186BF8
:10E68800104470475423002064000020074B9B6807
:10E698001B7803F07F03212B06D100F0DF0002284E
:10E6A80014BF022000207047022070475423002026
:10E6B800212810B508D1114B9B681B7803F07F0304
:10E6C800212B10D0022010BD2028FBD10B4B0C4A67
:10E6D8009B6810701B7803F07F03212B094B18BF30
:10E6E80000230BB9EEE7084B044A926800249361B3
:10E6F800548220469847204610BD00BF542300206E
:10E70800D0260020E5E50008FDE500087047034B2A
:10E718001A78202A04BF00221A707047D0260020D9
:10E72800014B04221A607047B4260020034B9B7DDE
:10E7380013B1034B05221A60704700BF5423002011
:10E74800B4260020F7B51E4B5A681D460AB95C6806
:10E7580000E0012493F828000021CAB2A24201F186
:10E76800010108D202AE2F1816443A4492F8292023
:10E7780006F8042CF1E75A68121B5A6093F828200F
:10E788005D68224483F82820A5B903204021F8F7C2
:10E7980087FC0C4A136823F4804323F070039BB270
:10E7A80083F4405343F4004343F080031360044B65
:10E7B80083F82850002CC6D09DF8040003B0F0BDA3
:10E7C800542300200C5C004010B50446B0F900004A
:10E7D800FFF767FEB4F90200FFF763FEB4F904001F
:10E7E800BDE81040FFF75DBE10B504460068FFF7AE
:10E7F80058FE6068FFF755FEA068BDE81040FFF7B7
:10E8080050BE2DE9F74F0120F8F700F8002488B32F
:10E81800012C2FD8194E4FF04C0909FB04FA06EBCE
:10E828000A0808F1B407BD7815B10134E4B2EEE77F
:10E8380090F9003090F804E01846114B03228DE857
:10E84800240001212A4653F82E30F7F7B7FD8346F6
:10E8580060B106F16C00504429464A4603F02DFF8A
:10E8680001231C44C8F86CB0BB70E4B20120F7F770
:10E87800B1FFCCE703B0BDE8F08F00BF5423002000
:10E88800B852010810B5184C002120461A2203F08E
:10E8980014FFA4F5F970142380F8F431052300223D
:10E8A800042180F8F83180F8FA3180F8003280F8D5
:10E8B800023280F8083280F80A325223012480F8A4
:10E8C800F91180F8FB2180F8011280F8032280F802
:10E8D800091280F80B2280F8F23180F8FC2180F8C8
:10E8E8000442A0F8F64110BDCA13002010B5F8F78D
:10E8F80003FD4FF43024012806D11CB1F8F7FCFCC5
:10E90800013CF8E7052010BD002C08BF052010BD0C
:10E9180070B50646441E14F8011F89B1094D2846F2
:10E9280003F001FF0028F6D005F1080398423FBF25
:10E93800054B401BC018A31B38BF80F88831EAE795
:10E9480070BD00BFC56D0108D8110020031EB8BFF7
:10E958002D2210B5B8BF58420C46B8BF01F8012B9C
:10E968000A22FAF709FD00230370204610BD07B5F7
:10E978001C4B03F58472C3F804211B4A92F89021BA
:10E988005AB1012A14D1032183F80A11072183F807
:10E998000C2183F80B110C2208E0022183F80A11DC
:10E9A800032183F80C2183F80B11072283F808212F
:10E9B8000E4B0F4A9A634020F7F728FF70B10122E7
:10E9C800002390F9000040218DE80C00094A4FF41B
:10E9D800E133F7F7F3FC003018BF012003B05DF80E
:10E9E80004FB00BF54230020D8110020640000203D
:10E9F800AD6C00082D6E000801200021FEF716BF3F
:10EA0800F0B51C4A92F80D31D2F8105192F81471F1
:10EA180092F8206192F82CE1022B0ED805EBC30482
:10EA2800591CA31CC9B206D02346A48814F0010FB0
:10EA380001D0204205D10B46EEE782F80D310020C7
:10EA4800F0BD93F902307CB29C4201D1002307E06B
:10EA580074B29C420CD04FFA8EF49C42EBD1022344
:10EA680082F80D110C2101FB0322D2F81801F0BD28
:10EA78000123F5E7542300200A4B10B519684FF617
:10EA8800FB720A401A60084A927D1C46074B0AB17D
:10EA9800052200E001221A60FFF7D4FB4FF4364349
:10EAA800236010BD405C004054230020B4260020A1
:10EAB8002DE9F04FAD490B7813F0010F85B003F045
:10EAC800040200F04581002A40F07281A8480768D6
:10EAD80017F0806740F06C81980700F1398143F0A6
:10EAE80004030B70A34BA44C1B882380A34B1A6808
:10EAF80012F4002F984600F00C81A14B80201F7063
:10EB0800FFF77EFF08B1FEF743FEA678012E40F01E
:10EB180000819C4D95F80A2722B195F80B370BB167
:10EB28009A4203D3012385F80A370FE018461146A5
:10EB380030B191FBF0FE00FB1E1E01467046F7E760
:10EB480092FBF1F285F80A2793FBF1F385F80B376E
:10EB580095F80C371BB18B4B002283F80C278A4B96
:10EB680095F80CA71B6841F6690203EBC3039342AF
:10EB780084BF40F2E242B3FBF2F3844A8CBFDBB2BB
:10EB880004231370BAF1000F1FD18020F7F73EFE5F
:10EB98008146D0B18021F7F713FE99F806207C4B07
:10EBA800E07053F8223099F90000DFF8CC91B3F502
:10EBB800613F0CBF0222002202218DE8060080215D
:10EBC8005246F7F7FBFB606008B90023A0E0514606
:10EBD80009F10800142203F070FD09F12803C9F8AF
:10EBE8001C3009F19403C9F8203009F58073C9F87D
:10EBF8002430684BD8F800101B88A9F86C3195F8B8
:10EC08009231654895F884910390002B6B79A3F1B4
:10EC1800190BC1F3C03C18BF4FF0010CDBF1000E1B
:10EC28004EEB0B0E95F80AB7012B95F80B370568D4
:10EC380008BF4FF0010E9B45584B1B780293C1F358
:10EC4800400A28BF4FF0000B01F4006138BF4FF0B5
:10EC5800010B721ED2B2531E132B35D8DFE803F016
:10EC68000C0C0C0C0C0C0C0C0A37377F2737811254
:10EC780012123137734675E0029B9342B4BF0023EA
:10EC8800012320E02B78022B0BD105EB820353EDF7
:10EC9800027AF5EE407AF1EE10FA14BF0123002350
:10ECA80011E0AB185B79003318BF01230BE021B1E9
:10ECB80009F1FF304342434100E00B4603F00103F2
:10ECC80050E05B464EE013B1012393401F43142EDE
:10ECD80002D80136F6B2BCE7039BC4F87071186815
:10ECE80019217930F7F724FE0023C4F87831A4F805
:10ECF8007C31A4F87E31C4F88831294BD4F88421BA
:10ED08001B68C4F88C3184F87401C4F8802102238C
:10ED1800A370234B1B4A1B6892F8E0214FF47A71C9
:10ED280001FB02331F4A1360D8F800301A0609D5D0
:10ED38001D4B1B789B0705D51C4B1B78042B01D951
:10ED4800062000E0052005B0BDE8F04FF7F75CBEEF
:10ED580072BB012005B0BDE8F04FF7F779BE534606
:10ED680000E06346002BAFD1B3E700BFCC260020FC
:10ED780004110020CC1100208C2400203026002013
:10ED880061240020D8110020E8210020F80000208C
:10ED9800B8520108481C00203C1100201720002010
:10EDA80054260020EC0A0020001900200619002033
:10EDB80005B0BDE8F08F10B5154A1378590725D569
:10EDC80023F004031370134B1B681B0319D5124C53
:10EDD800A378A3F10802012A0BD8FF200021F9F734
:10EDE8004BFD0E4B1B68C4F88C31FFF779FA0A23E8
:10EDF80006E0012B05D90A2B03D0FFF757FA0123A8
:10EE0800A3700420BDE81040F7F7FEBD10BD00BF99
:10EE1800CC260020302600208C24002054260020F8
:10EE28000C4B0D49DA684378D243C2F30222C2F18F
:10EE38000402934002781B010A44DBB282F80033D3
:10EE480003780122580903F01F0302FA03F341F87B
:10EE58002030704700ED00E000E100E073B50546A2
:10EE6800002100680122FBF75FFC2A6813889BB227
:10EE780043F001031380EB7A8DF804300124002657
:10EE880001A88DF805408DF806608DF80740FFF75A
:10EE9800C7FFEB7A1B2B0BD1192301A88DF804307F
:10EEA8008DF805408DF806608DF80740FFF7B8FF2C
:10EEB80002B070BDF0B5BE4C23782DED028B013B3E
:10EEC800012B85B000F26F816578854240F06B8137
:10EED800A378022B00F06781B64B5B5DE370237962
:10EEE8006D00F2EE048A1BB16319B3F9063009E02C
:10EEF8006319D4ED037AB3F90630F1EE677AC4EDFD
:10EF0800037A5B4208EE103A2369A94EB8EEC88A24
:10EF18001A0388EE288A35D5D6ED037AFDEEE77A0E
:10EF280028EE280A17EE903AD6ED057A8DF80A30C1
:10EF3800FDEEE77A17EE903A8DF80B3003F012FEEB
:10EF4800FCEEC07A96ED060A17EE903A20EE280AF3
:10EF5800ADF8083003F006FEFCEEC07A96ED070A1D
:10EF680017EE903A20EE280AADF80C3003F0FAFDBF
:10EF7800FCEEC07A0C2017EE903A02A9ADF80E30DC
:10EF8800F9F77AFCD4ED077A894BF5EE407AF1EE81
:10EF980010FA60D1D3ED067AB4EEE78AF1EE10FAF2
:10EFA80004DDDA6883ED068A5A61E8E0F5EEC07A96
:10EFB800F1EE10FA40F3E38093F8202042B1022AE0
:10EFC80000F2DD805A6B83ED078AFA329A63D6E045
:10EFD800D3ED037A38EE678AF7EE007AB4EEE78A63
:10EFE800F1EE10FAACBF01210021D3ED0A7A69B124
:10EFF8009FED717A27EE877ADFED707AB4EEE77AC3
:10F00800F1EE10FA58BFF0EE477A03E09FED6C7A04
:10F0180067EE877AC3ED0A7A2369654A1B0311D51F
:10F028008DF80810D378116B0B440B205A788DF8A3
:10F038000920DA7A8DF80A205B7D8DF80B3002A959
:10F04800F9F71AFC0123226B84F82030E378134483
:10F058000022DA7291E0B4EEE78AF1EE10FA48BFC6
:10F0680083ED078AA16B636B94ED067AD4ED076A8A
:10F07800591AC943C90F77EE667A59B9B7EE006ACB
:10F08800F4EEC67AF1EE10FA79DDB4EEE68AF1EE26
:10F0980010FA74DDD4ED056A454BB4EEE67AF1EE6C
:10F0A80010FACCBF0126002666B1D3ED097A9FED90
:10F0B800427A67EE877A9FED427AC3ED097AD3EDFB
:10F0C8000B7A0AE0B0EE007AF4EEC77AF1EE10FAA5
:10F0D80008DDD3ED0B7A9FED387A67EE877AC3EDBA
:10F0E8000B7A07E0D3ED097A9FED357A67EE877AD8
:10F0F800C3ED097AD4ED097A206BE27867EEA87A35
:10F108001044FCEEE77ACDED017A9DF804304370A7
:10F11800D4ED0B7A2769FCEEE77A3F03CDED017A4F
:10F128009DF8042042750ED546EA41018DF8081075
:10F138008DF80930C37A8DF80A300B2002A98DF8B2
:10F148000B20F9F799FB94F82020194B022A11D1CA
:10F15800D3ED0A7A9FED1B7A196B67EE877A002246
:10F1680083F82020FCEEE77ADA7817EE903A0A4422
:10F17800D37202E0022283F82020FBF77FFA22797B
:10F188000B4B0AB1104A00E0104ADA602544D4ED6E
:10F19800037AB5F9063000EE103AB8EEC00A80EEF0
:10F1A800280A37EEC00A05B0BDEC028BF0BD00BFDF
:10F1B8002026002078530108EC51783F6F12833ADB
:10F1C8000AD7833F00007A440000A0410000A0C194
:10F1D8002B4BF0B52B4D1E6805F110002F78F31955
:10F1E8002C46597801F00401013501F0FF0219B1EC
:10F1F8008542F3D10020F0BD224D631B022B0ADDAE
:10F208001AB102EB82025200D2B215F8013B303B30
:10F218001A44D2B2F1E70021AC420AD919B101EB84
:10F2280081014900C9B215F8013B303B1944C9B204
:10F23800F2E72E2F16D10134042000232578771900
:10F2480003EB83037F785B007F079BB244BF303DAD
:10F258005B1900F1FF3044BF01349BB210F0FF008E
:10F26800ECD100E0002308484143642000FB03136D
:10F278000620B3FBF0F3054800FB0230F0BD00BFE9
:10F28800FC0000205C26002040420F008096980079
:10F2980030B500231A4610498C1894F83C40BCB18C
:10F2A8002E2C06D1013298B18C180444002584F81C
:10F2B8003C5011440A2491F83C106343A1F13004F6
:10F2C800092C9CBF303B5B180E2A03D80132E2E7B9
:10F2D800184630BD002030BD202600200D4B0E49B9
:10F2E8001A680E4B92B213445B000D4A1B68C3F3B5
:10F2F800090310B5136013689BB201335B10002239
:10F308009A4206D0074851F8044B20F812400132BF
:10F31800F6E710BD505C0040206200401E3000201F
:10F32800582300207D230020014B00221A607047DB
:10F33800542300202DE9F843664B674E1B68DFF81D
:10F34800B881664A00254FF0C0099D7283F809907C
:10F35800DD723560D8F8003023F4EC4323F07003F5
:10F3680043F400739BB2C8F80030D8F8003023F497
:10F37800E04323F040039BB248F2800483F010037B
:10F388002343C8F80030336812FA83F35B00402740
:10F398001A681F6033689BB203F1005303F54053AA
:10F3A8005B0028461A6880221A60D8F8003023F4D7
:10F3B800F8731B051B0D2343C8F80030484B93F81E
:10F3C8002C10F7F76DFED8F80030464A464923F46A
:10F3D800804323F070039BB283F440532343C8F85F
:10F3E8000030136823F4EC4323F070039BB21360DE
:10F3F800336811FA83F35B0003201968C3F800909F
:10F4080013683A4923F4E04323F040039BB283F0A6
:10F41800200323431360136823F4804323F070030D
:10F4280023439BB21360536823F4EC4323F0700327
:10F4380043F4C0639BB25360336811FA83F35B00F3
:10F4480019684FF480711960536823F4804323F0DE
:10F45800700323439BB25360536823F4E04323F0C3
:10F4680040039BB283F0200323435360D8F80C3049
:10F478001F4A23F4EC4323F070039BB2C8F80C3006
:10F48800336812FA83F35B0039461A684FF48872BE
:10F498001A60F7F705FED8F80C3023F4804323F000
:10F4A80070039BB283F440532343C8F80C30D8F858
:10F4B8000C3023F4E04323F040031C43A4B2C8F803
:10F4C8000C402846FCF7B3FF0A4B01221A60BDE83E
:10F4D800F88300BF5C230020505C0040043000200B
:10F4E800BC000020045C00400830002010300020E0
:10F4F8001C300020B4260020005C0040134A144B46
:10F5080050681B68181810B5146808D011490822EB
:10F51800FCF779FF204610490422FCF774FF0F4BD3
:10F528001A68002393720E4A012111600D49136075
:10F538004FF4E0500B6010600B480B604FF43641FD
:10F5480001801160094A136010BD00BFB0F7FF1FAA
:10F55800ACF7FF1FA2000020B20000205C230020AF
:10F56800405C0040445C00406C260020B42600202B
:10F57800024B4FF480221A60704700BF1404014008
:10F58800014B33F8110070476C1B002000207047B6
:10F59800104B1B6803EB4002117E11B1022910D0F9
:10F5A8000BE0022805D9032807D10B4A1268D204B8
:10F5B80001D5D8897047988A7047084B33F81000EE
:10F5C8007047507E00EB800000EB800000F2EE20D8
:10F5D80080B270477026002030260020481B00208B
:10F5E80008B5FBF765FD054B02221A72044A5860FC
:10F5F80012685A61012283F82D2008BD7026002068
:10F608005426002008B5FBF753FD064B02221A7258
:10F618005A6900F5B71000F5587002F2DC525860CC
:10F628005A6108BD70260020044B1B6842F2010293
:10F638001A420CBF01200020704700BF302600206E
:10F64800104B93F83020012A10B51C460ED008D371
:10F65800022A0FD10C4A938A9BB283F48053938277
:10F6680008E0094B4FF480529A6103E0064B4FF4CF
:10F6780080521A85FBF71CFD00F5F42000F5907008
:10F68800606310BD702600200004004808B5044BD4
:10F698001B7803F00503052B01D1FBF7C7FEFEE736
:10F6A800A8260020D0400B1C1141203A03D49C46C8
:10F6B800134118436346524293401843704700BFB2
:10F6C80081F0004102E000BF83F0004330B54FEA0B
:10F6D80041044FEA430594EA050F08BF90EA020F78
:10F6E8001FBF54EA000C55EA020C7FEA645C7FEA0B
:10F6F800655C00F0E2804FEA5454D4EB5555B8BF2E
:10F708006D420CDD2C4480EA020281EA030382EA9E
:10F71800000083EA010180EA020281EA0303362D30
:10F7280088BF30BD11F0004F4FEA01314FF4801C03
:10F738004CEA113102D0404261EB410113F0004F15
:10F748004FEA03334CEA133302D0524263EB4303CC
:10F7580094EA050F00F0A780A4F10104D5F1200E6A
:10F768000DDB02FA0EFC22FA05F2801841F10001C5
:10F7780003FA0EF2801843FA05F359410EE0A5F199
:10F7880020050EF1200E012A03FA0EFC28BF4CF0CA
:10F79800020C43FA05F3C01851EBE37101F0004580
:10F7A80007D54FF0000EDCF1000C7EEB00006EEB8D
:10F7B8000101B1F5801F1BD3B1F5001F0CD3490817
:10F7C8005FEA30004FEA3C0C04F101044FEA44526E
:10F7D80012F5800F80F09A80BCF1004F08BF5FEAF5
:10F7E800500C50F1000041EB045141EA050130BDD5
:10F7F8005FEA4C0C404141EB010111F4801FA4F178
:10F808000104E9D191F0000F04BF01460020B1FACC
:10F8180081F308BF2033A3F10B03B3F120020CDA04
:10F828000C3208DD02F1140CC2F10C0201FA0CF0E2
:10F8380021FA02F10CE002F11402D8BFC2F1200C47
:10F8480001FA02F120FA0CFCDCBF41EA0C019040FD
:10F85800E41AA2BF01EB0451294330BD6FEA040446
:10F868001F3C1CDA0C340EDC04F11404C4F1200231
:10F8780020FA04F001FA02F340EA030021FA04F343
:10F8880045EA030130BDC4F10C04C4F1200220FA9A
:10F8980002F001FA04F340EA0300294630BD21FAD8
:10F8A80004F0294630BD94F0000F83F4801306BF9E
:10F8B80081F480110134013D4EE77FEA645C18BF92
:10F8C8007FEA655C29D094EA050F08BF90EA020F29
:10F8D80005D054EA000C04BF1946104630BD91EA21
:10F8E800030F1EBF0021002030BD5FEA545C05D124
:10F8F8004000494128BF41F0004130BD14F5800463
:10F908003CBF01F5801130BD01F0004545F0FE41D6
:10F9180041F470014FF0000030BD7FEA645C1ABF0B
:10F92800194610467FEA655C1CBF0B46024650EA42
:10F93800013406BF52EA033591EA030F41F400216E
:10F9480030BD00BF90F0000F04BF0021704730B5F4
:10F958004FF4806404F132044FF000054FF00001C9
:10F9680050E700BF90F0000F04BF0021704730B58A
:10F978004FF4806404F1320410F0004548BF40425F
:10F988004FF000013EE700BF42004FEAE2014FEAB4
:10F9980031014FEA02701FBF12F07F4393F07F4F8F
:10F9A80081F06051704792F0000F14BF93F07F4FC1
:10F9B800704730B54FF4607401F0004521F0004104
:10F9C80020E700BF50EA010208BF704730B54FF08A
:10F9D80000050AE050EA010208BF704730B511F08F
:10F9E800004502D5404261EB41014FF4806404F1C7
:10F9F80032045FEA915C3FF4DCAE4FF003025FEA49
:10FA0800DC0C18BF03325FEADC0C18BF033202EBD0
:10FA1800DC02C2F1200300FA03FC20FA02F001FA2A
:10FA280003FE40EA0E0021FA02F11444C1E600BFC9
:10FA38004FEA4102B2F1E04324BFB3F5001CDCF108
:10FA4800FE5C0DD901F0004C4FEAC0024CEA507040
:10FA5800B2F1004F40EB830008BF20F0010070476F
:10FA680011F0804F21D113F13872BCBF01F0004072
:10FA7800704741F480114FEA5252C2F11802C2F1A4
:10FA8800200C10FA0CF320FA02F018BF40F0010025
:10FA98004FEAC1234FEAD32303FA0CFC40EA0C00D7
:10FAA80023FA02F34FEA4303CCE77FEA625307D114
:10FAB80050EA01331EBF4FF0FE4040F4400070474B
:10FAC80001F0004040F0FE4040F40000704700BFE5
:10FAD8007BB972B90029BEBF00204FF0004106E093
:10FAE80008BF00281CBF6FF000414FF0FF3000F046
:10FAF80073B882B0EC462DE9005000F03DF8DDF80F
:10FB080004E002B00CBC704707EE900AF5EEC07A2C
:10FB1800F1EE10FA01D400F009B808B580F0004001
:10FB280000F004F8404261EB410108BDD0B5FFF791
:10FB38002BFF00220E4B06460F4600F04FF800F050
:10FB48005FFA0446FFF7FEFE00220A4B00F046F873
:10FB580002460B4630463946FFF7B6FD00F050FA2C
:10FB68002346002242EA000210461946D0BD00BFD3
:10FB78000000F03D0000F0412DE9F041069C1546DB
:10FB880006460F46984600F05BFA05FB01F300FBBA
:10FB98000838A5FB0023B21A434467EB0303C4E902
:10FBA8000023BDE8F08100BF2DE9F041069C904696
:10FBB80006460F461D4600F091FB00FB05F5A0FB2D
:10FBC800082308FB0155B21A2B4467EB0303C4E969
:10FBD8000023BDE8F08100BF704700BF70B54FF04B
:10FBE800FF0C4CF4E06C1CEA11541DBF1CEA1355C1
:10FBF80094EA0C0F95EA0C0F00F0DEF82C4481EA29
:10FC0800030621EA4C5123EA4C5350EA013518BF48
:10FC180052EA033541F4801143F4801338D0A0FB35
:10FC280002CE4FF00005E1FB02E506F00042E0FBE2
:10FC380003E54FF00006E1FB03569CF0000F18BFE8
:10FC48004EF0010EA4F1FF04B6F5007F64F5407490
:10FC580004D25FEA4E0E6D4146EB060642EAC62123
:10FC680041EA55514FEAC52040EA5E504FEACE2E90
:10FC7800B4F1FD0C88BFBCF5E06F1ED8BEF1004F93
:10FC880008BF5FEA500E50F1000041EB045170BD0F
:10FC980006F0004646EA010140EA020081EA030153
:10FCA800B4EB5C04C2BFD4EB0C0541EA045170BD4F
:10FCB80041F480114FF0000E013C00F3AB8014F1C9
:10FCC800360FDEBF002001F0004170BDC4F1000412
:10FCD800203C35DA0C341BDC04F11404C4F1200593
:10FCE80000FA05F320FA04F001FA05F240EA0200EE
:10FCF80001F0004221F0004110EBD37021FA04F624
:10FD080042EB06015EEA430E08BF20EAD37070BDDD
:10FD1800C4F10C04C4F1200500FA04F320FA05F03C
:10FD280001FA04F240EA020001F0004110EBD3703E
:10FD380041F100015EEA430E08BF20EAD37070BDAE
:10FD4800C4F1200500FA05F24EEA020E20FA04F387
:10FD580001FA05F243EA020321FA04F001F0004136
:10FD680021FA04F220EA020000EBD3705EEA430EA7
:10FD780008BF20EAD37070BD94F0000F0FD101F0D6
:10FD88000046400041EB010111F4801F08BF013C0F
:10FD9800F7D041EA060195F0000F18BF704703F04D
:10FDA8000046520043EB030313F4801F08BF013DD4
:10FDB800F7D043EA0603704794EA0C0F0CEA135590
:10FDC80018BF95EA0C0F0CD050EA410618BF52EA4A
:10FDD8004306D1D181EA030101F000414FF0000050
:10FDE80070BD50EA410606BF1046194652EA43065E
:10FDF80019D094EA0C0F02D150EA013613D195EAD2
:10FE08000C0F05D152EA03361CBF104619460AD119
:10FE180081EA030101F0004141F0FE4141F4700123
:10FE28004FF0000070BD41F0FE4141F4780170BD13
:10FE380070B54FF0FF0C4CF4E06C1CEA11541DBF78
:10FE48001CEA135594EA0C0F95EA0C0F00F0A7F87A
:10FE5800A4EB050481EA030E52EA03354FEA0131A7
:10FE680000F088804FEA03334FF0805545EA1313BA
:10FE780043EA12634FEA022245EA111545EA106582
:10FE88004FEA00260EF000419D4208BF964244F119
:10FE9800FD0404F5407402D25B084FEA3202B61A38
:10FEA80065EB03055B084FEA32024FF480104FF40C
:10FEB800002CB6EB020E75EB030E22BFB61A754680
:10FEC80040EA0C005B084FEA3202B6EB020E75EB13
:10FED800030E22BFB61A754640EA5C005B084FEA7B
:10FEE8003202B6EB020E75EB030E22BFB61A754648
:10FEF80040EA9C005B084FEA3202B6EB020E75EB53
:10FF0800030E22BFB61A754640EADC0055EA060E13
:10FF180018D04FEA051545EA16754FEA06164FEA56
:10FF2800C30343EA52734FEAC2025FEA1C1CC0D102
:10FF380011F4801F0BD141EA00014FF000004FF08F
:10FF4800004CB6E711F4801F04BF01430020B4F150
:10FF5800FD0C88BFBCF5E06F3FF6AFAEB5EB030C08
:10FF680004BFB6EB020C5FEA500C50F1000041EB05
:10FF7800045170BD0EF0004E4EEA113114EB5C04D2
:10FF8800C2BFD4EB0C0541EA045170BD41F48011A5
:10FF98004FF0000E013C90E645EA060E8DE60CEAAD
:10FFA800135594EA0C0F08BF95EA0C0F3FF43BAFCA
:10FFB80094EA0C0F0AD150EA01347FF434AF95EA81
:10FFC8000C0F7FF425AF104619462CE795EA0C0F65
:10FFD80006D152EA03353FF4FDAE1046194622E732
:10FFE80050EA410618BF52EA43067FF4C5AE50EA0C
:08FFF80041047FF40DAF52EA51
:020000040801F1
:1000000043057FF4EBAE12E74A0011D212F500125D
:1000100011D20DD56FF47873B3EB62520ED44FEA60
:10002000C12343F0004343EA505323FA02F07047E0
:100030004FF00000704750EA013002D14FF0FF301E
:1000400070474FF00000704700292DE9F043C0F2DF
:10005000A6800026002BC0F29C80884694469E46CF
:10006000154604460F46002B3DD18A4259D9B2FAB3
:1000700082F33BB1C3F120029F4020FA02F29D407F
:1000800017439C40290C220CB7FBF1FEA8B201FBE0
:100090001E7742EA074700FB0EF3BB420AD97F19DD
:1000A0000EF1FF3280F00581BB4240F20281AEF1D9
:1000B000020E2F44FF1AA4B2B7FBF1F301FB137732
:1000C00044EA074700FB03F0B84208D97F1903F15F
:1000D000FF3280F0F080B84240F2ED80023B43EA0C
:1000E0000E43002203E08B420FD900221346341C3A
:1000F00018BF012460424FF0000565EB45015840F0
:10010000514000196941BDE8F083B3FA83F2002A37
:1001100040F086808B4202D3844500F2DB800123CD
:10012000E5E712B90123B3FBF2F5B5FA85F0002833
:100130003BD1781B4FEA154E1FFA85FC0122B0FB1C
:10014000FEF8210C0EFB180741EA07470CFB08F3E9
:10015000BB4207D97F1908F1FF3102D2BB4200F23E
:10016000BD808846FF1AA4B2B7FBFEF30EFB1377DF
:1001700044EA07470CFB03FCBC4507D97F1903F190
:10018000FF3102D2BC4500F2A7800B4643EA084388
:10019000ADE752426FEA060663EB43035DE7404278
:1001A00061EB41014FF0FF3654E7C0F1200224FA21
:1001B00002F107FA00F385404FEA154ED740194384
:1001C000B7FBFEF20B0C0EFB12771FFA85FC43EA1D
:1001D00007430CFB02F79F4204FA00F407D95B19AE
:1001E00002F1FF3074D29F4272D9023A2B44DF1BD6
:1001F00089B2B7FBFEF80EFB187341EA03430CFB10
:1002000008F79F4208D95B1908F1FF315CD29F4281
:100210005AD9A8F102082B44D81B48EA02428EE7BB
:10022000C2F120032CFA03F10EFA02FE20FA03F7C2
:1002300041EA0E0E08FA02F028FA03F14FEA1E45D1
:100240003843B1FBF5F8030C05FB18111FFA8EF7C4
:1002500043EA014107FB08F38B420CFA02FC09D97F
:1002600011EB0E0108F1FF3930D28B422ED9A8F1E3
:1002700002087144C91A80B2B1FBF5F305FB1311F2
:1002800040EA014107FB03F78F4208D911EB0E0149
:1002900003F1FF3016D28F4214D9023B714443EA76
:1002A0000843C91BA3FB0C89494509D305D000228B
:1002B0001DE79646FEE6134611E794404445F6D204
:1002C000013BF4E70346EAE78846A5E7C846D1E7DD
:1002D00002468CE713460AE7023B57E7A8F10208FB
:1002E0002F443FE72DE9F041002B44D18A421546C7
:1002F00004464FD9B2FA82F70E464FB1C7F1200338
:10030000B94020FA03F602FA07F50E4300FA07F4A3
:100310004FEA154E230CB6FBFEF0AFB20EFB106198
:1003200043EA014307FB00F1994209D95B1900F147
:10033000FF3280F0EC80994240F2E98002382B4491
:100340005A1AA4B2B2FBFEF30EFB132244EA024295
:1003500007FB03F7974208D9521903F1FF3180F0E8
:10036000D880974240F2D580023B43EA0040002605
:100370003146BDE8F0818B4247D8B3FA83F6002EB0
:1003800048D18B4202D3824200F2CD800120314617
:10039000BDE8F08112B90125B5FBF2F5B5FA85F893
:1003A000B8F1000F77D14A1B4FEA154EAFB20126C4
:1003B000B2FBFEF0230C0EFB102143EA014107FBC8
:1003C00000F38B4207D9491900F1FF3202D28B4268
:1003D00000F2BA801046C91AA4B2B1FBFEF30EFBBC
:1003E000131144EA014407FB03F7A74208D9641933
:1003F00003F1FF3280F08F80A74240F28C80023BF5
:1004000043EA00403146BDE8F081002630463146DF
:10041000BDE8F081C6F1200422FA04F5B3402B4375
:1004200020FA04FC01FA06F721FA04F54FEA134E0C
:100430004CEA0707B5FBFEF8390C0EFB18551FFAFE
:1004400083FC41EA05450CFB08F1A94202FA06F2D9
:1004500004D9ED1808F1FF3467D3A0466D1ABFB276
:10046000B5FBFEF40EFB145547EA05410CFB04FCFA
:100470008C4504D9C91804F1FF355CD32C4644EAF5
:100480000844CCEB0101A4FB0223994248D344D099
:10049000204600266CE7C8F1200401FA08F305FAAB
:1004A00008F520FA04F7E1404FEA154E1F43B1FB6F
:1004B000FEF63A0C0EFB16111FFA85FC42EA0143C8
:1004C0000CFB06F29A4200FA08F407D95B1906F110
:1004D000FF3137D29A4235D9023E2B449B1ABFB224
:1004E000B3FBFEF00EFB103347EA03430CFB00F1B5
:1004F000994207D95B1900F1FF3221D299421FD9E5
:1005000002382B445A1A40EA0646674650E710461E
:1005100016E70B4629E7134672E7B0409042B7D280
:10052000601E002624E7304622E7A94295D9A8F1AB
:1005300002081D4492E78C45A0D9023C19449EE76D
:100540001046DFE70E46C9E70238294443E700BFFB
:100550004FF0FF3C06E000BF4FF0010C02E000BF8F
:100560004FF0010C4DF804CD4FEA410C7FEA6C5C72
:100570004FEA430C18BF7FEA6C5C1BD001B050EA15
:10058000410C0CBF52EA430C91EA030F02BF90EA00
:10059000020F0020704710F1000F91EA030F58BFBF
:1005A000994208BF90422CBFD8176FEAE37040F021
:1005B000010070474FEA410C7FEA6C5C02D150EABF
:1005C000013C07D14FEA430C7FEA6C5CD6D152EA7A
:1005D000033CD3D05DF8040B704700BF844610463F
:1005E00062468C461946634600E000BF01B5FFF73E
:1005F000B7FF002848BF10F1000F01BD4DF808ED0E
:10060000FFF7F4FF0CBF012000205DF808FB00BFDE
:100610004DF808EDFFF7EAFF34BF012000205DF838
:1006200008FB00BF4DF808EDFFF7E0FF94BF012085
:1006300000205DF808FB00BF4DF808EDFFF7CEFF86
:1006400094BF012000205DF808FB00BF4DF808EDC5
:10065000FFF7C4FF34BF012000205DF808FB00BF96
:1006600011481249026800608A4218D0002103E054
:100670000F4B5B58435004310E480F4B42189A42BF
:10068000F6D30E4A02E0002342F8043B0C4B9A4298
:10069000F9D3FDF7DBFD00F019F87047FEE70948D4
:1006A000D0F800D040680047FC9F0020EFBEADDED0
:1006B000FC6E010800000020680100206801002095
:1006C000D826002000D8FF1FFEE700002DE9804853
:1006D0009FB0EFF759FDAC4DDFF810832B78D8F8B9
:1006E000004033B1A94B1B68E31A002BA4BF0023C1
:1006F0002B70FEF79DFF10B1A54B00221A70A54B81
:1007000019680B0740F18281A34B1B681B7A062BEB
:1007100000F27081DFE813F0070007003200CC0020
:100720000501300130019D4B1A78002A00F06281EA
:1007300000221A709A4B1F789A4B1B6893F800E0BE
:10074000994B93F800C00222984EB35C3B4103F0F2
:100750000F03734502F101090CD20B2B9FBFB05C54
:1007600016F8096000EA0C0006EB00209CBF904ED2
:1007700046F823000232102AE6D102E18D4B1A78A6
:10078000002A00F0378100221A708B4B8B4A93F8B5
:1007900002E0DF7858780EF0070640EA062007F0FE
:1007A0003F06760146EADE061060187956605E79EB
:1007B00093F806E0800040EA971006F0010740EA4F
:1007C00087209060DF790EF00F00C00140EA5600EC
:1007D00007F07F06D0603601187A46EA1E1693F8B5
:1007E00009E0166140000EF0030640EAD71040EA27
:1007F00046209F7A5061D87A07F01F06B601C000E4
:1008000046EA9E0640EA571093F80DE09F7BD061C0
:10081000187B96610EF0070640EA062007F03F06B7
:10082000760146EADE061062D87B56621E7C93F89B
:1008300011E0800040EA971006F0010740EA8720A7
:1008400090629F7C0EF00F00C00140EA560007F056
:100850007F06360146EA1E16D062D87C166393F8EE
:1008600014E0400040EAD7100EF003065F7D40EA36
:1008700046205063987DDB7D07F01F06B601C0005F
:1008800040EA571046EA9E06DF07D06396634CBFE6
:1008900040F21470AD209E0710644CBF40F21470FB
:1008A000AD2013F0080F506414BF03230123A2E00E
:1008B000434A1378002B00F09D804248424F06784F
:1008C0000023137007EB460E404A9EF80390B2F8DF
:1008D00000C09EF8042042EA0922944540F08A8034
:1008E0007A78012A04D0812A40F08580032300E031
:1008F0001346102E84BF102202700778344800225D
:10090000D6B2BE4200F1020075D210F802EC10F827
:10091000016C46EA0E26DFF8D8E02EF812600132AC
:10092000EEE72C4B1A78002A64D000221A702A4B6A
:100930001A78A82A1E465DD1DA7C002A5AD106EB25
:1009400042009FED267AC778037903EB072307EE71
:10095000903AF8EEE77A224BC7EE877A9FED217A3C
:1009600077EEC77AFCEEE77A17EE900A43F822009A
:100970000132082AE3D104E01B4B1A78D2B30022DB
:100980001A70012337E000BF7B0A002068010020B5
:100990007C0A00203026002070260020A91B0020A1
:1009A0005E240020582400205F240020991B002092
:1009B000901A00201A1C0020011C0020001B00209F
:1009C000D11B0020D41B0020D51B0020D21B0020EF
:1009D000D81B0020CA1B0020B51B0020CDCCCC406A
:1009E000C01A00200080BB438C1A0020AC260020D7
:1009F000E01A00200023D80741BF83F00203A34A76
:100A00000120C3F3400344BF10702B704A0406D585
:100A10009F4A13780BB1002010709C4A137044F267
:100A200008030B403BB1994B1B7823B104F5C3334A
:100A3000984AA0331360CB070CD5964B5A79187996
:100A400082421FBF01222A7004F5C332A0321CBFAC
:100A50001A6058718F0409D500238F4A32F8132089
:100A6000002A41F0D28501330C2BF6D1874B894DFA
:100A70001B7823B9894B1B68E31A002B0ADBAB6890
:100A8000E41A14F15A0F05D5F0F726FD814B012227
:100A90001A7321E12B697F4A0133002BC8BF002361
:100AA0000E06136140F118817D4E33683446A3B9B8
:100AB0002B7D013B042B00F20F81DFE813F01400C3
:100AC00014001400FD00C800754B1868FAF740FBCD
:100AD000F9F76BF908B1FCF7DFF92068FAF73BFB8F
:100AE0000028F1D1E4E76A6B6A4C92F80090B9F102
:100AF000000F03D0B9F1010F10D0EDE0012B00F28F
:100B0000EB80627D674B30680C2101FB02335A7821
:100B1000654B53F82210FAF718FB59E03068604F24
:100B2000FAF710FB002800F0D780237D022B3ED07F
:100B3000032B4AD0012B40F0CF805C4B1968E36A4D
:100B4000CB1AC72B40F2C880A36A042B2DD8554A74
:100B5000E1620C203C6800FB0323A0685E789646A7
:100B60000023514A52F823708742D9B204D001338E
:100B7000082BF6D1002300E00B46B34205D02046F7
:100B800052F82610FAF7E1FAA6E06A7D0C2303FB7F
:100B900002E35E6816F8011B19B12046FAF7DEFA87
:100BA000F8E7AB6A0133AB6296E0022092E0627D27
:100BB0003C4B38680C2101FB02335A783A4B53F80E
:100BC0002210FAF7C2FA032084E0636B9B780BB91A
:100BD00004207FE094F830300BB984F8309095F819
:100BE00030302C4C012B12D1A36AB22B0AD82D4ADB
:100BF0003068134493F83C10FAF7B0FAA36A013353
:100C0000A36204E00023A362022384F8303095F845
:100C10003030204C022B15D1A26A0F2A0FD8636BFB
:100C200020495B78306803EB03130B44134493F8BB
:100C3000F010FAF793FAA36A0133A36202E00323E8
:100C400084F8303095F83030022B45D9C0E7EB6995
:100C500010490133EB616B6BDB784BB14B7D01339A
:100C6000DBB20522B3FBF2F202EB82029B1A4B7558
:100C70000E4B1B682B620E4B00221A700D4A137824
:100C800023F002031370012024E000BF7C0A00203F
:100C9000EE100020680100206C1B0020500A00208C
:100CA000D81C0020EC340108B8520108542600205A
:100CB0000619002000190020C24B2A6A1B689B1AE3
:100CC00040F6C412934207D9BF4A136823F02003A9
:100CD00013600520F9F75AFBFAF7EEF9DFF824B3B1
:100CE000C8F8000017AEDBF80C30304698479DF886
:100CF0005C3033B9B54BAA681B689B1A642B01F1B1
:100D00007384DFF80493D8F80030D9F80020B04895
:100D1000B04C1344AB60B04B1F68DBF8043098470D
:100D200030B9A94B1B6813F0020300F06284C9E0DC
:100D3000A74894F838200146F6F7A0FCA74B1B887B
:100D4000002B77D0E36B1B7808EE103A04F1400BD0
:100D500000224C34A14B9E48B3F800E030F912C099
:100D6000BEF57A7F02BF0023CBF800302361DBF8A9
:100D700000306344CBF80030236907EE90CA01339A
:100D8000012B4FEA4201F8EEE77A236106D10023F6
:100D9000C4ED017AC4ED007AA3601BE0D4ED006AD3
:100DA00007EE103A37EEE66AB8EEC77A86EE077AB3
:100DB00036EE877AD4ED026A84ED017A77EEC77A4F
:100DC00084ED007AE6EE276AF0EE667AC4ED036AF7
:100DD000C4ED026A002343528148DFF800A20B529F
:100DE000BEF1010F31D123690790012BC3BF03F17D
:100DF000FF3300EE103AD4ED037A9FED7A0A0691A4
:100E0000C8BFB8EEC00A0592C8BF87EE800A01F0DD
:100E10003FFF059A0699079818EE103A63B1F8EE6D
:100E2000C87AB4EEE70AF1EE10FA05DD4FF47A73F2
:100E3000AAF8003000231AE0DBF800304FF47A7E85
:100E400003F5FA7393FBFEF343520132032A0BF1CD
:100E5000040B04F114047FF47DAFBAF800000128FC
:100E600001D1F5F7D5FDBAF80030013BE0E758496C
:100E70005B4831F8132030F81300121A21F81320C0
:100E80000133032BF3D14CE7FAF716F9DBF898306E
:100E90009FED557ACBF89000C31A07EE903AF8EE22
:100EA000677A524BCBF8980067EE877A5B68CBED98
:100EB000257A0BF19C009847C0B995F88E30013324
:100EC00085F88E3095F88E40DFF808B1002CDBD025
:100ED000012C40F086830BF1D401DBED336A9BEDEE
:100EE000347A00220BF1E00B8C460AE1404B0BF107
:100EF0009C001A780146F6F7C1FB3E4B1B88002B7D
:100F000042D0DBF8A42023463A493B4C0988B1F58E
:100F1000C87F04BF002144F823102E494FEA830BF9
:100F200001F19C0C54F80B003CF913E0704444F8B8
:100F30000B0000202CF8130022F813000133032BC0
:100F4000E2D12C4C2388012B1BD1D1F8A8304FF4CF
:100F5000C87EC83393FBFEF31380D1F8AC30C8339E
:100F600093FBFEF35380D1F8B030C83393FBFEF30C
:100F7000A3F580739380A7F85800A7F85A00F8F7F4
:100F8000A5FE2388013B23801C4B1B685C0740F1B6
:100F9000A3801B4B1B88322B38D1D5F8A4301A887C
:100FA000A5F8B4205A889B88A5F8B830B7F858300F
:100FB000A5F8BA30B7F85A30A5F8B620A5F8BC3075
:100FC00026E000BF54260020FC180020AC2600209C
:100FD00024110020680100203C110020C4260020BC
:100FE000F001002000000000BD37863530230020CE
:100FF000CA260020F60A0020100200203026002019
:10100000F80A002004220020E8210020002B44D010
:10101000D5F8A4B00023CD4ACD4C1288322ACD4A4F
:1010200004BF002142F823104FEA830C04F19C0E08
:1010300052F80C103EF91300014442F80C10002243
:101040002EF813202BF813200133032B1146E2D185
:10105000DFF8F8B2BBF80030012B19D1BE4A11708D
:10106000BE4A0C201370F5F7D3FCD4F8A430B4F8C2
:10107000B4201A80B4F8B6205A80B4F8B8209A8008
:10108000B4F8BA30A7F85830B4F8BC30A7F85A30E2
:10109000BBF80030013BABF80030B14B1A78DAB145
:1010A000D5F8A410002232201A70D5F8C03093FB76
:1010B000F0F30B80D5F8C43093FBF0F34B80D5F8F8
:1010C000C83093FBF0F3A3F580738B80A7F858200A
:1010D000A7F85A20F8F7FAFDD5F8A420B5F89C3007
:1010E00011885B1AA5F89C305188B5F89E305B1AC0
:1010F000A5F89E309288B5F8A0309B1AA5F8A030CC
:10110000DBE6934C974804F19C0333F8123020F847
:1011100012301BB207EE903A934BF8EEE77A33F9B0
:10112000123067EEA67A0132E1EC017A07EE903ACE
:10113000F8EEE77A032A67EE877AEBEC017AE0D1E2
:1011400004F1E00004F1EC010246CDF814C0FAF716
:1011500012FA04F1E00004F1F80108AAFAF70BFA18
:1011600008A894ED250A0146FAF71EFADDED094AB2
:10117000DDED087A9DED0A5A94ED444AD4ED433AE8
:1011800094ED413AB6EE007A64EE874A67EE875AEC
:1011900064EEA47A25EE075AE5EEA57A0BA801467F
:1011A000B7EE008AE5EE057A0EAA0DF1440BF0EEDB
:1011B000482AE7EEC72A65EE846AD4ED427AE2EE69
:1011C000A36A25EE236AE4EE836A23EEE57AB1EEA4
:1011D000452AE2EE276AA2EEA76AA4EEA77A67EE96
:1011E000E57AF1EE641AE2EE837AA1EE846AA2EE69
:1011F000847AE1EEA37AA5EE836AA5EE037AE2EEA5
:10120000047A84ED426AC4ED417AB1EE466AC4EDD7
:10121000436A84ED447AF1EE666AB1EE477A8DED69
:101220000D7A8DED0B6ACDED0C6AFAF7A4F994ED09
:10123000410A4E4814A9FAF7B7F90BA84B493246B0
:10124000FAF77AF9304614A95A46FAF794F90EA833
:1012500059463246FAF770F95A4644483146FAF789
:101260008AF9434BD4ED457A9DED137A1A78384CC0
:10127000DDF814C0B4EEE77AF1EE10FACCBF42F01C
:10128000080222F008021A70D5F818311A78F0EE28
:10129000489A04F590735AB3D4ED478A05931846DB
:1012A000B0EE680A14A9FAF77FF994ED4B8A04F1BD
:1012B000D400B0EE480A3146FAF776F9059B14A837
:1012C0001A463146FAF757F904F59870B0EE680AF5
:1012D00014A9FAF769F911A83146B0EE480AFAF7ED
:1012E00063F914A8314604F59872FAF744F909E055
:1012F0009CE8070083E807009BE8070004F5987462
:1013000084E80700D5ED367AD5ED356A95ED377A64
:101310000F4C67EEA77A0023E6EEA67AE7EE077A8F
:101320009FED147AF4EEC77AF1EE10FA06DC9FED29
:10133000127AF4EEC77AF1EE10FA21D5C5F8F8303A
:10134000C5F8FC30C5F800312DE000BFF80A0020D8
:101350006801002028020020FA0A0020F30A002079
:10136000F40A0020C61100202411002030360108A4
:1013700000190020B81E8D3F3D0A673F6F12833A67
:1013800004F5907004F5987104F1F802FAF7D4F8B6
:10139000D4ED257A1FED070A04F1F80080EE270A44
:1013A0000146FAF701F9B5F83C31DA4C01339BB24A
:1013B000B3F57A7FA5F83C312ED194ED420AD4EDF5
:1013C000416A94ED437AD4ED447A20EE000AA6EE09
:1013D000A60AA7EE070AA7EEA70A01F059FC89EEB4
:1013E000800A0023A4F83C31D4ED426A94ED437A9C
:1013F000D4ED447A94ED416A60EE266A20EE077AD5
:1014000060EE277A26EE000AC4ED426A84ED410AB6
:1014100084ED437AC4ED447AD5ED428A95ED44AA31
:1014200095ED41BAD5ED43AA9FEDBB9A68EECA7A15
:10143000B7EE007AEBEE2A7A77EEA77AF4EEE97A45
:10144000F1EE10FA0EDCFFEE006AF4EEE67AF1EE51
:1014500010FA24D4F4EE477AF1EE10FAC8BFF0EE99
:10146000477A01E0F0EE477A17EE900AFEF790FA1D
:1014700041EC100B01F0AAFB51EC100BFEF7DCFA6B
:1014800008EE100AB5EEC08AF1EE10FA09DD78EE2A
:10149000497AF5EEC07AF1EE10FA10DC23E09FED08
:1014A0009F8AF1EE487A77EEC97AF5EEC07AF1EECE
:1014B00010FAB5EEC08A13DDF1EE10FA06DD38EE53
:1014C000499ADFED977AB4EEE79A03E09FED947ABC
:1014D000F4EEC77AF1EE10FA4CBF0123002312E0BC
:1014E000F1EE10FA06DD38EE499ADFED8E7AB4EEB1
:1014F000E79A03E09FED8B7AF4EEC77AF1EE10FAEB
:10150000CCBF0123002353B1B0EE4A0AF0EE4B0AE0
:10151000F8F756F89FED84CA70EE008A41E02AEE93
:101520008A0A6AEEAABAABEE280AB0EE6B7A30EEFF
:10153000000AA8EEA87AB5EE400AF0EE007AF0EEC6
:10154000690AF1EE10FAE7EE670AB0EE679A04D185
:10155000F5EE400AF1EE10FA04D0F8F731F8B0EEEB
:1015600040CA01E09FED70CA28EEAA0AEAEE0ABA64
:10157000ABEE0A0AF0EE690A30EE000AEBEEC90A99
:10158000B5EE400AF1EE10FA04D1F5EE400AF1EEA4
:1015900010FA04D0F8F714F8F0EE408A01E0DFED1D
:1015A000628A9FED629A624C2CEE090A01F098FA69
:1015B00028EE090A208001F093FADFED5E7A5E4A98
:1015C000608068EEE78AFDEEE88ACDED058ABDF819
:1015D000143013F4004F18BF03F5B47313800023C5
:1015E00000E00123002285F88E20002B7FF46AACF6
:1015F00005E0A5F89C30A5F89E30A5F8A030F9F7D5
:101600005BFDD5F840214D4BDFED4D0AC8F80000D9
:10161000821A92B21A80D9F80030059307EE903AF8
:10162000F8EE677A474BC5F8400167EEA00A3446EA
:10163000C3ED000A444B03F1080E186859682746A9
:1016400003C7083373453C46F7D118689B88386058
:10165000BB80BDF868E03D4F002400213B460846B2
:1016600033F802CF36F8018023F802CC02310C297E
:101670001CFB0800F4D1364931F81430BB8113FB50
:101680000E034FF4807093FBF0F321F81430013413
:10169000032C07F10E07E0D107EE902A1D4CB5F898
:1016A0006E61B8EE670A04F5B8700121F7F74AFDDC
:1016B000BCEEC00A8DED050ABDF81430B6FBF3F69A
:1016C0002B7B771CBFB2A5F87871002B44D0B4F8FF
:1016D0007A8100230F481F4A00F5C27400F5BE7CD2
:1016E00032F813E034F813203CF8131024F813E018
:1016F000C2EB0E0911FB08F13AB291FBF2F24A4437
:101700002CF813200133042BE4D100230373A0F839
:101710007A6126E068010020DB0FC93FDB0FC9BFFB
:1017200035FA0E3C35FA0EBC000000004D3D0F446A
:1017300026260020E12E6542CC110020F810002062
:10174000BD3786358C1F00203C360108AC020020D6
:1017500024110020481B0020B4F87A31013BA4F882
:101760007A31B5F87A01B64A03B2002B4FF0000384
:1017700013DDB2F97841B34931F81320083112FB77
:1017800000F231F8131092FBF4F28A1AAE4921F8F4
:1017900013200133042BEED101E0A2F87A31F1F7E6
:1017A00003FDAA4BDFF81CA31B68A94E13F480139A
:1017B00000F092803388180600F1DA80A54B1B7880
:1017C00003F0040303F0FF07002B73D0A24AA34BDE
:1017D000117811B195F88C1139B1A1490020086038
:1017E00001211970002185F88C111B78DAF800406E
:1017F0001370032B05D120469A49542200F056FF5E
:1018000051E0012B06D154229648214600F04EFFAC
:10181000002202E0022B02D10122934B1A70934A5C
:1018200001231370924A1370924A00231360924A64
:101830001360924B1C60924B22781A708A4B914A2B
:101840001B78D05C904B914A1870854B20441A60ED
:1018500042788F4B07EE902AF8EEE77AB2EE047AE0
:10186000C7EE877AC27A9FED8B7AC3ED007A07EED6
:10187000902AF8EEE77A427DC7EE877A9FED867A66
:10188000C3ED017A07EE902AF8EEE77A67EE877AE1
:10189000C3ED027AFCEEE77A17EE903A4375002327
:1018A000C372F8F7A9FE8020F7F774FF012385F8CB
:1018B000E4315DE06A4CD4ED007AF5EE407AF1EE69
:1018C00010FA55D0F8F702FA00232360624B1F701C
:1018D000624B01221A704BE0328811063DD55E4AF8
:1018E0001178481E01285D482CD8694C634BD4ED13
:1018F000017A9FED687A1A68634B67EE877A1978E8
:101900009FED667AFCEEE77A114417EE903ACB72BF
:10191000D4ED027A67EE877AFCEEE77A17EE903A1A
:101920004B75537807EE903AF8EEE77A77EEA77AA0
:10193000FCEEE77A17EE903AD370D37A5373537D67
:10194000D37504E0032902D11370012301E0037869
:10195000013303708020F7F70DFF3E4B1B785A07C9
:1019600006D495F8E4311BB1354B012283F88C2164
:101970004B4B4C4C1B78DFF85081ABB1324BB3F979
:101980000620B4F898319A420EDC6379012B01D01D
:10199000192B02D194F8E62132B90E2B04D0082B72
:1019A0001CBF0023A8F80430DAF8003093F818714F
:1019B000002F00F0918033889B0700F08D809FED11
:1019C0003A8ADFED3A7A88EE088AB4EEE78AF1EED9
:1019D00010FA7BD9B7EE000A30EE480A01F058F948
:1019E0009FED337ADFED337AE8EE077A9FED327AB6
:1019F000A8EE277ADFED317AE8EE077A20EE270AA3
:101A0000D5ED7A7A20EE270A01F06AF8B0F5617F09
:101A1000A8BF4FF4617007EE900AB8EEE70ADFED59
:101A2000287A80EE270AF7F73DFE07EE907AF8EE67
:101A3000E77A27EE800A01F053F880B247E000BF52
:101A400068010020E4020020481B0020041100204F
:101A5000C4190020CC2600202026002000000020F1
:101A60002C260020F8020020212600202426002019
:101A7000402600203C26002038260020502600204A
:101A80002226002078530108232600200000A041D0
:101A90004426002000007A445555553F9A99993FB5
:101AA00001000020D8110020000000008FC2753C0A
:101AB000306E99BC2716983D843459BEA40DC93F99
:101AC000EFB6B0443C110020D01100200020B8F83F
:101AD00006301844A8F80600C04B1B689F0640F16A
:101AE0009980338803F03003002B00F09380BC4BC7
:101AF0001B78DE0740F18E80BA4BDFEDBB7AB3F97D
:101B00000030DFF828B308EE103AB8EEC88A28EEA5
:101B1000278AB0EE480AF7F7C5FDF0EE408AB0EE2E
:101B2000480AF7F71FFEB14B1B68D978B04BB0EEEF
:101B3000409AB2EE048A002948D0AE4AB3F9027046
:101B40005688079130B2381A06920593F8F770FC60
:101B50000799059B069AC1F10009484503DB8842B5
:101B6000A8BF084600E0484687191688B3F9000068
:101B7000059233B2BFB2C01A57800691F8F758FCED
:101B80004845059A04DB06998842A8BF0846814665
:101B90004E44B6B2168036B207EE106A3FB2B8EEC7
:101BA000C70A07EE907A28EEC07AF8EEE77A20EEC0
:101BB000090AA7EE897AA7EEA80A87EE087ABDEE91
:101BC000C77A17EE103AABF800301BE0B3F90220E9
:101BD000B3F9003000EE103A07EE102AB8EEC00A52
:101BE000B8EEC77A68EEC07A20EE090AE7EE097A05
:101BF000A7EE280AC7EE887AFDEEE77A17EE903A4C
